:020000040000FA
:200000000207B60200800402003F000200081B222222FF02008014FFFFFFFF0200801CFFA1
:20002000FFFFFF020080244653373530543220202020202020204C56312E30EB7002E722CB
:2000400089828A831410E704F593E022F593E49322BB0002F722BB8000500989828A838BC1
:20006000931593F022BC000BBE0029EF8DF084FFADF022E4CCF875F008EF2FFFEE33FEEC9A
:2000800033FCEE9DEC984005FCEE9DFE0FD5F0E9E4CEFD22EDF8F5F0EE008420D21CFEADD5
:2000A000F075F008EF2FFFED33FD4007985006D5F0F222C398FD0FD5F0EA22A3F8E0C5F033
:2000C00025F0F0E582158270021583E0C838F0E822BB0006F709A7F01922BB8000500D8985
:2000E000828A838B931593F0E5F0A3F022E88FF0A4CC8BF0A42CFCE98EF0A42CFC8AF0ED79
:20010000A42CFCEA8EF0A4CDA8F08BF0A42DCC3825F0FDE98FF0A42CCD35F0FCEB8EF0A40D
:20012000FEA9F0EB8FF0A4CFC5F02ECD39FEE43CFCEAA42DCE35F0FDE43CFC22EB9FF5F0F0
:20014000EA9E42F0E99D42F0E89C45F022E8600FEFC333FFEE33FEED33FDEC33FCD8F122D5
:20016000BB0006E9F802000332BB8000500C89828A838B9315930200017B22ECF0A3EDF035
:20018000A3EEF0A3EFF022EB700C87F009E608B5F019DFF6801589828A831410E70FF59383
:2001A000E0F5F0A3E608B5F002DFF5806AF593E493F5F0A3E608B5F05EDFF4805ACB701311
:2001C00088828C838B9387F009E493A3B5F048DFF580441410E71F88848C858B9589828ACD
:2001E00083F593758620E0F5F0E493A3A3B5F024DFF4DEF2801E88848C858B9589828A83F8
:20020000F593758620E493F5F0E493A3A3B5F004DFF3DEF17586007FFFB5F0020F22400245
:200220007F012202000187809488F0EF60010E4E60F0ED60EE1410E7EECB701288828C8370
:20024000F59387F009E0A3B5F0CDDFF680C91410E71E88848C858B9589828A83F593758682
:2002600020E0F5F0E0A3A3B5F0AADFF5DEF380A488848C858B9589828A83F593758620E47F
:2002800093F5F0E0A3A3B5F08BDFF4DEF28085EB7008E709F608DFFA801B89828A831410E7
:2002A000E70AF593E0A3F608DFFA8009F593E493A3F608DFF9ECFAA9F0EDFB2288F0EF601A
:2002C000010E4E60F088F0ED60C51410E7E7CB700E88828C838B93E709F0A3DFFA80D614AF
:2002E00010E71C88848C858B9589828A83F593758620E0F0A3A3DFFADEF875860080B68875
:20030000848C858B9589828A83F593758620E493F0A3A3DFF9DEF77586008099C5F0F8A3AF
:20032000E028F0C5F0F8E582158270021583E038F022ECF608EDF608EEF608EFF62290008E
:200340007004E0F54090007005E0F541854082854183E020E7077E007F00C2D72289428A6E
:20036000435407F54512000539E02402F54450020545120003E0053AE53A7002053BE54050
:200380002544F540E541354530E604C2E6242DF5411200040090007004E540F090007005A2
:2003A000E541F0AE45AF44D2D72290007010E020E61EA3EDF0A3E9F0A3EAF0EC5407D2E6EA
:2003C00090007010F00538E53870020539D2D7227C007D00C2D72290007010E0A2E6B32247
:2003E00075F001800375F0041200040078407F06900070921200052190007090E5F0F02217
:2004000090007090E0540770F7221200046D90007008742DF0900070107508101200045861
:20042000E490007004F090007006F0742D90007005F090007007F0751D10751C10751E008B
:20044000751F2D75832D758200E4F0753800753900753A00753B0022E4A808F0A3D8FC22F2
:20046000120005171200040A120004AB22900004A175080A79707860120005287518C075CD
:2004800019A8751A00751B647510C07511A87512007513017514FF7515FF7516FF7517006E
:2004A00022000B78667788C0A800649000706AE0440CF0229000706AE054F3F02290007017
:2004C0006AE04401F0229000706AE054FEF0229000706AE04402F0229000706AE054FDF0A0
:2004E000229000706AE04440F0229000706AE054BFF02290007000E04410F0229000700045
:20050000E054EFF02290007000E04420F02290007000E05420F0229000700AF000000000F0
:2005200022E6F008A3DFFA2289A0E493A3F208B800030989A0D508F222A3E58330E6037569
:20054000832D22754300754200754100754000754508754400120003E5754308754200758E
:200560004108754000754508754400120003E51200040090000000750910750800750B00D7
:20058000750A0012000638400B9000706CE04408F0D2D722C2D7227543007542007541000E
:2005A000754000754508754400120003E5754308754200754108754000754508754400129A
:2005C0000003E51200040090000000750910750800750B00750A00120006384051754310DA
:2005E000754200754110754000754508754400120003E575431875420075411875400075D5
:200600004508754400120003E51200040090001000750910750800750B10750A00120006F2
:2006200038400B9000706CE04418F0D2D722C2D722E6F008A3DFFA22A90B89A0A80AE49397
:20064000F5F0A3E265F0701008B800030989A01200067D50E9C2D722D2D722A90B89A0A88D
:200660000AE0F5F0A3E265F0701008B800030989A01200067D50EAC2D722D2D722E50860BA
:200680000A14F50845097007D2D72215091508C2D7229000700B7418F09000700C7420F0A2
:2006A00075A06022120006927824E2E2B408157400F21200072912000721120007071200B4
:2006C000070E802E22120006927816E2E2703708E2E2B4013178281200079C5029120007F9
:2006E0003912000779120007411200078178177402F27800E2E2FC4480F208E2E2FD7918FC
:200700007A20120003AA22781AE4F208F222782680F7E2E2F5F0E3E3F2E5F0F30809DAF2BF
:20072000227A04781C792080E9790878027A0680E1E2E2F30809DAF922780879027A0680EF
:20074000F0780879227A0680E8E4F309F3227A08E480037A04E4F309DAFC22E0F3A309E013
:20076000F3227A04E0F3A309DAFA227A0280027A04E2E2F0A308DAF922900070607A068041
:20078000E3781879227A0A8089E0F5F0E2E265F0700708A3DAF3D2D722C2D7229000706605
:2007A0007A0480E59000200AE0FEA3E08E8375820075814F732275C7AA75C755759D027856
:2007C0007FE4F6D8FD900000007F007E607D01E4F0A3DFFCDEFADDF875815212000517D239
:2007E0000D120004B41200040A12001F0812001F2412001158EF7004020008070200081566
:200800001200000FEF700EC20D120004AB1200000702000DF4D20D02008000300D040200FA
:20082000800CC0E0C0D075D00012001EBDD0D0D0E0320D0A20426C616E6B20436865636B2B
:20084000696E67002E2E2E5B6661696C5D0A002E2E2E5B6F6B5D0A000D0A205446333331E4
:2008600046553A536563746F722D62617365642832353620736563746F72732920466C61C3
:2008800073682045726173652028314D29002E2E2E5B6F6B5D2E00496C6C6567616C2066F4
:2008A00069726D77617265002E000D0A20496E76616C6964206669726D7761726520210057
:2008C0000D0A20466C617368206572726F722021000D0A2849503D200025752E00257529A8
:2008E000000D0A284D41433D200025782E00257829000D5446545020646F6E652E204A75DC
:200900006D7020307825782E0A001B5B324A000D0A436865636B204D6167696320436F643F
:20092000652E2E2E004F4B2121004661696C2121004387049000555574AAF090002AAA7440
:2009400055F09000555574A0F08F828E838D93E54AF05387FB229000262FEEF0A3EFF0E493
:200960007851F608F6D390002630E094009000262FE094005003010BE690002620E0FF94A6
:20098000094003010AA2EF705E9000262FE0FEA3E0FFD39400EE940040317851E6FC08E669
:2009A0007B012448F974203CFA1200003B643A601A90002630E024FFF09000262FE034FF56
:2009C000F0785206E61870C10680BEEF4E7003010BE6784E7601900026207401F0785206FA
:2009E000E618704F06804C90002620E0784EF6784EE6C39409504E90002630E09400900062
:200A0000262FE09400403E78510806E6188606700106147B012448F974203EFA1200003BA9
:200A2000FF784EE6062423F582E43426F583759300EFF090002630E024FFF09000262FE00C
:200A400034FFF080AA784EE690002620F0C394095003010BE69000261A7426F0A37423F0AE
:200A600012001AF3EF64014E700690002620F02212001AF3EF64044E7003010B977D027F7F
:200A80000112001AF79000261CEFF07D067C007F037E0012001AFB90002614EEF0A3EFF031
:200AA000807E9000261DE0FFA3E090002614CFF0A3EFF090002621E06066D390002630E0E2
:200AC00094009000262FE0940040559000261A7426F0A37421F078510806E6188606700140
:200AE00006147B012448F974203EFA1200003B90002622F090002630E024FFF09000262F5C
:200B0000E034FFF07D017C00E4FFFE12001AFB120016CCE490002621F09000261CE014F07B
:200B20009000261A7420F0A37448F0A3E0FF784F760008A607D37850E6940018E6940040B7
:200B400049D390002630E094019000262FE0940040387851E6FE08E6FF2401FDE43EFC1261
:200B6000001AFB120016CC7852740226F618E436F618E6161870011690002630E024FEF05D
:200B80009000262FE034FFF080AB7850E69000261CF0E61846700890002620F00109659051
:200BA00000262FE07004A3E06401702678510806E6188606700106147B012448F974203E6F
:200BC000FA1200003B90002621F0E49000262FF0A3F090002614E0FFA3E09000261DCFF0FD
:200BE000A3EFF00109652290002640EFF0A3EBF0A3EAF0A3E9F0ECF9EDFA30C90320C808DE
:200C000012001F5012001E4112001F3B90002640E044A0F5225322AF5322FEA21792C9D228
:200C2000C8C2C8A21692C9D2C8C2C8A21592C9D2C8C2C8A21492C9D2C8C2C8A21392C9D2DE
:200C4000C8C2C8A21292C9D2C8C2C8A21192C9D2C8C2C8A21092C9D2C8C2C8D218D2C9D255
:200C6000C8A2C99218C2C8301803010DEFAF018F22A21792C9D2C8C2C8A21692C9D2C8C2BD
:200C8000C8A21592C9D2C8C2C8A21492C9D2C8C2C8A21392C9D2C8C2C8A21292C9D2C8C282
:200CA000C8A21192C9D2C8C2C8A21092C9D2C8C2C8D218D2C9D2C8A2C99218C2C830180300
:200CC000010DEFAF028F22A21792C9D2C8C2C8A21692C9D2C8C2C8A21592C9D2C8C2C8A26E
:200CE0001492C9D2C8C2C8A21392C9D2C8C2C8A21292C9D2C8C2C8A21192C9D2C8C2C8A226
:200D00001092C9D2C8C2C8D218D2C9D2C8A2C99218C2C8301803010DEF12001F3B9000261C
:200D200040E044A0F5225322AF432201A21792C9D2C8C2C8A21692C9D2C8C2C8A21592C98D
:200D4000D2C8C2C8A21492C9D2C8C2C8A21392C9D2C8C2C8A21292C9D2C8C2C8A21192C9C5
:200D6000D2C8C2C8A21092C9D2C8C2C8D218D2C9D2C8A2C99218C2C83018028072D2C9D2B7
:200D8000C9D2C8A2C99217C2C8D2C9D2C8A2C99216C2C8D2C9D2C8A2C99215C2C8D2C9D242
:200DA000C8A2C99214C2C8D2C9D2C8A2C99213C2C8D2C9D2C8A2C99212C2C8D2C9D2C8A25C
:200DC000C99211C2C8D2C9D2C8A2C99210C2C8D2C9D2C8A2C99218C2C812000011900026A4
:200DE00041E0FBA3E0FAA3E0F9E5221200005112001F502275B0FB7F0A7E0012001A51EF3E
:200E0000784DF612001EE5900070FFE0784DF61200141D7E087FD1E4FDFC12000FF0E47805
:200E20004DF6784DE6FDC39403501E7E087FD974042DF582E43420F583759300E0FD7C00F4
:200E400012000FF0784D0680D97E087FDD90002007E0FD7C0012000FF07E087FE1E4FDFC97
:200E600012000FF0E4784DF6784DE6FDC39405501E7E087FEA74122DF582E43420F5837512
:200E80009300E0FD7C0012000FF0784D0680D97E087FEE90002017E0FD7C0012000FF07B92
:200EA000017A2079181200033E90002608EEF0A3EFF0D39424EE940040E590002026E0B4F9
:200EC000081FA3E0B4061A90002609E024F0F090002608E034FFF0120006C5784DA6078061
:200EE000BE90002026E0B408B6A3E0B400B19000202AE0FFA3E090002608CFF0A3EFF09059
:200F0000002034E0FCA3E0FDA3E0FEA3E0FF900020001200017BE4784DF6784DE6FF7C001B
:200F20007B012420F9EC3420FA1200003BFE740C2FF582E43420F583759300EEF006E6B417
:200F400006D890002028E064456003010E9F9000202EE0543F6003010E9F90002031E0B46A
:200F6000010E120006A4E490002608F0A3F0805190002031E0B411499000203EE07004A3FC
:200F8000E06445701690002609E024E4F090002608E034FFF0120012BB80269000203EE097
:200FA00064FC7004A3E064036003010E9F90002609E024E4F090002608E034FFF0120017E1
:200FC000D890002656E07003010E9F12001F5E9000200A741FF0A374FCF07E087FF2FD7CED
:200FE0001F12000FF0C2A9C2AF120007A4010E9F90002638EEF0A3EFF0A3ECF0A3EDF0909D
:20100000002638E475F001120000BB85F082F583759300E4939000263DF07003011157E0CE
:20102000642560030111389000263C740AF090002638E475F001120000BB85F082F5837531
:201040009300E49324DB7003011138800090002639E024FFF090002638E034FFF0900026C1
:2010600038E475F001120000BB85F082F583759300E4939000263DF0E0249D601424EE60C9
:201080001924FD60030111389000263C7410F080099000263BE0FF0111509000263E740AD6
:2010A000F09000263AE07002A3E0605A9000263CE0FBFD7C009000263AE0FEA3E0FF120019
:2010C0000065AA059000263AE0FEA3E0FFEBFD7C00120000659000263AEEF0A3EFF0D3EAC4
:2010E00064809489EA40052457FF80032430FF9000263EE014F02457F582E43426F583757B
:201100009300EFF0809B9000263EE0B40A047F30803E9000263EE0C3940A4003010FFFE0D8
:20112000FF04F074572FF582E43426F583759300E0FF12001F6780DA9000263DE0FF1200D8
:201140001F679000263DE0640A6003010FFF7F0D12001F67010FFF22E4FFFEFDFC90002671
:201160002F1200017BE490002633F07F0AFE12001A51EF12001EE57E097F0AE4FDFC1200EE
:201180000FF07E097F0FE4FDFC12000FF07FFC7EFF7D0F7C00900026341200017B9000261F
:2011A0002FE0F8A3E0F9A3E0FAA3E0FBC000C001C002C003A3E0FFE4FDFEA3A3E0F9A3E0A8
:2011C000FAA3E02FFFEE3AFEED39FDE42FFFE43EFEED3481FDA907AA06AB051200003BFFEE
:2011E000D003D002D001D000EB4FFFEAFEE9FDE8FC9000262F1200017B9000262FE0FCA3E7
:20120000E0FDA3E0FEA3E0FF78081200014D9000262F1200017B90002633E004F0E0C394A7
:2012200003500301119D9000262FE0F8A3E0F9A3E0FAA3E0FBC000C001C002C003A3E0FFED
:20124000E4FDFEA3A3E0F9A3E0FAA3E02FFFEE3AFEED39FDE42FFFE43EFEED3481FDA90798
:20126000AA06AB051200003BFFD003D002D001D000EB4FFFEAFEE9FDE8FC9000262F12009A
:20128000017B7F557EAA7D557CAA9000262FE0F8A3E0F9A3E0FAA3E0FBC31200013C700D1B
:2012A0007E097F25FDFC12000FF07F01227E097F2AE4FDFC12000FF07F002290002044E0C4
:2012C000FEA3E0FFEE600301141CEF24FD606404600301141C12001D5B9000203CE0FFA3A8
:2012E000E09000264CCFF0A3EFF09000203EE0FEA3E0FF9000264AEEF0A3EFF09000204429
:20130000E4F0A37404F0E4A3F0A3F09000203CEEF0A3EFF09000264CE0FFA3E09000203E46
:20132000CFF0A3EFF090002608E4F0A37404F0020015759000203EE0FEA3E0FF9000264AF5
:20134000E06E7003A3E06F600301141490002648E0FEA3E0FF90002046E0B50608A3E0B51F
:20136000070301141090002649E02401FF90002648E03400FE90002046E06E7003A3E06F82
:2013800060030114149000203CE0FFA3E09000264CCFF0A3EFF07E087FA8E4FDFC12000F85
:2013A000F0C390002609E09404FF90002608E09400FE120009569000262EE0702B9000268E
:2013C00017E0C3941450067E087FAA80047E087FC0E4FDFC12000FF07F047E0012001CEF51
:2013E000900026567401F02290002649E004F0700790002648E004F0C390002609E0940444
:2014000090002608E094025007900026567401F002001E83E490002608F0A3F022D2A9D299
:20142000AFE49000262FF0A3F09000262FE0FEA3E0FFC39402EE9400505BEF2404FFE43EAE
:20144000FE12001A5190002631EEF0A3EFF0E0FD90002630E025E0FB9000262FE033FA74C1
:20146000042BF58274203AF583759300EDF090002631E0FF74052BF58274203AF58375936C
:2014800000EFF090002630E004F0709D9000262FE004F08094E49000262FF0A3F0900026D7
:2014A0002FE0FEA3E0FFC39403EE9400505412001A5190002631EEF0A3EFF0E0FD900026C6
:2014C00030E025E0FB9000262FE033FA74122BF58274203AF583759300EDF090002631E0F0
:2014E000FF74132BF58274203AF583759300EFF090002630E004F070A49000262FE004F010
:20150000809BE4784EF6784EE6FF2404F582E43420F583759300E0FEEF2466FDE434708DA5
:2015200082F583759300EEF006E6B404D9E4784EF6784EE6FF2412F582E43420F58375939E
:2015400000E0FEEF2460FDE434708D82F583759300EEF006E6B406D99000706CE054FDF03C
:2015600090007001743FF0900070007410F0900070DAE4F02290002609E02408FE90002604
:2015800008E0340090002040F0A3CEF0E4A3F0A3F090002000E0FCA3E0FDA3E0FEA3E0FFD5
:2015A000900020381200017B90002004E0FCA3E0FDA3E0FEA3E0FF900020341200017B90A0
:2015C000002609E0241CF090002608E03400F0900020287445F0E4A3F09000202E7440F090
:2015E000E4A3F0A37410F0A304F090002608E0FFA3E09000202ACFF0A3EFF090002009E0F2
:2016000004F0700790002008E004F090002008E09000202CF090002009E09000202DF0E425
:2016200090002032F0A3F0900020187490F090002609E02412F090002608E03400F0C3A39C
:20164000E0944090002608E094005006E4F0A37440F090002018E054F8FE90002608E04E55
:20166000FFA3E090002018CFF0A3EFF0E4FF740C2FF582E43420F583759300E0FEEF7C00D5
:201680007B01241AF9EC3420FAEE120000510FEFB406DBE4FF74122FF582E43420F5837545
:2016A0009300E0FE74202FF582E43420F583759300EEF00FEFB406DD900020267408F0A36F
:2016C000E4F07B017A207918020003AA90002618EEF0A3EFF090002614E475F0011200008C
:2016E000BBAFF090002631F0A3EFF090002619E0FF9000262CF090002046E07004A3E06486
:2017000001600301178790002631E0FCA3E0FDC39427EC9400403CD3ED943AEC9400503378
:2017200090002617E004F08D828C83759300E4936F6006E49000262DF090002617E0B4146A
:20174000129000262DE07004A3F080079000262E7401F090002616E0702DA3E06414702702
:201760009000262EE06020E4F54B12000597120018C412001990EF70069000262EF02290BF
:201780000026167401F02290002631E0FEA3E04E7002054B9000262EE06401703A900026A5
:2017A00016E0640170319000262CE0FDF46028E54B7011C3EE9440401E90002631E0FEA3F6
:2017C000E0FF800F90002631E0FEA3E0FF9000262CE0FD12001C81227FF27ED27D077C0CF7
:2017E00090002054E0F8A3E0F9A3E0FAA3E0FBC31200013C60030118C390002046E0FEA3CE
:20180000E0FF64014E6007EF4E60030118C3E490002052F0A3F090002050E0FEA3E0FFEE9C
:2018200060030118C3EF24FB600B24FB6009240960030118C3802D78127C207D017B017AB5
:201840002079487E007F0612000229EF707590002608E4F0A37428F090002050E4F0A374E7
:201860000BF0800E12001DAE90002050E4F0A3740CF078487C207D017B017A2079127E0022
:201880007F06120002BC90002044E4F0A37402F0A3E4F0A304F09000204EE4F0A304F0901B
:2018A00000203EE0FEA3E0FF9000203CE0FDA3E0A3CDF0A3EDF09000203CEEF0A3EFF012E0
:2018C000001575227E087F58E4FDFC12000FF0E4F54BF525752608AE25AF26E4FCFDFB7A36
:2018E00010F9F8120000ED8F2A8E298D288C27A2AFE433F524C2AF4387049000555574AAF8
:20190000F090002AAA7455F0900055557480F074AAF090002AAA7455F0E47FFF7EFFFDFC99
:20192000AB2AAA29A928A827D31200013C401BE4252AFFE43529FEE5283401FDA907AA06D1
:20194000AB05743012000051800C852A828529837593007430F05387FBE52424FF92AFAE56
:2019600025AF26E4FCFDFB7A10F9F8120000ED12001B880526E52670020525C3E525940132
:2019800050030118D77E087F8EE4FDFC02000FF07E087F32E4FDFC12000FF0E4752702F5F7
:2019A00026F525F524E47F3FFEFDFCAB27AA26A925A824D31200013C4003011A43E4F52835
:2019C000F529E4FF7E40FDFCAB27AA26A925A824120000ED8F2D8E2C8D2B8C2AE4FCFDE56E
:2019E0002D2529F52DE52C3528F52CED352BF52BEC352AF52AE4252DFFE4352CFEE52B3428
:201A000081FDA907AA06AB051200003BF4600D7E087F44E4FD12000FF07F00220529E52972
:201A200070020528C3E52894404097E5272401F527E43526F526E43525F525E43524F52437
:201A40000119A57E087F4FE4FDFC12000FF07F012290002638EEF0A3EFF0E49000263FF0CC
:201A600090002639E025E0F090002638E033F0E49000263CF0A3F09000263CE0FEA3E0FF06
:201A8000C39402EE64809480505F90002639E02FF090002638E03EF09000263FE0FF90000A
:201AA0002638E0FCA3E0FD7B017A26793E12000BE79000263CE07002A3E09000263E700B5F
:201AC000E09000263AF0A3E4F0800CE0FF9000263AE0F0A3E04FF09000263DE004F0709714
:201AE0009000263CE004F0808E9000263AE0FEA3E0FF227D087F077C007E0090002631ECC8
:201B0000F0A3EDF0E4A3F0A3F0AD07AC06C390002632E09D90002631E09C40629000261AE8
:201B2000E0FEA3E08E837593002DF582E5833CF583759300E0F990002634E0C4F8540FC8D9
:201B400068F090002633E0C454F048F0E9D39439500BE9C39430FFE49400FE8013C3E99488
:201B600041FFE49400CF240ACF3400FE90002633E04EF0A3E04FF00DBD00010C808F900070
:201B80002633E0FEA3E0FF22900026361200017B752B01E4F52EF52F90002636A3E0FDA315
:201BA000E0FEA3E02400FFE43EFEED3481FDA907AA06AB051200003BF52C532C40E52B6035
:201BC0004090002636A3E0FDA3E0FEA3E02400FFE43EFEED3481FDA907AA06AB0512000051
:201BE0003BF52D532D40E52CB52D03E4F52B852D2C052FE52F7002052EB4FFC1E52EB4FFC9
:201C0000BCE52B7F0060027F01229000262FEBF0A3EAF0A3E9F0E490002637F0A3F09000D8
:201C2000263574FFF5F0120000BB45F0604690002632E0FBA3E0FAA3E0F91200003BFF90B1
:201C400000262FE0FBA3E0FAA3E0F990002637E475F001120000BBFCE925F0F9EA3CFAEF55
:201C60001200005160B890002633E475F0011200031C80AA9000262FE0FBA3E0FAA3E0F9A2
:201C80002290002633EEF0A3EFF0A3EDF0AF4BE4FCFDFEFBFA7901F8120000ED8F288E27B2
:201CA0008D268C2590002633E0FEA3E0FFE4FCFDE5282FF528E5273EF527ED3526F526EC8C
:201CC0003525F525A3E0F54AA2AFE433F524C2AFAF28AE27AD26AC2512000931AF28AE2794
:201CE000AD26AC2512001B88E52424FF92AF22900070007429F090002044E4F0A37405F09B
:201D0000A3EEF0A3EFF064044E7020900026327481F0A37408F0A37497F0A3E4F0A3741161
:201D2000F07B017A20794812001C0A9000264AE0FFA3E09000203CCFF0A3EFF09000264C13
:201D4000E0FFA3E09000203ECFF0A3EFF090002608E4F0A37415F002001575E490002648D6
:201D6000F0A3F090002000E0FCA3E0FDA3E0FEA3E0FF9000264E1200017BE49000264AF06B
:201D8000A3F0A3F0A3F090002656F09000262EF090002617F090002616F09000262D04F06A
:201DA000900070007421F0900070DAE4F0227B017A20796CE475F004120000D1740229F90B
:201DC000E43AFAE475F008120000D1740229F9E43AFA90002004E0FCA3E0FDA3E0FEA3E0F3
:201DE000FF12000160740429F9E43AFEC3E99444FFEE942090002608F0A3EFF0229000268E
:201E000067EEF0A3EFF0E4F54CD3ED9400EC9400402C90002667E0FEA3E0AA06F97B811261
:201E200000003B254CF54CED1D70011C90002668E004F070D490002667E004F080CBAF4CB1
:201E400022E4FFFE90002644F0A304F0A3E4F0A37402F07D037C0090002646E0FBA3E09098
:201E6000002644CBF0A3EBF0A3ECF0A3EDF090002644E0FCA3E0FD0FBF00010EBE27D8BF11
:201E800010D52290002044E4F0A37404F09000264AE0FFA3E09000203CCFF0A3EFF0900049
:201EA000264CE0FFA3E09000203ECFF0A3EFF090002608E4F0A37404F002001575C0D0C2A4
:201EC000A9C2AFE5492401F549E43548F548E43547F547E43546F546758C5D758A3DD2AF68
:201EE000D2A9D0D0227598504387805389CF438920EFB40108758DF3758CF38006758DE565
:201F0000758CE5D28ED29922E58954F04401F589758C5D758A3DE4F549F548F547F546D237
:201F2000B9D28C227598504387805389CF438920758DE5758CE5D28ED29922D2C9D2C81229
:201F4000000011C2C912000011C2C81200001122C2C9D2C812000011D2C90200001190006D
:201F6000706CE054E7F0223099FDC2998F9922FFFFFFFFFFFFFFFFFFFFFFFFFFFFFFFFFFFE
:201F8000FFFFFFFFFFFFFFFFFFFFFFFFFFFFFFFFFFFFFFFFFFFFFFFFFFFFFFFFFFFFFFFF61
:201FA00075C7AA75C755759D02787FE4F6D8FD900000007F007E607D01E4F0A3DFFCDEFA5B
:201FC000DDF875815212000517C20D120004B41200040A12001F0812001F24C20D1200048A
:201FE000AB02000DF4FFFFFFFFFFFFFFFFFFFFFFFFFFFFFFFFFFFFFFFFFFFFFF020007B68B
:2020000002002724E5242445F582E43420F583759300E005242290002042301704900020BA
:2020200045E475F00112002673020024622010E57F2ED2108018EF540F2490D43440D4FF81
:2020400030140BEF24BFB41A0050032461FFE525600215250528E528700205273017119054
:20206000002042E475F00112002673EF0200247802003EF77403D2178003E4C217F52490FC
:202080000020421200268AE4F525F527F528E52560087F201200204E80F47526FFC211C2B1
:2020A00010C212C213C215C216C21812002016FF700E3017067F001200205FAF28AE2722EE
:2020C000B42563C2D5C21412002016FF24D0B40A00501A75F00A782530D50508B6FF01061A
:2020E000C6A426F620D5047002D21380D824CFB41A00EF5004C2E5D2140200228CD211800E
:20210000C4D21080BED21280BAD2D580B8D21580B27F201200204E2012077401B5250040DE
:20212000F012002004FF1200204E0200208ED218D216808F12002004FB12002004FA1200F6
:202140002004F94A4B700679637A237B8120123DE52560397E00E9C0E02EF9EAC0E03400E4
:20216000FA12002462F9D0E0FAD0E0C960060EEE652670E2C2D5EBC0E0EAC0E0E9C0E0EE4F
:20218000120022D4D0E0F9D0E0FAD0E0FB12002462FF6096EBC0E0EAC0E0E9C0E0120020DC
:2021A0004ED0E02401F9D0E03400FAD0E0FBE5260460DAD526D70200212A7BFF7A2279D0B3
:2021C000D2128089791080027908C216C2188008D2D5790A8004790AC2D5E526047002F50E
:2021E00026E4FAFDFEFF12002004FC7B0820111612002004FD7B1030100C12002004FE1295
:20220000002004FF7B20EC3382D592D55013C3E43010069FFFE49EFEE42011039DFDE49C83
:20222000FCE4CBF8C211EC700CCFCECDCCE824F8F870F38017C3EF33FFEE33FEED33FDEC88
:2022400033FCEB33FB994002FB0FD8E9EB301105F8D0E0C448B211C0E00AEC4D4E4F7820D0
:202260007B0070C2EAB5260040BCC0E0120022D6D0F0D0E0201104C4C0E0C4B211C0F012F4
:20228000002037D0F0D5F0EA0200208E1200269321345321C45821014C20FD4221C84F21F2
:2022A000D04421D04921174321D65521BA4621BA4521BA4723805021052D21092E21302B8C
:2022C000210D23212E20236C2A20C348000021263F3F3F00790AA2D5201314301509B910FE
:2022E000020404B9080104A2D520160250010420126D9212B525005036C0E07F2030131ACB
:202300007F30A2127216721550101200232FC212C216C215C2187F308010301503E9C0E01A
:202320001200204E301503D0E0F9D0E0B525CA3015197F30B9100D1200204E7F5830140753
:202340007F788003B908041200204E3012067F2D0200204E7F202018F77F2B2016F2229206
:202360001280CC286E756C6C2900D211120020043011F7C211782530D50108F6020020C349
:20238000120020047F4960087F4310E7027F5814C0E0EF1200203F743A1200203FD0E06002
:2023A0000DC0E0C412002037D0E012002037D213752504020021C4EB7008E709F608DFFA96
:2023C000801B89828A831410E70AF593E0A3F608DFFA8009F593E493A3F608DFF9ECFAA9C3
:2023E000F0EDFB2288F0EF60010E4E60F088F0ED60C51410E7E7CB700E88828C838B93E78C
:2024000009F0A3DFFA80D61410E72A89828A83F593ECFAE0A3C8C582C8CCC583CCCBC593D9
:20242000CBF0A3C8C582C8CCC583CCCBC593CBDFE2DEE080AA89828A83F593ECFAE493A350
:20244000C8C582C8CCC583CCCBC593CBF0A3C8C582C8CCC583CCCBC593CBDFE1DEDF020020
:2024600023DFEB7002E72289828A831410E704F593E022F593E49322BB0002F722BB800011
:20248000500989828A838B931593F022BC000BBE0029EF8DF084FFADF022E4CCF875F00882
:2024A000EF2FFFEE33FEEC33FCEE9DEC984005FCEE9DFE0FD5F0E9E4CEFD22EDF8F5F0EEA6
:2024C000008420D21CFEADF075F008EF2FFFED33FD4007985006D5F0F222C398FD0FD5F0EE
:2024E000EA22A3F8E0C5F025F0F0E582158270021583E0C838F0E822EB7007E7F5F009E79B
:20250000192289828A831410E708F593E0F5F0A3E022F593E493F5F074019322BB0006F79D
:2025200009A7F01922BB8000500D89828A838B931593F0E5F0A3F022CFF4CFCEF4CECDF4ED
:20254000CDCCF4CC22C3E49FFFE49EFEE49DFDE49CFC22E8600FECC313FCED13FDEE13FE0E
:20256000EF13FFD8F122E8600FEFC333FFEE33FEED33FDEC33FCD8F122EB7006E9F80200AE
:20258000261689828A831410E706F59302002622F5930200262EBB0006E9F802002667BB3A
:2025A0008000500C89828A838B931593020025CE22EB7006E9F80200263E89828A83141066
:2025C000E706F5930200264BF59302002657ECF0A3EDF0A3EEF0A3EFF022D093D083D08283
:2025E000E4937012740193700DA3A393F8740193F5828883E4737402936C70127403936D3D
:20260000700C7404936E70067405936F60DDA3A3A3A3A3A380CAE6FC08E6FD08E6FE08E6D4
:20262000FF22E0FCA3E0FDA3E0FEA3E0FF22E493FC740193FD740293FE740393FF22E6FB6D
:2026400008E6F908E6FA08E6CBF822E0F8A3E0F9A3E0FAA3E0FB22E493F8740193F9740281
:2026600093FA740393FB22ECF608EDF608EEF608EFF622F8E0FBA3A3E0F925F0F0E582156B
:202680008270021583E0FA38F022EBF0A3EAF0A3E9F022D093D083D082F8E4937012740126
:2026A00093700DA3A393F8740193F5828883E4737402936860EFA3A3A380DF736D692D31A9
:2026C0000A00736D692D320A00736D692D330A00736D692D340A00736D692D350A00736D42
:2026E000692D360A00736D692D370A00442086000000015C206A000000000000000000007C
:202700000000000000000000000000000000000000000D0A5B5048595F49442578003D256B
:20272000785D0A000200405E12003C8B120033AC7F017E007D197C009000202D120025CE5E
:20274000E47F3F7E28FDFC90002031120025CEE4FF12003D7EE4FFFE7D17FC900020191256
:202760000025CE9000201D7406F0A37401F0E47F01FEFDFCA3120025CEE4FF12002E91E48C
:20278000FFFE7D18FC90002019120025CE9000201D7406F0A37401F0E47F01FEFDFCA3128E
:2027A0000025CEE4FF12002E917F017E007D177C0090002019120025CE9000201D740AF05B
:2027C000A37401F0E47F01FEFDFCA3120025CEE4FF12002E917F017E007D187C009000207B
:2027E00019120025CE9000201D740AF0A37401F0E47F01FEFDFCA3120025CEE4FF12002E52
:202800009190002002E4F0A304F090002002E0FEA3E0FFC39407EE6480948040030128A0A8
:20282000EE3395E0FDFC781012002566EF4401FFED4410FDEC9000202D120025CEE47F3210
:202840007EC9FDFC90002031120025CEE4FF12003D7E90002002E0FEA3E0FFEE3395E0FDFD
:20286000FC781012002566EF4404FFED4410FDEC9000202D120025CEE47F7F7E01FDFC900B
:20288000002031120025CEE4FF12003D7E90002003E004F0700790002002E004F001280A7B
:2028A0007F1C7E007D1B7C009000202D120025CEE47F0AFEFDFC90002031120025CEE4FFDC
:2028C00012003D7E7F047E007D1B7C0090002019120025CE9000201D740EF0A37401F0E41D
:2028E000FFFEFDFCA3120025CEE4FF12002E91E4FFFE7D1BFC9000202D120025CE9000207F
:20290000317401F0A37420F0A37404F0E4FF12003B6290002004A3A3E0FEA3E4FFEE54407D
:20292000FEE4FDFCEE70C8FE120034A490002002E4F0A37407F090002003E0FF90002008D0
:20294000F07B017A2079097D1612003E5490002009E0547FF0A3E0F090002009E0F0A3E0DD
:202960004403F090002008E0FFA3E0FAA3E0FB7D1612003F80900020097471F0A37477F01E
:2029800090002008E0FFA3E0FAA3E0FB7D1012003F8090002008E0FF7B017A2079097D118A
:2029A00012003E5490002009E0F0A3E0540FF090002009E0F0A3E04430F090002008E0FF0D
:2029C000A3E0FAA3E0FB7D1112003F8090002008E0FF7B017A2079097D1612003E549000A7
:2029E0002009E04480F0A3E0F090002008E0FFA3E0FAA3E0FB7D1612003F8090002003E01E
:202A000004F0700790002002E004F0C390002003E0940990002002E06480948050030129CB
:202A2000367D017C00E4FFFE120034A4E4FFFE7D17FC9000202D120025CEE47FC67E1EFD86
:202A4000FC90002031120025CEE4FF12003D7EE4FFFE7D18FC9000202D120025CEE47FC667
:202A60007E1EFDFC90002031120025CEE4FF12003D7E90002000E4F0A304F090002001E07F
:202A8000FFC0077F047E007D197C0090002019120025CE9000201D7407F0A37402F0E47FEB
:202AA00002FEFDFCA3120025CED00712002E9190002001E0FFC0077F017E007D197C0090D6
:202AC000002019120025CEE49000201DF0A37406F0E47F3EFEFDFCA3120025CED0071200E1
:202AE0002E9190002001E0FFC0077F067E007D197C009000202D120025CEE47FFF7E04FDE8
:202B0000FC90002031120025CED00712003D7E90002001E0FFC0077F0A7E007D1B7C00902D
:202B2000002019120025CE9000201D7403F0A37401F0E47F01FEFDFCA3120025CED007122F
:202B4000002E9190002001E0FFC0077F057E007D197C0090002019120025CE9000201D743C
:202B60000FF0A37401F0E47F01FEFDFCA3120025CED00712002E9190002001E004F07007A7
:202B800090002000E004F0C390002001E0940790002000E0648094805003012A7B7F047E40
:202BA000007D197C0090002019120025CE9000201D7408F0A37401F0E4FFFEFDFCA3120065
:202BC00025CEE4FF12002E91E490002000F0A3F0E490002002F0A3F090002002E0FCA3E00D
:202BE000FDC3940AEC648094804003012CB790002001E0FFC007AF05AE04EE3395E0FDFC20
:202C0000781012002566EF4408FFED4410FDEC90002019120025CE9000201D740AF0A3740B
:202C200002F0E4FFFEFDFCA3120025CED00712002E9190002003E0FF74017E00A8070880BC
:202C400005C333CE33CED8F9F4FFEEF45407FE3395E0FDFC90002004120025CE90002001A0
:202C6000E0FFC007A3E0FEA3E0FFEE3395E0FDFC781012002566EF4406FFED4410FDEC9005
:202C800000202D120025CE90002004E0FCA3E0FDA3E0FEA3E0FF90002031120025CED00712
:202CA00012003D7E90002003E004F0700790002002E004F0012BD890002001E004F07007C3
:202CC00090002000E004F0C390002001E0940790002000E0648094805003012BD0229000F8
:202CE0002037EFF0A3EDF0A3EBF090002037E075F02FA4FFAEF02495F974403EFA7B811258
:202D000000246264026003012E68120038DEEF640160097B817A2679BB012E87900020387A
:202D2000E075F020A4FFE5F04488FEA3E0FDED4FFFEE44109000203DF0A3EFF090002037A9
:202D4000E075F02FA42496F9744035F0FA7B8112002462FF9000203DE0FAA3E0FBE4FD120A
:202D6000003C2EEF60097B817A2679C2012E879000203F7403F0A374E8F090002037E07583
:202D8000F02FA42496F9744035F0FA7B8112002462FF7B017A20793DE4FD1200365CEF60B7
:202DA000097B817A2679C9012E879000203DE0A330E769E490002041F090002041E004F0FC
:202DC000E0B402F59000203F74FFF5F0120024E2FEC3E5F09401EE940050097B817A2679EE
:202DE000D0012E8790002037E075F02FA42496F9744035F0FA7B8112002462FF7B017A201F
:202E0000793DE4FD1200365CEF60087B817A2679D780749000203DE0A320E7A8900020373A
:202E2000E075F02FA42496F9744035F0FA7B8112002462FF7B017A20793D7D011200365C73
:202E4000EF60087B817A2679DE803C9000203DE0F9A3E0FF9000203AE0FBA3E0FAA3E0C996
:202E60008FF01200251C802690002038E0FFA3E0FDA3E0FBA3E0FAA3E0F91200365CEF6029
:202E80000D7B817A2679E51200207A7F01227F002290002018EFF0C007A3E0FCA3E0FDA32C
:202EA000E0FEA3E0FF9000202D120025CE900020317401F0A37420F0A37423F0D007120050
:202EC0003B629000202BEFF06003E0FF229000201DE0F9FFA3E0FB2FFFE433FEC3EF94206B
:202EE000EE648094804012E47F01FEFDFCA80112002566120025458044E47F01FEFDFC90CE
:202F000000201DE02BF9F812002566C004C005C006C007E47F01FEFDFCE0F9F812002566FC
:202F2000A804A905AA06AB07D007D006D005D004C3EF9BFFEE9AFEED99FDEC98FC900020FA
:202F400027120025CE90002023E0F8A3E0F9A3E0FAA3E0FBA3E0FCA3E0FDA3E0FEA3E0FF21
:202F600012002538EB5FFFEA5EFEE95DFDE85CFC90002023120025CE90002023E0F8A3E0CA
:202F8000F9A3E0FAA3E0FBC000C001C0029000201FE0FCA3E0FDA3E0FEA3E0FF9000201DFF
:202FA000E0F9F81200256690002027E0F8A3E0F9A3E0FAA3E05FFFEA5EFEE95DFDE85CFC51
:202FC000D002D001D000EB4FFFEA4EFEE94DFDE84CFC90002023120025CE90002019E0FC2F
:202FE000A3E0FDA3E0FEA3E0FF9000202D120025CE90002023E0FCA3E0FDA3E0FEA3E0FF3A
:2030000090002031120025CE90002018E0FF12003D7E9000202BEFF02290002012EEF0A337
:20302000EFF0A3ECF0A3EDF090002012E475F001120024E285F082F583759300E493900010
:203040002017F07003013180E06425600301316190002016740AF090002012E475F0011273
:203060000024E285F082F583759300E49324DB7003013161800090002013E024FFF0900091
:203080002012E034FFF090002012E475F001120024E285F082F583759300E4939000201722
:2030A000F0E0249D601424EE601924FD6003013161900020167410F0800990002015E0FF02
:2030C00001317990002018740AF090002014E07002A3E0605A90002016E0FBFD7C00900012
:2030E0002014E0FEA3E0FF1200248CAA0590002014E0FEA3E0FFEBFD7C001200248C9000F1
:203100002014EEF0A3EFF0D3EA64809489EA40052457FF80032430FF90002018E014F0240E
:20312000B3F582E43420F583759300EFF0809B90002018E0B40A047F30803E90002018E034
:20314000C3940A4003013028E0FF04F074B32FF582E43420F583759300E0FF12003EF78074
:20316000DA90002017E0FF12003EF790002017E0640A60030130287F0D12003EF70130288B
:20318000229000209AEFF0FBA3E0FCA3E0FDA3A3E4FFFEEC781012002553900020A2EEF095
:2031A000A3EFF09000209BE0FCA3A3E0FEA3E0FF900020A4EEF0A3EFF0AF03900020A2E028
:2031C000FAA3E0FB7D0412003C2EEF6001229000209AE0FF900020A4E0FAA3E0FB7D05129F
:2031E000003C2EEF600122900020A87464F09000209AE0FF7B017A2079A67D1F1200365C35
:20320000EF600122900020A8E014F0C3940150037F0122900020A7E030E0D39000209AE06F
:20322000FF7B017A2079A27D061200365CEF6001229000209AE0FF7B017A2079A47D0712D3
:2032400000365CEF600122900020A2E0FEA3E0FFE4FCFD9000209FE0FBA3E0FAA3E0F912A6
:203260000025969000209FE0FBA3E0FAA3E0F912002579781012002566120025969000201E
:203280009FE0FBA3E0FAA3E0F9C003C002C001120025B1900020A4E0FEA3E0FFEB4FFFEAB6
:2032A0004EFEE9FDE8FCD001D002D003120025967F00229000208AEFF0FBA3E0FCA3E0FD01
:2032C000A3A3E4FFFEEC78101200255390002093EEF0A3EFF09000208BE0FCA3A3E0FEA348
:2032E000E0FF90002095EEF0A3EFF0AF0390002093E0FAA3E0FBE4FD12003C2EEF6001222E
:203300009000208AE0FF90002095E0FAA3E0FB7D0112003C2EEF6001229000208FE0FCA3CD
:20332000E0FDA3A3E4FFFEEC781012002553A3EEF0FAA3EFF0FB9000208FE0FCA3A3E0FE54
:20334000A3E0FF90002095EEF0A3EFF09000208AE0FF7D0212003C2EEF6001229000208A86
:20336000E0FF90002095E0FAA3E0FB7D0312003C2EEF600122900020997464F09000208A18
:20338000E0FF7B017A2079977D1F1200365CEF60012290002099E014F0C3940150037F011E
:2033A0002290002098E030E1D37F0022E49000200BF0A3F0E490002010F0A3F09000200C39
:2033C000E0C454F044079000200FF0E49000200DF0A3F090002010E064017004A3E0644146
:2033E000606C9000200BE0FEA3E0FF4E702BFDFC120034A49000200FE0FF7B017A207910DD
:203400007D0212003E549000200BE0FEA3E0FF7D017C00120034A480129000200FE0FF7BDF
:20342000017A2079107D0212003E0D9000200EE004F070079000200DE004F0C39000200E71
:20344000E094089000200DE06480948040859000200DE07004A3E0640A70227E277F12903C
:2034600000200BE0FCA3E0FD120030197E277F1E90002010E0FCA3E0FD1200301990002001
:203480000CE004F070079000200BE004F0C39000200CE094079000200BE064809480500366
:2034A0000133B42290002012EEF0A3EFF0ED4C606DE0FFC0077F047E007D1B7C009000206F
:2034C00019120025CE9000201D740EF0A37401F0E47F01FEFDFCA3120025CED00712002E6D
:2034E0009190002013E0FFC0077F047E007D1B7C009000202D120025CE900020317401F095
:20350000A37420F0A37414F0D00712003B6290002014A3A3E0FEEE5440FEEE60C4229000B7
:203520002013E0FFC0077F047E007D1B7C0090002019120025CE9000201D740EF0A3740178
:20354000F0E4FFFEFDFCA3120025CED00712002E9190002013E0FFC0077F047E007D1B7CD3
:20356000009000202D120025CE900020317401F0A37420F0A37414F0D00712003B629000CB
:203580002014A3A3E0FEEE5440FEEE70C42290002035EFF0A3EDF0A3EBF090002035E07513
:2035A000F02FA4FFAEF02495F974403EFA7B811200246264026003013640120038DEEF64BE
:2035C0000160037F012290002035E075F02FA42496F9744035F0FA7B8112002462FF90003F
:2035E0002038E0FAA3E0FB7D0112003C2EEF60037F012290002036E075F020A4FFE5F04426
:2036000084FEA3E0FDED4FFFEE44109000203AF0A3EFF090002035E075F02FA42496F974AB
:203620004035F0FA7B8112002462FF9000203AE0FAA3E0FBE4FD12003C2EEF601C7F0122EC
:2036400090002036E0FFA3E0FDA3E0FAA3E0FB12003C2EEF60037F01227F00229000204821
:20366000EFF0A3EDF0A3EBF0A3EAF0A3E9F0E4F5F01200251C9000204F7405F09000708070
:20368000E054FEF090002048E090007082F090002049E090007083F07DE87C03900070800E
:2036A000E0FF20E709ED1D70011C144C70EEED4C606990007085E09000204DF090007084EE
:2036C000E09000204EF09000204DE0FF9000204AE0FBA3E0FAA3E0F9E48FF01200251C902C
:2036E00000204AE0FBA3E0FAA3E0F9120024F875F0001200251C9000204AE0FBA3E0FAA3B1
:20370000E0F9120024F8FF9000204EE0FDEF4DFFE5F08FF01200251C7F00229000204FE066
:2037200014F0600301367C7F012290002006EBF0A3EAF0A3E9F090002005EFF0C394075001
:203740003AE0FF74017E00A807088005C333CE33CED8F9FFEE3395E0FDFC90002086E0F8EF
:20376000A3E0F9A3E0FAA3E05FFFEA5EFEE95DFDE85C4D4E4F60047F0180027F00EF700371
:203780007F012290002006E0FBA3E0FAA3E0F974011200247890002005E075F02FA4249653
:2037A000F9744035F0FA7B8112002462FF90002009E0FBA3E0FAA3E0F9EF120024787F0001
:2037C00022900020D6EDF0A3EBF0A3EAF0A3E9F0900020D5EFF0C39407503AE0FF74017ECF
:2037E00000A807088005C333CE33CED8F9FFEE3395E0FDFC90002086E0F8A3E0F9A3E0FA62
:20380000A3E05FFFEA5EFEE95DFDE85C4D4E4F60047F0180027F00EF70037F012290002077
:20382000D5E075F02FA424A4F9744035F0FA7B81A3E07E0029F9EE3AFAC003C002A3E0FBC3
:20384000A3E0FAA3E0F8AC02AD03D002D0037F01120023E47F002290002021EBF0900020D7
:203860001FEFF0A3EDF07B017A20792712003F05EF60037F0122900020217B017A20792545
:2038800012003A6B90002025E0FEA3E0F4FFEEF4FEA3E05EF0A3E05FF090002021E0FF9085
:2038A000002023E0FEA3E0A807088005C333CE33CED8F9FF90002025E05EFEA3E05FFFA3FE
:2038C000E04EF0A3E04FF09000201FE0FFA3E0FD90002027E0FAA3E0FB12003FF22274963C
:2038E0002FF974403EFA12002462FF90002042EFF07B017A207943E4FD1200365CEF6003A3
:203900007F0022900020457403F0A374E8F090002043E030E74BE490002047F090002047C4
:20392000E004F0E0B402F59000204574FFF5F0120024E2FEC3E5F09401EE940050037F0044
:203940002290002042E0FF7B017A207943E4FD1200365CEF60037F002290002043E020E750
:20396000C67F0122E490002004F090002003F090002000F090002000E0FFC39407504E1277
:20398000003DC6EF603E90002000E0FF900020097401F0A37420F0A37402F07B017A20792B
:2039A000011200372AEF60037F012290002001E0FF70069000200304F0EFB4010790002097
:2039C000047401F090002000E004F080A790002004E0B401041200408690002003E0B40166
:2039E000041200408B7F002290002016EDF0A3EBF090002015EFF07B017A20791B12003F85
:203A0000B9EF60012290002015E0FFE4FDFC1200402EEF600122E47F01FEFDFC9000202FCE
:203A2000120025CE90002016E0FF12003CF6AE0790002015E0FFAD0690002018E0F9A3E068
:203A4000FAA3E09000203AC9F0A3EAF0A3E9F090002017E0FB12002CDE90002015E090005A
:203A6000201B12004028EF60012222E0FFA3E0FD90002029EFF0A3EDF02FFFE433FEC3EF71
:203A80009410EE64809480401E90002029E0FF74017E00A807088005C333CE33CED8F9FFC2
:203AA000C3E49FFFE4803990002029E0FFA3E02FFF74017E00A807088005C333CE33CED8EF
:203AC000F9FDAC0690002029E0FF74017E00A807088005C333CE33CED8F9FFC3ED9FFFEC88
:203AE0009E8FF01200251C22900020CFEDF0A3EBF0900020CEEFF07B017A2079D312003F4A
:203B0000B9EF600122900020CEE0FFE4FDFC1200402EEF600122E47F01FEFDFC9000202F14
:203B2000120025CE900020CFE0FF12003CF6AE07AD07900020D0E0FBA3E0FFA3E090002065
:203B400038CFF0A3EFF0900020CEE0FF1200358E900020CEE0900020D312004028EF60010F
:203B60002222AB079000202DE0FCA3E0FDA3A3E4FFFEEC781012002553AA079000202DE083
:203B8000FCA3A3A3E0FFAE07AF03AD02AB069000203A7401F0A37420F0A37435F012002CAA
:203BA000DE90002034EFF07019A3E0FEA3E0FFE4FCFD90002031E0FBA3E0FAA3E0F9120034
:203BC000259690002034E0FF2290002022EBF090002024E0FBA3E0FAA3E0F912003F05EFAB
:203BE00060037F0122900020227B017A20792712003A6B90002024E0FBA3E0FAA3E0F912C7
:203C00000024F8FF90002027E055F0FEA3E05FFF90002022E0FDEFA805088005CEC313CE64
:203C200013D8F9FFEE8FF01200251C7F0022A907EA90002042F0EBA3F0A37405F09000208A
:203C400043E090007084F090002042E090007085F090007080E04401F090007082E9F0A3F3
:203C6000EDF07BE87A0390007080E0FF20E709EB1B70011A144A70EEEB4A60037F00229002
:203C8000002044E014F070B57F0122E49000200BF09000200BE0FFC394075049C0077F03AC
:203CA0007E007D107C009000202D120025CE900020317401F0A37420F0A3740CF0D0071232
:203CC000003B629000200CE0FCA3E0FDA3E0FEA3E0FF780412002553AC06AD079000200B05
:203CE000E004F080AC22E47F03FEFDFC9000202F120025CEE4FFAA079000202FE0FCA3E08F
:203D0000FDA3E0FEA3E0FF120025DA3D21000000013D25000000023D2B0000000300003D27
:203D20002FAB02800CEA2410FB80067B1B80027B1CAF032290002019EFF0A903AF05C0072A
:203D4000E47F01FEFDFC9000202F120025CED00712003CF6AE0790002019E0FFAD06AE014A
:203D6000AB069000201CE0F9A3E0FAA3E09000203AC9F0A3EAF0A3E9F012002CDE22AB0761
:203D80009000202DE0FCA3E0FDA3A3E4FFFEEC781012002553AA079000202DE0FCA3A3A372
:203DA000E0FFAE07AF03C007AD02AF06AB0790002033E0FFA3E090002038CFF0A3EFF0D0A2
:203DC000071200358E22EFC39407503874017E00A807088005C333CE33CED8F9FFEE339596
:203DE000E0FDFC90002086E0F8A3E0F9A3E0FAA3E05FFFEA5EFEE95DFDE85C4D4E4F6004E7
:203E00007F0180027F00EF7F017001FF2290002012EBF0A3EAF0A3E9F0AE07AC05EE7F00B7
:203E200030E7027F01EF60037F0422EEC45407FFEE540FFDAE04AB0690002012E0F9A3E017
:203E4000FAA3E090002018C9F0A3EAF0A3E9F0120039E82290002012EBF0A3EAF0A3E9F080
:203E6000AE07AC05EE7F0030E7027F01EF60037F0422EEC45407FFEE540FFDAE04AB069092
:203E8000002012E0F9A3E0FAA3E09000201CC9F0A3EAF0A3E9F012003D34229000200FEF46
:203EA000F0A903AF05C007E47F01FEFDFC9000202F120025CED00712003CF6AE07AD07AF79
:203EC00001AB0790002012E0FFA3E090002038CFF0A3EFF09000200FE0FF1200358E22E469
:203EE000FFFEFDFC900020CBE0FBA3E0FAA3E0F9120025967F01223099FDC2998F9922FFA4
:203F0000120027242290002029EFF0A3EDF0A3EBF0A3EAF0A3E9F012003CE6AE07900020DA
:203F200029E0FFAD069000202BE0F9A3E0FAA3E09000203AC9F0A3EAF0A3E9F09000202A9C
:203F4000E0FB12002CDE22AE07AC058B828A83EE7F0030E7027F01EF60037F0422EEC454C5
:203F600007FFC007EE540FFDAF04AB07AE83AF82900020D1EEF0A3EFF0D00712003AE82251
:203F8000AE07AC058B828A83EE7F0030E7027F01EF60037F0422EEC45407FFC007EE540F80
:203FA000FDAF04AB07AE83AF8290002012EEF0A3EFF0D00712003E9B229000201DEBF0A3EC
:203FC000EAF0A3E9F0900020237401F09000201DE0F9A3E0FAA3E090002024C9F0A3EAF0A3
:203FE000A3E9F07B0E7D0412003BC9EF6001227F002290002029EFF0A3EAF0A3EBF0A905B1
:2040000012003CE6AE07AD07AF01AB079000202AE0FFA3E090002038CFF0A3EFF09000208C
:2040200029E0FF1200358E22FFE0FCA3E0FD9000201DECF0A3EDF0900020227401F0900036
:20404000201DE0FDA3E090002023CDF0A3EDF07B0E7D0412003857EF6001227F00221200E3
:204060003964E4FFFE0FBF00010EBE4EF8BF20F50200272890007080E054FBF0A3E054F84E
:204080004402F07F002212004074227F01227F0122000001A5020A0A090001020304050643
:2040A0000708090A00081018202830384048800303030303030303030206000000000F09BB
:2040C0000000009502010B1E000102030405060708090A00081018202830384048800202FC
:2040E000020202020202060306000000000E090000009502020B1E000102030405060708A8
:20410000090A00081018202830384048800202020202020202060306000000000E0900006E
:20412000009502030B1E000102030405060708090A00081018202830384048800202020295
:2041400002020202060306000000000E090000009502040B1E000102030405060708090A36
:2041600000081018202830384048800202020202020202060306000000000E09000000958C
:2041800002050B1E000102030405060708090A0008101820283038404880020202020202C4
:2041A0000202060306000000000E090000009502060B1E000102030405060708090A0008D0
:2041C0001018202830384048800202020202020202060306000000000E09FFFFFFFFFFFFCF
:2041E000FFFFFFFFFFFFFFFFFFFFFFFFFFFFFFFFFFFFFFFFFFFFFFFFFFFFFFFFFFFFFFFFDF
:20420000FFFFFFFFFFFFFFFFFFFFFFFFFFFFFFFFFFFFFFFFFFFFFFFFFFFFFFFFFFFFFFFFBE
:20422000FFFFFFFFFFFFFFFFFFFFFFFFFFFFFFFFFFFFFFFFFFFFFFFFFFFFFFFFFFFFFFFF9E
:20424000FFFFFFFFFFFFFFFFFFFFFFFFFFFFFFFFFFFFFFFFFFFFFFFFFFFFFFFFFFFFFFFF7E
:208000000200D3EF74007400740074000204D9447400740002069DD425730056312E312E9C
:20802000360074000206B06AEB7008E709F608DFFA801B89828A831410E70AF593E0A3F681
:2080400008DFFA8009F593E493A3F608DFF9ECFAA9F0EDFB2288F0EF60010E4E60F088F0C9
:20806000ED60C51410E7E7CB700E88828C838B93E709F0A3DFFA80D61410E72A89828A837D
:20808000F593ECFAE0A3C8C582C8CCC583CCCBC593CBF0A3C8C582C8CCC583CCCBC593CB12
:2080A000DFE2DEE080AA89828A83F593ECFAE493A3C8C582C8CCC583CCCBC593CBF0A3C877
:2080C000C582C8CCC583CCCBC593CBDFE1DEDF02008050EB7002E72289828A831410E704E7
:2080E000F593E022F593E49322F8EB7006E7C828F3E82289828A831410E708F593E0C82825
:20810000F0E822F593E49322BB000327F722F8EB89828A831410E706F593E028F022F59310
:20812000E4932822BB0002F722BB8000500989828A838B931593F022EF8DF0A4A8F0CF8C21
:20814000F0A428CE8DF0A42EFE22BC000BBE0029EF8DF084FFADF022E4CCF875F008EF2F97
:20816000FFEE33FEEC33FCEE9DEC984005FCEE9DFE0FD5F0E9E4CEFD22EDF8F5F0EE008423
:2081800020D21CFEADF075F008EF2FFFED33FD4007985006D5F0F222C398FD0FD5F0EA2249
:2081A000C2D5EC30E709B2D5E4C39DFDE49CFCEE30E716B2D5E4C39FFFE49EFE1200814A94
:2081C000C3E49DFDE49CFC80041200814A30D507C3E49FFFE49EFE22C5F0F8A3E028F0C581
:2081E000F0F8E582158270021583E038F022A3F8E0C5F025F0F0E582158270021583E0C880
:2082000038F0E822EB7007E7F5F009E7192289828A831410E708F593E0F5F0A3E022F5932E
:20822000E493F5F074019322F8EB700C09E5F027C7F5F019E837C72289828A831410E7075D
:20824000F593E8020081EEF593E4740193F5F0E49322BB000B09C5F027F7C5F01937F7228B
:20826000F8EB89828A831410E707F593E8020081D8F59374019325F0F5F0E4933822BB0010
:2082800006F709A7F01922BB8000500D89828A838B931593F0E5F0A3F022E88FF0A4CC8BB4
:2082A000F0A42CFCE98EF0A42CFC8AF0EDA42CFCEA8EF0A4CDA8F08BF0A42DCC3825F0FDC9
:2082C000E98FF0A42CCD35F0FCEB8EF0A4FEA9F0EB8FF0A4CFC5F02ECD39FEE43CFCEAA466
:2082E0002DCE35F0FDE43CFC2275F008758200EF2FFFEE33FECD33CDCC33CCC58233C5822A
:208300009BED9AEC99E58298400CF582EE9BFEED9AFDEC99FC0FD5F0D6E4CEFBE4CDFAE482
:20832000CCF9A88222B800C1B90059BA002DEC8BF084CFCECDFCE5F0CBF97818EF2FFFEE35
:2083400033FEED33FDEC33FCEB33FB10D703994004EB99FB0FD8E5E4F9FA227818EF2FFFE3
:20836000EE33FEED33FDEC33FCC933C910D7059BE99A4007EC9BFCE99AF90FD8E0E4C9FA23
:20838000E4CCFB2275F010EF2FFFEE33FEED33FDCC33CCC833C810D7079BEC9AE899400ADA
:2083A000ED9BFDEC9AFCE899F80FD5F0DAE4CDFBE4CCFAE4C8F922CFF4CFCEF4CECDF4CDC2
:2083C000CCF4CC22C3E49FFFE49EFEE49DFDE49CFC22EB9FF5F0EA9E42F0E99D42F0EC64DD
:2083E00080C864809845F022EB9FF5F0EA9E42F0E99D42F0E89C45F022E8600FECC313FC91
:20840000ED13FDEE13FEEF13FFD8F122E8600FEFC333FFEE33FEED33FDEC33FCD8F122EB0C
:208420007006E9F8020089D889828A831410E706F593020089E4F59302008474BB0006E936
:20844000F802008A39BB8000500C89828A838B9315930200850B22EB7006E9F802008A2246
:2084600089828A831410E706F593020084DFF59302008474E493FC740193FD740293FE7471
:208480000393FF22EB7006E9F8020089F089828A831410E706F593020089FDF59302008A1B
:2084A000097401FF3395E0FEFDFCA3A3A3E0CF2FF0E582158270021583E0CE3EF0E5821589
:2084C0008270021583E0CD3DF0E582158270021583E0CC3CF0227401FF3395E0FEFDFCA37E
:2084E000A3A3E02FFFF0E582158270021583E03EFEF0E582158270021583E03DFDF0E582AB
:20850000158270021583E03CFCF022ECF0A3EDF0A3EEF0A3EFF022F5F0C582A4C582C5F043
:20852000C583A42583F58322A42582F582E5F03583F58322EB7006E9F802008A4589828A7C
:20854000831410E706F59302008A57F59302008A97BB001CD093D0F0D0E0F8D0E0C9FBD08B
:20856000E0FAD0E0CBC8C0E0C0F0C09302008A4EBB80005022D093D0F0D0E0F8D0E0C9F57B
:2085800082D0E0CAF583D0E0CB14C8C0E0C0F0C093889302008A8ED093D083D082D0E0D0B0
:2085A000E0D0E0E473D093D083D082F8E4937012740193700DA3A393F8740193F5828883FB
:2085C000E4737402936860EFA3A3A380DFD093D083D082F8E4937012740193700DA3A393E5
:2085E000F8740193F5828883E473740293B5F0067403936860E9A3A3A3A380D8D093D08399
:20860000D082E4937012740193700DA3A393F8740193F5828883E4737402936C701274036A
:20862000936D700C7404936E70067405936F60DDA3A3A3A3A3A380CA8B938A83898215931D
:2086400053937FE473759308E5512582F582E5503583F583B550048582512210AF06858246
:2086600051F55022858251F550D2AF22759308E5512582F582E5503583F58322EB700C8729
:20868000F009E608B5F041603F80F489828A831410E70FF593E0F5F0A3E608B5F02A602893
:2086A00080F3F593E493F5F0A3E608B5F01A601880F2CB701588828C838B9387F009E493AB
:2086C000A3B5F004600280F380611410E72E89828A83F593ECFAE0F5F0A3C8C582C8CCC509
:2086E00083CCCBC593CBE493A3C8C582C8CCC583CCCBC593CBB5F033603180DA89828A83A3
:20870000F593ECFAE493F5F0A3C8C582C8CCC583CCCBC593CBE493A3C8C582C8CCC583CC76
:20872000CBC593CBB5F004600280D97F00F845F0600EE863F0806480D395F01F40027F01F5
:20874000220200867C020086B2ED60F51410E7F5CB701488828C83F59387F009E0A3B5F0DF
:20876000CA60C880F480C41410E72D89828A83F593ECFAE0F5F0A3C8C582C8CCC583CCCBA7
:20878000C593CBE0A3C8C582C8CCC583CCCBC593CBB5F097609580DB89828A83F593ECFA7C
:2087A000E493F5F0A3C8C582C8CCC583CCCBC593CBE0A3C8C582C8CCC583CCCBC593CBB538
:2087C000F0A360A180DAEB7008E709F60870FA801B89828A831410E70AF593E0A3F60870AF
:2087E000FA8009F593E493A3F60870F9ECFAA9F0EDFB2288F0ED60CE1410E7F0CB700E8805
:20880000828C83F593E709F0A370FA80DF1410E72889828A83F593ECFAE0A3C8C582C8CC14
:20882000C583CCCBC593CBF0A3C8C582C8CCC583CCCBC593CB70E280B589828A83F593ECEB
:20884000FAE493A3C8C582C8CCC583CCCBC593CBF0A3C8C582C8CCC583CCCBC593CB70E1D6
:20886000808CEB700C87F009E608B5F019DFF6801589828A831410E711F593E0F5F0A3E6E5
:2088800008B5F002DFF502008913F593E493F5F0A3E608B5F07DDFF48079CB701388828C70
:2088A000838B9387F009E493A3B5F067DFF580631410E73089828A83F593ECFAE0F5F0A391
:2088C000C8C582C8CCC583CCCBC593CBE493A3C8C582C8CCC583CCCBC593CBB5F035DFDC9F
:2088E000DEDA802F89828A83F593ECFAE493F5F0A3C8C582C8CCC583CCCBC593CBE493A3CD
:20890000C8C582C8CCC583CCCBC593CBB5F004DFDBDED97FFFB5F0020F2240027F0122025C
:208920000088620200889A88F0EF60010E4E60EEED60EC1410E7ECCB701288828C83F59399
:2089400087F009E0A3B5F0CBDFF680C71410E72F89828A83F593ECFAE0F5F0A3C8C582C889
:20896000CCC583CCCBC593CBE0A3C8C582C8CCC583CCCBC593CBB5F09ADFDDDEDB809489B0
:20898000828A83F593ECFAE493F5F0A3C8C582C8CCC583CCCBC593CBE0A3C8C582C8CCC54B
:2089A00083CCCBC593CBB5F004DFDCDEDA02008913EF4E6022EF60010EEDBB0007F709DF15
:2089C000FCA9F022BB8000500E89828A838B931593F0A3DFFCDEFA22E6FC08E6FD08E6FE48
:2089E00008E6FF22E0FCA3E0FDA3E0FEA3E0FF22E6FB08E6F908E6FA08E6CBF822E0F8A3E9
:208A0000E0F9A3E0FAA3E0FB22E493F8740193F9740293FA740393FB227401FF3395E0FEAC
:208A2000FDFC080808E62FFFF618E63EFEF618E63DFDF618E63CFCF622ECF608EDF608EEAC
:208A4000F608EFF622E6FB08E6FA08E6F922EBF608EAF608E9F622E0FBA3E0FAA3E0F92277
:208A6000F8E0FBA3A3E0F925F0F0E582158270021583E0FA38F022F8E0FBA3A3E025F0F9CC
:208A8000F0E582158270021583E038FAF022EBF0A3EAF0A3E9F022E493FB740193FA7402DA
:208AA00093F922E526245DF582E43494F583759308E00526229008945A301F049008945D42
:208AC000E475F00112008A60020080D32018E57F2ED2188018EF540F2490D43440D4FF305E
:208AE0001C0BEF24BFB41A0050032461FFE52760021527052AE52A70020529301F11900858
:208B0000945AE475F00112008A60EF020081240200D7BF7403D21F8003E4C21FF526900890
:208B2000945A12008A8EE4F527F529F52AE52760087F2012008AED80F47528FFC219C2187F
:208B4000C21AC21BC21DC21EC22012008AB5FF700E301F067F0012008AFEAF2AAE2922B4F9
:208B60002563C2D5C21C12008AB5FF24D0B40A00501A75F00A782730D50508B6FF0106C6EA
:208B8000A426F620D5047002D21B80D824CFB41A00EF5004C2E5D21C02008D2BD21980C4E3
:208BA000D21880BED21A80BAD2D580B8D21D80B27F2012008AED201A077401B5270040F07D
:208BC00012008AA3FF12008AED02008B2DD220D21E808F12008AA3FB12008AA3FA12008A14
:208BE000A3F94A4B700679027A8E7B81201A3DE52760397E00E9C0E02EF9EAC0E03400FA4D
:208C0000120080D3F9D0E0FAD0E0C960060EEE652870E2C2D5EBC0E0EAC0E0E9C0E0EE125D
:208C2000008D73D0E0F9D0E0FAD0E0FB120080D3FF6096EBC0E0EAC0E0E9C0E012008AEDB5
:208C4000D0E02401F9D0E03400FAD0E0FBE5280460DAD528D702008BC97BFF7A8D796FD20D
:208C60001A8089791080027908C21EC2208008D2D5790A8004790AC2D5E528047002F52893
:208C8000E4FAFDFEFF12008AA3FC7B0820191612008AA3FD7B1030180C12008AA3FE120085
:208CA0008AA3FF7B20EC3382D592D55013C3E43018069FFFE49EFEE42019039DFDE49CFC64
:208CC000E4CBF8C219EC700CCFCECDCCE824F8F870F38017C3EF33FFEE33FEED33FDEC333F
:208CE000FCEB33FB994002FB0FD8E9EB301905F8D0E0C448B219C0E00AEC4D4E4F78207B6E
:208D00000070C2EAB5280040BCC0E012008D75D0F0D0E0201904C4C0E0C4B219C0F0120048
:208D20008AD6D0F0D5F0EA02008B2D120085A58BD3538C63588BA04C8B9C428C674F8C6F59
:208D4000448C6F498BB6438C75558C59468C59458C59478E1F508BA42D8BA82E8BCF2B8B66
:208D6000AC238BCD208E0B2A8B624800008BC53F3F3F00790AA2D5201B14301D09B910023D
:208D80000404B9080104A2D5201E02500104201A6D921AB527005036C0E07F20301B1A7F21
:208DA00030A21A721E721D501012008DCEC21AC21EC21DC2207F308010301D03E9C0E01234
:208DC000008AED301D03D0E0F9D0E0B527CA301D197F30B9100D12008AED7F58301C077FB0
:208DE000788003B9080412008AED301A067F2D02008AED7F202020F77F2B201EF222921A37
:208E000080CC286E756C6C2900D21912008AA33019F7C219782730D50108F602008B621211
:208E2000008AA37F4960087F4310E7027F5814C0E0EF12008ADE743A12008ADED0E0600DE1
:208E4000C0E0C412008AD6D0E012008AD6D21B75270402008C630D0A204949435F53444159
:208E6000206C6F77206F72204949435F53434C206C6F772C2073746F7020636F6E64697424
:208E8000696F6E2067656E65726174652E2E2E2E2E000A206932635F7265616420737465AC
:208EA000702031206932632061636B206572726F722E2E2E000A206932635F72656164206D
:208EC00073746570322D31206932632061636B206572726F722E2E2E000A206932635F720C
:208EE0006561642073746570322D32206932632061636B206572726F722E2E2E000A206907
:208F000032635F72656164207374657033206932632061636B206572726F722E2E2E000A67
:208F2000206932635F7772697465207374657031206932632061636B206572726F722E2E69
:208F40002E000A206932635F77726974652073746570322D31206932632061636B20657261
:208F6000726F72000A206932635F77726974652073746570322D32206932632061636B20F2
:208F80006572726F72000A206932635F7772697465207374657033206932632061636B2059
:208FA0006572726F72000A20616464723D25640044656661756C740070617373776F7264C4
:208FC00000004D444C3A465337353054325F56312E312E3620202020202020202020202096
:208FE000202020202020202000256C640077726974652D6F6E6C790044656661756C74009D
:20900000465337353054320000000000000000000000000000000000000000000000000095
:20902000000000000000000000465337353054320000000000000000000000000000000075
:2090400000000000000000000000000000000000000056312E312E36000000000000740052
:2090600074000000000000000000000000000000000056312E312E3600001223344566011D
:2090800080C200000F74006472697665724877436E746C496E6974204661696C21210A00B3
:2090A000475420696E6974204641494C21210A000A5B4D41435F49442D2564203D2025300F
:2090C00032785D0A000A5B5048595F494425643D25785D0A00736574204754205452554E03
:2090E0004B2044656C657465206661696C0A00736574204754205452554E4B204372656196
:209100007465206661696C0A0067766C6E476574566C616E506F727473202850424153457D
:2091200029206661696C0A0067766C6E44656C566C616E506F727420285042415345292042
:209140006661696C0A0067766C6E536574566C616E506F727473202850424153452920667B
:2091600061696C0A00636865636B206D6769705F6964206661696C0A007365742044656C71
:20918000205258706F7274206661696C0A007365742044656C205458706F72742066616918
:2091A0006C0A00736574205258706F7274206661696C0A00736574205458706F7274206635
:2091C00061696C0A00736574205258534E46706F7274206661696C0A00736574205458535C
:2091E0004E46706F7274206661696C0A0073657420516F73205472757374206D6F6465208A
:209200006661696C0A0073657420516F73205062617365206661696C0A0073657420516F0C
:20922000732E3170207472757374206D6F6465206661696C0A0073657420516F732E317091
:20924000206661696C0A007365742067766C6E536574506F7274496E677265737346696C5E
:20926000746572696E67206661696C0A007365742067766C6E536574506F7274496E67721B
:2092800065737346696C746572696E67202D2D20756E6D6F6469666979206661696C0A00AB
:2092A0007365742067766C6E536574506F72744163634672616D6554797065206661696C6A
:2092C0000A007365742067766C6E53657450766964206661696C0A0067766C6E47657456AF
:2092E0006C616E506F727473206661696C0A0067766C6E476574566C616E506F72747320B5
:209300006E6F20666F756E640A0067766C6E44656C566C616E506F7274202D2043505520B3
:209320006661696C0A0067766C6E536574566C616E506F727473206661696C0A00676574F5
:209340002043505520636F756E746572206661696C21210A00740087EDC987EDD187EDD49F
:2093600087EDD787F11687F11E87F12487F12B87F13387F13B61007400203C74643E0A2070
:209380003C73656C656374206E616D653D25732025733E0A003C74723E3C746820636F6CA5
:2093A0007370616E3D343E25730A3C74723E0A203C74643E3C623E42797465730A203C7411
:2093C0006420636F6C7370616E3D333E256C750A0A003C74723E0A203C74643E3C623E2574
:2093E000730A203C74643E256C750A203C74643E3C623E25730A203C74643E256C750A0AF2
:209400000074007400740000000000000074007400740074007400428AAE0000448AD00094
:2094200000012C418AAA0042AB0E0000439558FFFFFF4AA699000000000000000000004198
:20944000A9FD0041A9FCFF41B07F014297EE000A4297F600004297EA00004297EC000042A6
:2094600097E600004297F800004297F0FFFF4297E880004497E2000000004297DC000042E2
:2094800097DE00004297E00000413DF600469FB1FFFFFFFFFFFF469FA70180C20000004388
:2094A00071BA8190854771B37F7F7F000000004672B60180C200000F4294F20000429F1E7C
:2094C00000004F9F0F87E62A87E63687E64787E65987E6474CA3FA88D04088D04888D04B63
:2094E00088D04E4C88C888797588797C8879808879875888B088798C88799488799C8879DE
:20950000A58879AE8879B78879BE8879C55889078879CD8879D58879DF8879E98879F288E9
:2095200079FB88798C887A00602788E0887A05887A0F887A19887A25887A31887A3D887A6B
:2095400049887A54887A5F887A6A887A75887A7A887A004688D4887A7A887A824688DA88D8
:209560007A89887A8D43AF8787FFFC4E8B5600010009001100190021002900314E8B950012
:2095800008001000180020002800300032437DAF000000629B041087B0096367695F6475C6
:2095A0006D790000000000000000000000008585206367695F6C6F67696E000000000000F0
:2095C000000000000086EB0E6367695F706F727400000000000000000000000082DCC8632C
:2095E00067695F736574706F72740000000000000000008511206367695F766C616E000032
:2096000000000000000000000000855DB16367695F736574766C616E000000000000000028
:209620000084BD8F6367695F64656C766C616E000000000000000000840EBE6367695F7090
:2096400076696400000000000000000000000082924E6367695F7669640000000000000090
:209660000000000000008307C86367695F6164647669640000000000000000000081D895AC
:209680006367695F6465766963650000000000000000000082A6426367695F6465746169C5
:2096A0006C00000000000000000000844DDA6367695F7374617469737400000000000000F5
:2096C0000000856C096367695F7472756E6B000000000000000000000083731F6367695F23
:2096E0006D6972726F72000000000000000000008611F66367695F706173730000000000F9
:209700000000000000000082D4026367695F73797300000000000000000000000000877FFA
:20972000D66367695F6261636B757000000000000000000000861D096367695F62616B5F80
:209740006461746100000000000000008780236367695F7265736574000000000000000090
:2097600000000087A88B6367695F716F730000000000000000000000000086CE0C636769B7
:209780005F7170626173650000000000000000000086DDDF6367695F713170000000000008
:2097A0000000000000000000837F936367695F7374700000000000000000000000000083A8
:2097C00016706367695F736E6D70000000000000000000000000858BA06367695F61636C41
:2097E000000000000000000000000000008657E56367695F61646461636C000000000000BC
:209800000000000085B5216367695F64656C61636C000000000000000000000000000000F6
:2098200000000000000000000000000000000000000042AEFA000042898700004289890098
:20984000004240FB000042462E00004242EE00044942CD81D2A381D2B181D2D95245588171
:20986000D2F081D30781D31D81D33381D34B81D3674C460081D38481D3A181D3BF81D3D6DD
:209880006032463000000000000000000000000000000000000000000000000000000000C0
:2098A000000000000000000000000000000000000000000000006064409700010003000603
:2098C00000010004000111AE000B00050001000000000000000000000000000000000000B2
:2098E00000000000000000000000000B00000000000000000000000000000000000000005D
:20990000000000000000000000000000000000000000000000000000000000000000606483
:20992000426900010003000600010004000111AE000B00050002000000000000000000009B
:20994000000000000000000000000000000000000000000B000000000000000000000000FC
:209960000000000000000000000000000000000000000000000000000000000000000000E7
:20998000000000000000609641D3000100030006000100020001000200020001000100FFAA
:2099A0000000000000000000000000000000000000000000000000000000000B0001000398
:2099C000000600010004000111AE000B0005000300000000000000000000000000000000A9
:2099E000000000000000000000000000000B0000000000000000000000000000000000005C
:209A0000000000000000000000000000000000000000000000000000000000000000000046
:209A20006096456A000100030006000100020001000200020001000100FF0000000000006E
:209A40000000000000000000000000000000000000000000000B00010003000600010004EC
:209A6000000111AE000B000500040000000000000000000000000000000000000000000012
:209A8000000000000000000B000000000000000000000000000000000000000000000000BB
:209AA00000000000000000000000000000000000000000000000000000006064402F000172
:209AC0000003000600010004000111AE000B000500050000000000000000000000000000A3
:209AE0000000000000000000000000000000000B000000000000000000000000000000005B
:209B0000000000000000000000000000000000000000000000000000000000000000000045
:209B2000000060643FCB00010003000600010004000111AE000B0005000600000000000072
:209B400000000000000000000000000000000000000000000000000B0000000000000000FA
:209B60000000000000000000000000000000000000000000000000000000000000000000E5
:209B80000000000000000000000060643F6500010003000600010004000111AE000B00057E
:209BA000000700000000000000000000000000000000000000000000000000000000000B93
:209BC000000000000000000000000000000000000000000000000000000000000000000085
:209BE000000000000000000000000000000000000000606441010001000300060001000450
:209C0000000111AE000B00050008000000000000000000000000000000000000000000006C
:209C2000000000000000000B00000000000000000000000000000000000000000000000019
:209C4000000000000000000000000000000000000000000000000000000060644165000199
:209C60000003000600010004000111AE000B000500090000000000000000000000000000FD
:209C80000000000000000000000000000000000B00000000000000000000000000000000B9
:209CA0000000000000000000000000000000000000000000000000000000000000000000A4
:209CC00000004441CF094097004442EA094269004442E60941D30144461309456A014441C7
:209CE000C909402F004440FD093FCB00444093093F65004442DE094101004442E209416505
:209D000000423F6300004AA711FC06FC03FC0400A12000426D45000143AFA287FFFE43AF9C
:209D2000A588FFFE43AFA8891FC44C9E2F81CCB381CCBA81CCBE81CCC5469E2981CCCA8111
:209D4000CCD94CA41E89031689031D89032189032843AFAB891FC643AE00891FC860408E0A
:209D60001C00081018202830380A121A220C141C240E161E262E01020304050607090B0D5C
:209D80000F11131517191B1D1F21232527292A2B2C2D2F31323334353637393A3B3C3D3E8D
:209DA0003F437E70097E9D437F0E097EA1437E91097EA5437F1D097EA9437E6D097EAD43E5
:209DC0007F17097EB1437E85097EB5437F05097EB9437E79097EBD437E8B097EC1437E97C2
:209DE000097EC5437F0B097EC9437E7F097ECD437E76097ED1437F14097ED5437E94097EC9
:209E0000D9437F20097EDD437E73097EE1437F1A097EE5437E88097EE9437F08097EED4305
:209E20007E7C097EF1437E8E097EF5437E9A097EF9437F11097EFD437E82097F014399DC2F
:209E40000999E2427D0A0004437CF2097D24437CF5097D28437D1B097D2C437D0F097D30E2
:209E6000437D94097D34437D9D097D38437D01097D3C437D0C097D40437D97097D44437CC4
:209E8000EF097D48437CFE097D4C437D15097D50437D18097D54437DA0097D58437CF8091B
:209EA0007D5C437DAC097D60437D1E097D64437DA6097D68437D07097D6C437D12097D70DA
:209EC000437D9A097D74437D04097D78437DA3097D7C437CFB097D80437CEC097D84437DD2
:209EE00021097D88437DA9097D8C5478C000010003000600010004000111AE0064000400F5
:209F0000044378BA0978E34378E00979374378DD0979674378DA09796B4378BD0979804350
:209F200078D40979954378D70979AA4387F20988074387EC09880B4387EF09880F4387CD6A
:209F40000988134387FB0988174387F809881B4387E909881F4387FE098823438804098843
:209F6000274387E009882B4387E309882F4388010988334387E60988374387F509883B4311
:209F8000961709962043961D09962443961409962843961A09962C43AFB781800443756F55
:209FA0000975754374E309757943754809757D4375390975814374DA0975854374E0097589
:209FC000894374DD09758D43753F09759143754E09759543757209759943754209759D43A1
:209FE00075540975A143753C0975A54375510975A94375690975AD4375450975B143756C96
:20A000000975B543754B0975B94375360975BD4375C50975C143A0EA09683D43A0F009682F
:20A020003D43A0ED09683D43A0E409683D43A0E709683D428AA8740060598A4F4E6F746568
:20A040003A3C62723E0A54313A2061757468656E7469636174696F6E206661696C3C6272E3
:20A060003E0A54323A2064657669636520626F6F7475703C62723E0A54333A206C696E6BA8
:20A08000207570202F206C696E6B20646F776E3C62723E0A004FA0F38885B08885B88885FD
:20A0A000BE8885C58885CE4324CC8190606028157E00000000000000000000000000000076
:20A0C0000000000000000000000000000000000000000000000000000066721E5400000036
:20A0E000000000000000000000000000000000000000000000000000000000000000000060
:20A1000000000000000000000000000000000000000000000000000000000000000000003F
:20A1200000000000000000000000000000000000000000000000000000000000000000001F
:20A140000000000000000000000000000000000000000000000000000000000000000000FF
:20A74000000000000000000000000000000000667215A60000000000000000000000000066
:20A760000000000000000000000000000000000000000000000000000000000000000000D9
:20A780000000000000000000000000000000000000000000000000000000000000000000B9
:20A7A000000000000000000000000000000000000000000000000000000000000000000099
:20A7C000000000000000000000000000000000000000000000000000000000000000000079
:20ADC000000000000060321E220000000000000000000000000000000000000000000000A1
:20ADE0000000000000000000000000000000000000000000000000000000006064259800D2
:20AE0000000000000000000000000000000000000000000000000000000000000000000032
:20AE2000000000000000000000000000000000000000000000000000000000000000000012
:20AE40000000000000000000000000000000000000000000000000000000000000000000F2
:20AE6000000000606424CF000000000000000000000000000000000000000000000000001B
:20AE80000000000000000000000000000000000000000000000000000000000000000000B2
:20AEA000000000000000000000000000000000000000000000000000000000000000000092
:20AEC000000000000000000000000060641C2400000000000000000000000000000000006E
:20AEE000000000000000000000000000000000000000000000000000000000000000000052
:20AF0000000000000000000000000000000000000000000000000000000000000000000031
:20AF20000000000000000000000000000000000000000060642534000000000000000000F4
:20AF40000000000000000000000000000000000000000000000000000000000000000000F1
:20AF60000000000000000000000000000000000000000000000000000000000000000000D1
:20AF800000000000000000000000000000000000000000000000000000000061901C8E0016
:20AFA000000000000000000000000000000000000000000000000000000000000000000091
:20AFC000000000000000000000000000000000000000000000000000000000000000000071
:20AFE000000000000000000000000000000000000000000000000000000000000000000051
:20B00000000000000000000000000000000000000000000000000000000000000000000030
:20B02000000000000000000000000000000000000000000000000000000000000000000010
:20B040000000000000000000000000000000000000000000000000000000000000000000F0
:20B060000000000000000000000000000000000000000000000000000000000000000000D0
:20B080000000000000000000000000000000000000000000000000000000000000000000B0
:20B0A000000000000000000000000000000000000000000000000000000000000000000090
:20B0C000000000000000000000000000000000000000000000000000000000000000000070
:20B0E000000000000000000000000000000000000000000000000000000000000000000050
:20B1000000000000000000000000000000000000000000000000000000000000000000002F
:20B12000000000000000000000000000000000411C1F014624C60180C20000004125330086
:20B14000421C8C000043AFCC891FCA43AFCF81940D449D8500000000449D890000001444CA
:20B160009D810000000143AFDB81800643AFDE81800843AFE181800A43AFE481801043AF4C
:20B18000E781801243AFEA818022E64809B0FD000000000006600A050040340000014C0696
:20B1A000000000000060A10204000009000011000000A02603803F000000A4000100190721
:20B1C0008000040200000004004030128398A4048040301EE6B16A050040300149CA3004D4
:20B1E00000405402C40001040040540004014004004054000481400400405402C400000458
:20B2000000405402C50001040040540005014004004054000581400400405402C500000433
:20B2200000405402C60001040040540006014004004054000681400400405402C60000040F
:20B2400000405402C70001040040540007014004004054000781400400405402C7000004EB
:20B2600000405402C80001040040540008014004004054000881400400405402C8000004C7
:20B2800000405402C90001040040540009014004004054000981400400405402C9000004A3
:20B2A00000405402CA000104004054000A014004004054000A81400400405402CA0000047F
:20B2C00000405402CB000104004054000B014004004054000B81400400405402CB0000045B
:20B2E00000405402CC000104004054000C014004004054000C81400400405402CC00000437
:20B3000000405402CD000104004054000D014004004054000D81400400405402CD00000412
:20B3200000405402CE000104004054000E014004004054000E81400400405402CE000004EE
:20B3400000405402CF000104004054000F014004004054000F81400400405402CF000005C9
:20B3600000405402D00002050040540010004005004054001080400500405402D0000005A3
:20B3800000405402D080000500405402D10002050040540011004005004054001180400500
:20B3A00000405402D100000500405402D180000500405402D20003050040540212711E0589
:20B3C0000040540232441005004054025242050500405402D20002050040540012004005BE
:20B3E0000040540012804004004054021205880500405402D200000500405402D28000054F
:20B4000000405402D30003050040540213711E050040540233441005004054025342050527
:20B4200000405402D30002050040540013004005004054001380400400405402130588050A
:20B4400000405402D300000500405402D380000400404000019015048040400001901505BC
:20B4600000404000019015058040400001901504000010000078CC04000110000078CC0446
:20B48000000210000078CC04000310000078CC04000410000078CC04000510000078CC043E
:20B4A000800010000078CC04800110000078CC04800210000078CC04800310000078CC0426
:20B4C000800410000078CC04800510000078CC05000010000078CC05000110000078CC05FF
:20B4E000000210000078CC05000310000078CC05000410000078CC05000510000078CC05DA
:20B50000800010000078CC05800110000078CC05800210000078CC05800310000078CC05C1
:20B52000800410000078CC05800510000078CC0400402800100000048040280010000005D8
:20B54000004028001000000580402800100000040000001403020104000100140302030433
:20B560000002001403020504000300140302070400040014030209040005001403020B0429
:20B580008000001403020D048001001403020F0480020014030211048003001403021304F1
:20B5A0008004001403021504800500140302170500000014030219050001001403021B05AA
:20B5C0000002001403021D050003001403021F050004001403022105000500140302230565
:20B5E0008000001403022505800100140302270580020014030229058003001403022B052D
:20B600008004001403022D058005001403022F018005000804020101810500080402010261
:20B620000400040000FA5002000000400000000200100040000000020020004000000002C0
:20B640000030004000000002004000400000000200500040000000020060004000000002C2
:20B6600000700040000000020080004000000002009000400000000200A0004000000002A2
:20B6800000B000400000000200C000400000000200D000400000000200E000400000000282
:20B6A00000F00040000000020100004000000002011000400000000201200040000000025F
:20B6C00001300040000000020140004000000002015000400000000201600040000000023E
:20B6E0000170004000000004004054032405550500405403240555040041006124FF9B04FE
:20B7000000410C0000A00004004104111100000480410422223434050041006124FF9B05F2
:20B7200000410C0000A00005004104111100000580410422223434030000007FCFF7FC03F3
:20B7400000003000FFFFFF018000040392FBF3030000200780C826030000240400740E016E
:20B76000800C800000310801810C800000310801800C000000310901800C1000003109019E
:20B78000800C200000310901800C300000310901810C000000310901810C1000003109012B
:20B7A000810C200000310901810C3000003109000000000006600B050040540012894005C0
:20B7C0000040540013894005004054001291400500405400139140E05009B0AD04004054D2
:20B7E000032405550500405403240555040041006124FF9B0400410C0000A0000400410410
:20B80000111100000480410422223434050041006124FF9B0500410C0000A00005004104F0
:20B82000111100000580410422223434419E5700479E5800000000000000429E4D0000448C
:20B84000973C000000015C9720000000000000000000000000000000000000000000000001
:20B86000000000000041AE3E0044AE3A000000004289ED00005889EF0000000000000000E7
:20B8800000000000000000000000000000000000588A0700000000000000000000000000BF
:20B8A0000000000000000000000000588A1F00000000000000000000000000000000000087
:20B8C000000000000000588A3700000000000000000000000000000000000000000000004F
:20B8E000004E9EBD099EBD099EBD099EBD000000000000716F73747970653D00716F73745A
:20B900007970653D256400516F7320547970652053657474696E6700546F20656E61626C3B
:20B9200065203830322E317020516F532C20596F75206E656564206368616E676520746F18
:20B94000203830322E315120564C414E2E006367695F716F730070253032643D00256400F8
:20B96000706F72743D00706F72743D253032640073706565643D0073706565643D256400B3
:20B980007365745F666C6F773D007365745F666C6F773D2564006367695F736574706F72AF
:20B9A000743D256400506F72742053657474696E67004D65646961207479706520697320CC
:20B9C0006368616E6765642E3C62723E43757272656E742073706565642073657474696E56
:20B9E00067206973206E6F74207375697461626C652E00766C616E5F69643D00766C616E01
:20BA00005F69643D256400646573633D002600564C414E206465736372697074696F6E201D
:20BA20006D75737420626520302D25642063686172616374657273006367695F61646476DF
:20BA40006C616E3F6E756D3D256400564C414E2053657474696E67007663623D0076636274
:20BA60003D25303264006367695F736574766C616E3D25640054686520766C616E2067725E
:20BA80006F757020706F7274206D7573742073657420746F207468652073616D65207472E8
:20BAA000756E6B2073657474696E67006E756D3D006E756D3D2564007663623D2564006313
:20BAC00067695F64656C766C616E0076747970653D0076747970653D25303264004465666D
:20BAE00061756C74007379733D006C6F633D006C6F67696E3D0053797374656D206E616D42
:20BB000065206D75737420626520302D256420636861726163746572730053797374656D25
:20BB20002053657474696E67006367695F737973004C6F636174696F6E206E616D65206D8F
:20BB400075737420626520302D2564206368617261637465727300496E76616C6964206C09
:20BB60006F67696E2074696D656F75742076616C756500646863703D00646863703D256473
:20BB80000069703D00496E76616C69642049502061646472657373006D6B3D00496E766166
:20BBA0006C6964207375626E6574206D61736B0067773D00496E76616C696420676174652C
:20BBC000776179204950004950207375626E6574206D75737420657175616C20746F206766
:20BBE000617465776179207375626E65740061636C5F69643D0061636C5F69643D2564004E
:20BC0000495020416363657373204C6973742053657474696E67006367695F61636C004954
:20BC200070204163636573732063616E206E6F74206265206475706C6963617465640049F0
:20BC40005020616464726573732063616E6E6F74206265207468652073616D6520617320C9
:20BC6000537769746368006F6C645F706173733D006E65775F706173733D0072656E657702
:20BC80005F706173733D004368616E67652050617373776F72640070617373776F72642005
:20BCA0006C656E6774682063616E6E2774206265207A65726F006367695F70617373005047
:20BCC000617373776F72642053657474696E67004E65772050617373776F7264206D757351
:20BCE0007420626520302D32302063686172616374657273006F6C642070617373776F725C
:20BD0000642069732077726F6E67006E65772070617373776F726420697320696E636F6E66
:20BD200073697374656E7400656E61626C65253032643D00746B70253032643D002530326C
:20BD40006426005472756E6B2053657474696E67005468652073656C6563746564207472B7
:20BD6000756E6B20706F72742073657474696E67206D7573742073657420746F20746865B9
:20BD80002073616D652056414C4E2047726F7570006367695F7472756E6B006D6F64653DB7
:20BDA000006D6F64653D2530326400736E69666665723D00736E69666665723D2530326477
:20BDC000006D63623D006D63623D2530326400647669643D00505649442053657474696EEC
:20BDE0006700496E76616C6964205649442076616C7565006367695F7076696400564944AD
:20BE00002025303264206973206E6F742065786973742C6F7220506F727420253032642060
:20BE20006973206E6F7420746865206D656D626572206F662056494420253032642E002764
:20BE40006367695F7076696427007461675F69643D007461675F69643D2564007669643D23
:20BE6000005649442053657474696E67006367695F6164647669640054686520564944209F
:20BE8000697320657869737420564944207461626C65007669645F6D656D3D0054686520EF
:20BEA00064656661756C7420766964206F6620706F727420253032642069732025642C2064
:20BEC000736F2069742063616E6E277420626520756E73656C65637465642E00276367696D
:20BEE0005F7365747669643D25642700546865207669642069732074686520646566617561
:20BF00006C7420766964206F6620706F727420253032642C20736F2069742063616E6E27E7
:20BF2000742062652064656C657465642E006367695F7365747669643D25640052656D6F07
:20BF4000766520564C414E007061737377643D00666C61673D00666C61673D2564006661E8
:20BF600073743D00666173743D256400627072693D005370616E6E696E6720547265652031
:20BF800053657474696E6700496E76616C696420427269646765205072696F72697479000D
:20BFA0006367695F73747000626167653D00496E76616C696420427269646765204D617852
:20BFC00020416765006268656C6C6F3D00496E76616C6964204272696467652048656C6CA8
:20BFE0006F2054696D650062646C61793D00496E76616C69642042726964676520466F725F
:20C00000776172642044656C61790064633D00496E76616C6964205061746820436F737432
:20C020002076616C75650064703D00496E76616C6964205072696F726974792076616C7591
:20C04000650000534E4D502053657474696E6700496E76616C696420534E4D5020486F73D0
:20C06000742049502E006367695F6E6577736E6D705F686F737400636F6D6D25643D0043F9
:20C080006F6D6D756E697479206E616D65206D75737420626520302D256420636861726168
:20C0A0006374657273006367695F736E6D700070726925643D0030007431616C6C3D006152
:20C0C000646D696E007431616C6C3D25640028256429543174726170323A25640A00747219
:20C0E00025643D0025732525640061646D696E25643D00486F73742049702063616E206E0E
:20C100006F74206265206475706C696361746564006270747970653D006270747970653D74
:20C1200025640020534F484F202D20736F686F44756D70506F727452656773206465765B71
:20C14000256C755D2D205374617274200A00506F727420256C750A00202530326C7520205A
:20C16000000A3D3D3D3D3D3D3D3D3D3D3D3D3D3D3D3D3D3D3D3D3D3D3D3D3D3D3D3D3D3D8F
:20C180003D3D3D3D3D3D3D3D3D3D3D3D3D3D3D3D3D3D3D3D3D3D3D3D3D3D3D3D3D3D3D3DFF
:20C1A0003D3D3D3D3D3D3D0A000A4661696C20746F207265616420726567697374657220E0
:20C1C000256C7520726320256C750A002025303478000A0020534F484F202D20736F686F8A
:20C1E00044756D70476C6F6252656773206465765B256C755D2D205374617274200A000AE8
:20C200003D3D3D3D3D3D3D3D3D3D3D3D3D3D3D676C6F62616C2D313D3D3D3D3D3D3D3D3D97
:20C220003D3D3D3D3D3D3D3D3D3D3D3D3D3D3D3D3D3D3D3D3D3D3D3D3D3D3D3D3D3D3D3D5E
:20C240003D3D3D3D3D0A000A4661696C20746F207265616420676C6F62616C203120726585
:20C2600067697374657220256C7520726320256C750A000A3D3D3D3D3D3D3D3D3D3D3D3DFF
:20C280003D3D3D676C6F62616C2D323D3D3D3D3D3D3D3D3D3D3D3D3D3D3D3D3D3D3D3D3D16
:20C2A0003D3D3D3D3D3D3D3D3D3D3D3D3D3D3D3D3D3D3D3D3D3D3D3D3D0A000A4661696CF9
:20C2C00020746F207265616420676C6F62616C203220726567697374657220256C7520727F
:20C2E0006320256C750A000A4661696C20746F20777269746520726567697374657220250D
:20C300006C7520726320256C750A000A0A0A0020534F484F202D207472756E6B44756D7069
:20C32000206465765B256C755D2D205374617274200A007472756E6B496420696E20746887
:20C340006520706F727420636F6E74726F6C200A00706F72745B256C755D202D2D20747245
:20C36000756E6B4964205B256C755D200A007472756E6B20726F757465207461626C6520EF
:20C380000A007472756E6B5B25322E326C755D202D2D20726F757465426D70205B307825DF
:20C3A000332E336C785D205B62696E2025735D0A007472756E6B206D61736B207461626C12
:20C3C00065200A00696E6465785B25322E326C755D202D2D206D61736B426D70205B3078DE
:20C3E00025332E336C785D205B62696E2025735D0A00564C414E5461626C652070657220D0
:20C40000706F7274200A00706F72745B25322E326C755D20564C414E5461626C6520626DF0
:20C42000705B307825332E336C785D205B62696E2025735D0A00207472756E6B44756D70D2
:20C44000202D20456E64200A00204D435F5354415449435F554E4C494D495445445F52415B
:20C46000544500204D435F4D474D5F53544154494300204D435F53544154494300204D4385
:20C480005F5052494F5F5354415449435F554E4C494D495445445F5241544500204D435F38
:20C4A0005052494F5F4D474D5F53544154494300204D435F5052494F5F535441544943006B
:20C4C000756E6B6E6F776E204D4320737461746520307825312E316C780055435F44594E18
:20C4E000414D494320307825312E316C780055435F53544154494320307825312E316C78A1
:20C50000002025346C75207C002025322E326C783A25322E326C783A25322E326C783A2561
:20C52000322E326C783A25322E326C783A25322E326C78207C202573207C307825382E3880
:20C540006C78207C2020307825312E316C752020207C202020307825322E326C7820207CA2
:20C560002025730A0020542000424D500020534F484F202D2061747544756D702064657681
:20C580005B256C755D2D205374617274200A00204552524F52200A0020696E646578207CB0
:20C5A0000020206D616341646472202848455829202020207C54797065207C706F727456E4
:20C5C00065632020207C207072696F207C2044424E756D207C20656E74727953746174657C
:20C5E000200A00206E756D20656E7472696573203A205B256C755D0A0A0020534F484F20C2
:20C600002D2076747544756D70206465765B256C755D2D205374617274200A0020767475B7
:20C6200044756D70202D2D20565455207461626C652064756D70202D2053544152540A00C8
:20C64000564C414E20506F727420656772657373206D656D626572736869703A20256C758F
:20C660002D3E554E4D4F4449462C20256C752D3E554E544147202C256C752D3E5441472C3C
:20C6800020256C752D3E4E4F545F4D454D4245520A0A00564C414E20202020444220202056
:20C6A000202070727430207072743120707274322070727433207072743420707274352047
:20C6C000707274362070727437207072743820707274392070727431302044425F53570A34
:20C6E000002530346C752020202530336C752020202020202025326C752020202025326CAC
:20C70000752020202025326C752020202025326C752020202025326C752020202025326C39
:20C72000752020202025326C752020202025326C752020202025326C752020202025326C19
:20C740007520202025326C7520202025326C750A00565455207263203D256C750A0056541F
:20C7600055207461626C652064756D70202D20454E440A0020534F484F202D206D69727298
:20C780006F7244756D70206465765B256C755D2D205374617274200A0020485720527820B7
:20C7A000616E616C797A657220706F7274205B256C755D0A0020485720547820616E616CDF
:20C7C000797A657220706F7274205B256C755D0A00204857205278206D6F6E69746F72658C
:20C7E0006420706F727473205B307825332E336C785D200A00204857205478206D6F6E69B8
:20C80000746F72656420706F727473205B307825332E336C785D200A0020485720706F722B
:20C82000747320746861742044454E5920554320666C6F6F64205B307825332E336C785DE7
:20C84000200A0020485720706F72747320746861742044454E59204D4320666C6F6F642072
:20C860005B307825332E336C785D200A00206D6972726F7244756D703A20456E64200A0A9B
:20C88000002068656C7044756D70203A74686520737570706F727465642066756E637469EF
:20C8A0006F6E73206172653A200A0025730A0068656C7044756D7000736F686F44756D703C
:20C8C000506F72745265677300736F686F44756D70476C6F625265677300736F686F44754C
:20C8E0006D70416C6C506F7274416E64476C6F625265677300736F686F536574506F7274EB
:20C9000052656700736F686F536574476C6F6252656700736F686F536574476C6F62325285
:20C920006567007472756E6B44756D700061747544756D700076747544756D70006D697244
:20C94000726F7244756D7000E52B30240104F82328245CF582E43492F5837593082290085F
:20C9600092593024049008925CE475F00112008A60020080D360E6C52F7002152E14C52F5C
:20C98000202405FF0200D88C9008925974FFF5F002008A77FF0206A8EFE52C6006D52C03F2
:20C9A0007F00222024101200D840EF6008052FE52F7002052E229008925912008A5712006A
:20C9C00080D3FF60E590089259E475F00112008A6080D71200C9A3EFC0E01200C994D0E074
:20C9E00040F18091D2248002C2249008925912008A8EE4F52DF52BF52EF52F752C00C223F7
:20CA0000C221C222C2251200C95EFF7005AF2D7E0022B425321200C95EFF24D0B40A0050FA
:20CA20000C75F00AC52CA4252CF52C80E824CFB41A00EF5002C2E50200CC7ED22280D6D2FB
:20CA40002180D2D22580CEEF1200C99450091200C9D3EF600F80A4EFC0E01200C9A3D0E07A
:20CA60006F6098EF70040200CAEE1200C975809D1200C9A3EF6077E52C7008052C80041231
:20CA800000C9A3EF60172025111200C948E475F00112008A60EF12008124D52CE220250433
:20CAA000052B052D80AF1200C999EFC0E01200C994D0E050051200C975E4FF2025111200D3
:20CAC000C948E475F00112008A60EF12008124EF70D4202504052B052D0200CA55E52C60E9
:20CAE00002052C1200C9D31200C999EF70BD302405E41200C975E52D60030200CA0D7EFF6D
:20CB00007FFF2220251474FFFCFDFEFF1200C94812008A571200843C052B0200C9FBD0E025
:20CB200080CC7900800A7910800679088002790AD226E52C6002052CE9C0E01200C9D3EF4F
:20CB400060DC1200C9A3BF2D04D2238003BF2B0B1200C9D3EF60C71200C999D0E0B40A0216
:20CB60008034B40802802FBF302870027408C226C0E01200C999D0E0BF78028003BF5816FA
:20CB8000052CD52C028007D52C04D226800B7410801B7002740ABF000BEFF8E4FCFDFEFFB8
:20CBA0000200CC26C0E0EF1200C975D0E0F9E4FCFDFEFFE9C0E0ECC0E0EDC0E0EEC0E0EF00
:20CBC000C0E01200C999EFF8D0E0FFD0E0FED0E0FDD0E0FCD0F0E8604DB461004007B47BC4
:20CBE000005002C2E524D0503DFA24F6500724F95034240AFAEAB5F000502BCFA9F0A42F42
:20CC0000FF92D5E9C5F0CEA4A2D53EFE92D5E9C5F0CDA4A2D53DFD92D5E9C5F0CCA4A2D5D8
:20CC20003CFCC226808DE8C0E0202530202609052D302304120083C41200C94812008A5783
:20CC4000052B20210C20220FEE8FF01200827E800B1200843C8005EF12008124D0E012003D
:20CC6000C9750200C9FB2025131200C94812008A57052BE52E852FF01200827E80E41200D3
:20CC800085A5CADD53CB2658CA3F4CCA3B42CA1548CB2A4FCB2E44CA7043CB2249CB2E55E2
:20CCA000CB0346CB0345CB0347CA432ACC664E0000CA474C6F77657374004C6F77004E6F03
:20CCC000726D616C004869676800506F727420426173656420516F530049454545203830B1
:20CCE000322E317020426173656420516F5300485454502F312E3020323030204F4B0D0A80
:20CD0000507261676D613A206E6F2D63616368650D0A436F6E74656E742D547970653A2048
:20CD2000746578742F68746D6C0D0A436F6E6E656374696F6E3A20636C6F73650D0A0D0A85
:20CD40003C68746D6C3E0A3C736372697074206C616E67756167653D4A6176615363726915
:20CD600070743E0A66756E6374696F6E206765747061676528290A7B0A20646F63756D65A7
:20CD80006E742E716F732E7375626D697428293B0A7D0A3C2F7363726970743E0A3C6C69F8
:20CDA0006E6B2072656C3D7374796C65736865657420687265663D666F726D2E6373733E45
:20CDC0000A3C666F726D206E616D653D716F73206D6574686F643D504F53543E0A203C74CC
:20CDE00061626C653E0A203C74642077696474683D3330303E3C68313E25733C2F68313EE8
:20CE00000A203C74643E0A203C73656C656374206E616D653D716F7374797065206F6E633D
:20CE200068616E67653D6765747061676528293E0A0073656C65637465640000203C6F70B8
:20CE400074696F6E2076616C75653D25642025733E25730A00203C2F73656C6563743E0A2A
:20CE6000203C2F7461626C653E0A3C696E70757420747970653D68696464656E206E616D84
:20CE8000653D706F73745F75726C2076616C75653D6367695F716F732E3E0A3C2F666F72F1
:20CEA0006D3E0A0025730A000A20203C73656C656374206E616D653D70253032643E0A0074
:20CEC00020203C6F7074696F6E2076616C75653D25642025733E25730A0090007004E0F5C9
:20CEE0004090007005E0F541854082854183E020E7077E007F00C2D72289428A435407F5B9
:20CF0000451200D0D5E02402F544500205451200CF7C053AE53A7002053BE5402544F5400A
:20CF2000E541354530E604C2E6242FF5411200CF9C90007004E540F090007005E541F0AEA7
:20CF400045AF44D2D72290007010E020E61EA3EDF0A3E9F0A3EAF0EC5407D2E69000701032
:20CF6000F00538E53870020539D2D7227C007D00C2D72290007010E0A2E6B32275F0018005
:20CF80000375F0041200CF9C78407F06900070921200D0BD90007090E5F0F0229000709033
:20CFA000E0540770F7221200D00990007008742FF0900070107508101200CFF4E4900070D1
:20CFC00004F090007006F0742F90007005F090007007F0751D10751C10751E00751F2F75CA
:20CFE000832F758200E4F0753800753900753A00753B0022E4A808F0A3D8FC221200D0B326
:20D000001200CFA61200D047229000D03D75080A797078601200D0C47518C07519A8751AA1
:20D0200000751B647510C07511A87512007513017514FF7515FF7516FF75170022000B78AD
:20D04000667788C0A800649000706AE0440CF0229000706AE054F3F0229000706AE04401C1
:20D06000F0229000706AE054FEF0229000706AE04402F0229000706AE054FDF022900070A1
:20D080006AE04440F0229000706AE054BFF02290007000E04410F02290007000E054EFF0E8
:20D0A0002290007000E04420F02290007000E05420F0229000700AF00000000022E6F00898
:20D0C000A3DFFA2289A0E493A3F208B800030989A0D508F222A3E58330E60375832F2247E3
:20D0E00045542000696E6465782E68746D00706F73745F75726C3D002E006367695F6C6F98
:20D10000676F757400636F6E6669672E62696E006367695F62616B5F646174610063676987
:20D120005F0066617669636F6E2E69636F006367695F6C6F67696E004C6F67696E004F6EE0
:20D140006C79206F6E6520757365722063616E206C6F67696E006367695F6465766963651C
:20D160000077726F6E672070617373776F726400496E76616C69642061636365737320492D
:20D18000502061646472657373006C6F67696E2074696D656F7574006367695F706F7274A2
:20D1A000006367695F64656C766C616E006367695F766C616E006367695F7472756E6B00EE
:20D1C0006367695F6D6972726F72006367695F737973006367695F737470006367695F7046
:20D1E000617373006367695F716F73006367695F717062617365006367695F7131700063EE
:20D2000067695F736E6D70006367695F61636C006367695F64656C61636C006367695F7363
:20D2200065747674797065006367695F70766964006367695F736574766964006367695FE5
:20D24000766964006367695F64656C766964006367695F7265736574006367695F737772DE
:20D2600065736574006367695F636C7273746174006367695F73746174697374006367699D
:20D280005F616464766C616E006367695F736574766C616E006367695F7365747669643D68
:20D2A00025640053797374656D20626F6F747570004C6F67696E20696E76616C6964207017
:20D2C000617373776F72642066726F6D2025642E25642E25642E25640052656D6F7465201D
:20D2E00049503A2025642E25642E25642E256400506F727420256420666962657220696E20
:20D3000073657274656400506F72742025642066696265722072656D6F76656400506F72CD
:20D3200074202564206669626572206C696E6B20757000506F72742025642066696265725F
:20D34000206C696E6B20646F776E00506F72742025642066696265722072656365697665AE
:20D36000206572726F7200506F7274202564206669626572207472616E736D697420657264
:20D38000726F7200506F727420256420636F707065722072656365697665206572726F72F6
:20D3A00000506F727420256420636F70706572207472616E736D6974206572726F7200504A
:20D3C0006F727420256420636F70706572206C696E6B20757000506F727420256420636F93
:20D3E00070706572206C696E6B20646F776E0075C7AA75C755759D0275C7AA75C75575C693
:20D4000000787FE4F6D8FD755004755100758151D20D0200D4400202B9FBE493A3F8540776
:20D42000240CC8C333C4540F4420C8834004F456800146F6DFE4800C01020408102040808F
:20D4400090009417E47E019360CCA3FF543F30E509541FFEE493A360010ECF54E0B4E02A61
:20D46000E493FBA3E493FAA3E493F9A3E493C083C082C09312008124D093D082D083A309B6
:20D48000E970010ADFE6DEE480BA54C025E0602B4088E493A3FAE493A3F8E493A3C8C582AC
:20D4A000C8CAC583CA759308F0759300A3C8C582C8CAC583CADFE3DEE18089E493A3F8E4EA
:20D4C00093A34003F68001F208DFF40200D4442872627429637265617465205242545B25E0
:20D4E000705D20616E6420726F6F745B25705D0A002872627429616464206B65795B2570B6
:20D500005D2C206C6566745B25705D2C2072696768745B25705D0A002872627429726F6FC0
:20D5200074206B65795B25705D2C206C6566745B25705D2C2072696768745B25705D0A00BC
:20D54000783D25702C782D3E6C6566743D25702C782D3E72696768743D25702C782D3E6B7C
:20D5600065793D25700A006C6F676F2E67696600696E6465782E68746D006C6566742E680C
:20D58000746D00746F702E68746D0068656C702E68746D00666F6C642E67696600666F7270
:20D5A0006D2E637373006C6566742E6373730068656C702E637373006461726B626C7565FB
:20D5C0002E676966006E6574676561722E6A7067006D6F64656C2E6A706700752E67696639
:20D5E00000622E67696600742E6769660068656C6C6F3F3F3F0068696869232323006D61E3
:20D600006320777269746500676F206C6F6164657200636C6F7365746D006D6163207265D0
:20D620006164002573006D6163006D6F64656C2072656164006D6F64656C3A00667776658C
:20D640007220726561640066777665723A00726263686B004661696C004F6B000A0A776508
:20D6600062207365727665722072756E6E696E672E2E2E205B25645D0A000A537973746559
:20D680006D20696E6974206661696C7572652E0A00496E69742066696E69736865642E0AD3
:20D6A000005B54494D4525643A2044256420204825643A4D25643A5325645D0A005262548A
:20D6C0007265652052656C65617365204D656D426C6F636B2025700A0052625472656520E0
:20D6E000416C6C6F63617465204E6F6465204641494C0A0052625472656520416C6C6F63CA
:20D70000617465204E6F646520535543434553532025700A009008ADBCE0FFA3E0FEA3E04D
:20D72000CF9008945DF0A3EEF0A3EFF09008ADBFE0CBF0A3E0CAF0A3E0C9F07F22900894B9
:20D7400060AD82AC83120080D38D828C83F0A309E970010ADFEB9008ADBFE0FBA3E0FAA3BF
:20D76000E0F902008B137374617274202D2D20736574206D616320656E74727921210A002D
:20D78000736574206D616320656E747279206661696C21210A007365742067707274506FAA
:20D7A0007274466C6F77436E74726C4175746F4E6567456E61626C65206661696C0A00EF39
:20D7C000B40A08740D1200D7CB740A309811A899B8130CC2983098FDA899C298B811F63036
:20D7E00099FDC299F59922310032202D3E2064657625640A00330034003500360037003867
:20D80000003900313000313100E94A4B700122120080D3FF6D700122EF7004FBFAF922091B
:20D82000E970EC0A80E946455F2564004762455F256400566C616E31007075626C696300A6
:20D8400010290D1200D882BF0D027F0A0200D7BF9008B0ACE0FF22E4FFFE120080D3600C80
:20D860000FEF70010E09E970F10A80EE22257320257300465337353054320056312E312E1F
:20D8800036003098FDAF99C2987E00229008B0ACEFF0D22922900806ABE0FBA3E0FAA3E037
:20D8A000F912008204FFAEF0E5F0600301F2A1EF120085A5D90601DD5102DDB403DDD507E6
:20D8C000DE3008E06A09E0EE0AE2B90BE3760CE6CE0DE7210EE9910FECA810ECA814ECA8BC
:20D8E00015EE7416F0AF17F16219F1621CF1621FF1CB20F1DB21F25722F26423F26432F271
:20D9000064330000F2A19008945D7487F0A374E6F0A37492F090086D39E0FBA3E0FAA3E0CA
:20D92000F912008B1390086E5AEEF0A3EFF0E49008883FF0A3F09008883FE475F0011200FD
:20D9400081D8AFF0FE600301DD3EEF14B40D00400301DD3E9000D96375F004A4C58325F0F9
:20D96000C583730200D9970200D9AD0200D9D30200DA070200DA430200DA580200DA6D02C3
:20D9800000DA8B0200DA9B0200DB310200DB4C0200DB6C0200DB99900888607487F0A37433
:20D9A000E8F0A374CDF01206A3D101DB44900888607487F0A374E8F0A374DAF07E007F28AF
:20D9C0007D007B097A887963120089B11206A40B01DB44900888607487F0A374E8F0A374C4
:20D9E000EBF09008945D7487F0A374E8F0A374FCF0A3E4F0A37402F0A3E4F0A304F0A3E4D1
:20DA0000F0A3740301DCAB900888607487F0A374E9F0A37409F01206ADAFEF64014E70087B
:20DA20007B877AE9790E80067B877AE97915C003C002C00178637C887D09D001D002D00360
:20DA400001DB65900888607487F0A374E9F0A3741DF01206AA0D8028900888607487F0A381
:20DA600074E9F0A37428F01206AA1D8013900888607487F0A374E9F0A37434F01206AA2D33
:20DA80009008888C1200850B01DC2D90088840E004F070079008883FE004F090088860745C
:20DAA00087F0A374E9F0A37444F07B097A88796312069B979008945D7487F0A374E9F0A301
:20DAC0007450F090088863E0FF3395E090089460E4F0A3EFF090088864E0FF3395E0900803
:20DAE0009462E4F0A3EFF090088865E0FF3395E090089464E4F0A3EFF090088866E0FF3350
:20DB000095E090089466E4F0A3EFF090088867E0FF3395E090089468E4F0A3EFF090088890
:20DB200068E0FF3395E09008946AE4F0A3EF01DCAB900888607487F0A374E9F0A3746EF0A2
:20DB40001206AEA578637C887D098019900888607487F0A374E9F0A3747AF01206AEAC7896
:20DB6000637C887D09120087F301DCB6900888607487F0A374E9F0A37488F01206AD9D90BD
:20DB8000089460EEF0A3EFF09008945D7487F0A374E9F0A374A001DCAB900888607487F01B
:20DBA000A374E9F0A374A3F09008A3D97409F0A37488F0A37492F0A37409F0A37488F0A3E0
:20DBC0007494F0A37409F0A37488F0A37496F07B097A88799012066E999008945D7487F0EF
:20DBE000A374E9F0A374B1F090088890E0FFA3E090089460CFF0A3EFF090088892E0FFA36A
:20DC0000E090089462CFF0A3EFF090088894E0FFA3E090089464CFF0A3EFF090088896E0D8
:20DC2000FFA3E090089466CFF0A3EF807E9008945D7487F0A374E9F0A374D5F09008888C95
:20DC4000E0FCA3E0FDA3E0FEA3E0FF7818120083F9E490089460F0A3EFF09008888CE0FCDD
:20DC6000A3E0FDA3E0FEA3E0FF7810120083F9E490089462F0A3EFF09008888CE0FCA3E01C
:20DC8000FDA3E0FEA3E0FF7808120083F9E490089464F0A3EFF09008888CE0FCA3E0FDA3E5
:20DCA000A3E0FEE490089466F0A3CEF07B097A88796312008B137B097A8879631200D85767
:20DCC000EF4E701078637C887D097B877AE979E1120087F390086D39E0FBA3E0FAA3E0F9C5
:20DCE00090086E5AE0FEA3E0FFE92FF9EA3EFAC002C0019008945D7487F0A374E9F0A37433
:20DD0000E8F090088860E0F9A3E0FAA3E090089460C9F0A3EAF0A3E9F0A37409F0A37488E5
:20DD2000F0A37463F0D001D00212008B1390086E5BE02FF090086E5AE03EF001D9369008C0
:20DD400006ABE0FBA3E0FAA3E0F9E475F00201E71A90086D39E0FBA3E0FAA3E0F990086ED9
:20DD60005AE0FEA3E0FFE92FF9EA3EFA9008945D7487F0A374EAF0A37402F012008B139008
:20DD8000086E5BE02FF090086E5AE03EF0900806ABE0FBA3E0FAA3E0F9E475F00312008248
:20DDA0007E900806BCE0FBA3E0FAA3E0F9E475F00101E71AE4FFFE120304F5EF4E7002FFCE
:20DDC00022900806ABE0FBA3E0FAA3E0F9E475F0071200827E1206ADA6EF4E700301E06A3C
:20DDE0009008945D7487F0A374EAF0A37451F090086D39E0FBA3E0FAA3E0F912008B139014
:20DE0000086E5AEEF0A3EFF0900806ABE0FBA3E0FAA3E0F9E475F0081200827E900806BCF8
:20DE2000E0FBA3E0FAA3E0F9E475F0011200827E900806BCE0FBA3E0FAA3E0F912008204EC
:20DE4000C39401FFE5F09400FE9008888CF0A3EFF09008A6E47409F0A37488F0A3748EF033
:20DE60007B097A8879471205FF55EF4E702B900806ABE0FBA3E0FAA3E0F9E475F009120098
:20DE8000827ED390086E5BE0940090086E5AE09400500301EC917F00229008888EE0FBA368
:20DEA000E0FAA3E0F91200D857EF4E700F9008888E7487F0A374E9F0A374E1F090086D3960
:20DEC000E0FBA3E0FAA3E0F990086E5AE0FEA3E0FFE92FF9EA3EFAC002C0019008945D74FB
:20DEE00087F0A374EBF0A37403F09008888DE02401FE9008888CE0340090089460F0A3CE52
:20DF0000F09008888EE0F9A3E0FAA3E090089462C9F0A3EAF0A3E9F0D001D00212008B13F7
:20DF200090086E5BE02FF090086E5AE03EF0E490088845F0A3F0C390088AC9E09401FF9095
:20DF4000088AC8E09400FE90088845E0FCA3E0FDC39FEE6480F8EC648098400301E003ED8C
:20DF6000AE047803CEA2E713CE13D8F82447F58274883EF583759308E0FD7C0090088846F6
:20DF8000E05407FF74017E00A807088005C333CE33CED8F9FFEE5CFEEF5D4E605390086DE9
:20DFA00039E0FBA3E0FAA3E0F990086E5AE0FEA3E0FFE92FF9EA3EFA9008945D7487F0A34A
:20DFC00074EBF0A37430F090088846E02401FE90088845E0340090089460F0A3CEF01200EA
:20DFE0008B1390086E5BE02FF090086E5AE03EF090088846E004F0700790088845E004F0CB
:20E0000001DF3690086D39E0FBA3E0FAA3E0F990086E5AE0FEA3E0FFE92FF9EA3EFA90084D
:20E02000945D7487F0A374EBF0A37436F012008B1390086E5BE02FF090086E5AE03EF090C7
:20E040000806BCE0FBA3E0FAA3E0F9E475F00112008252C390086E5BE094B090086E5AE06A
:20E060009404500301DE307F00221206ADA6EF64014E700301E6CE9008945D7487F0A37445
:20E08000EBF0A37439F090086D39E0FBA3E0FAA3E0F912008B1390086E5AEEF0A3EFF012D1
:20E0A0000619E1900806ABE0FBA3E0FAA3E0F9E475F00A1200827E900806BCE0FBA3E0FA2C
:20E0C000A3E0F9E475F0011200827EC390088AC9E09401FF90088AC8E09400F9900806B59C
:20E0E000E0FBA3E0FAA3E0C98FF01200827E900806B5E0FBA3E0FAA3E0F912008204FFAE7F
:20E10000F0900806BCE0FBA3E0FAA3E0F912008204D39FE5F09E402B900806ABE0FBA3E052
:20E12000FAA3E0F9E475F00B1200827ED390086E5BE0940090086E5AE09400500301E2B998
:20E140007F002290086D39E0FBA3E0FAA3E0F990086E5AE0FEA3E0FFE92FF9EA3EFA900881
:20E16000945D7487F0A374EBF0A37495F012008B1390086E5BE02FF090086E5AE03EF0E4D3
:20E180009008883FF0A3F0900806B5E0FBA3E0FAA3E0F912008204FFAEF0900806BCE0FB0C
:20E1A000A3E0FAA3E0F912008204FDACF0D39FEC9E5079C3ED9401FFEC9400FE7B097A8828
:20E1C000794E12068C8790086D39E0FBA3E0FAA3E0F990086E5AE0FEA3E0FFE92FF9EA3E42
:20E1E000FAC003C002C0019008945D7487F0A374EBF0A374A9F0900806BCE0FBA3E0FAA374
:20E20000E0F912008204FF90089460E5F0F0A3EFF09008884EE0540FFFA3E090089462CF2B
:20E22000F0A3EFF0D001D002D003802A90086D39E0FBA3E0FAA3E0F990086E5AE0FEA3E079
:20E24000FFE92FF9EA3EFA9008945D7487F0A374EBF0A374BFF012008B1390086E5BE02F40
:20E26000F090086E5AE03EF0900806BCE0FBA3E0FAA3E0F9E475F001120082529008884082
:20E28000E004F070079008883FE004F0C390088840E094049008883FE064809480500301DA
:20E2A000E187C390086E5BE094B090086E5AE09404500301E0EE7F0022C390088AC9E094F1
:20E2C00001FF90088AC8E09400F9900806B5E0FBA3E0FAA3E0C98FF01200827E90086D3921
:20E2E000E0FBA3E0FAA3E0F990086E5AE0FEA3E0FFE92FF9EA3EFAC003C002C001900894E5
:20E300005D7487F0A374EBF0A374D6F0900806B5E0FBA3E0FAA3E0F912008204FFE5F0C390
:20E3200013FEEF13FF90089460EEF0A3EFF0D001D002D00312008B1390086E5BE02FF090C9
:20E34000086E5AE03EF0900806BCE0FBA3E0FAA3E0F9E475F0011200827E900806ABE0FB31
:20E36000A3E0FAA3E0F9E475F00C1200827EE49008ACAAF0A3F0900806BCE0FBA3E0FAA393
:20E38000E0F912008204C39401FFE5F09400FE7B097A88795012066287EF4E702B90080688
:20E3A000ABE0FBA3E0FAA3E0F9E475F00D1200827ED390086E5BE0940090086E5AE09400FA
:20E3C000500301E6CE7F00229008ACAAE07002A3E090086D397038E0FBA3E0FAA3E0F99087
:20E3E000086E5AE0FEA3E0FFE92FF9EA3EFA9008945D7487F0A374ECF0A3748DF09008889F
:20E4000050E0FFA3E090089460CFF0A3EF8025E0FBA3E0FAA3E0F990086E5AE0FEA3E0FF34
:20E42000E92FF9EA3EFA9008945D7487F0A374EBF0A37495F012008B1390086E5BE02FF097
:20E4400090086E5AE03EF09008883FE4F0A304F0900806B5E0FBA3E0FAA3E0F912008204C5
:20E46000FFE5F0C313FEEF13FF9008883FE0FCA3E0FDD39FEC9E506590086D39E0FBA3E0EB
:20E48000FAA3E0F990086E5AE0FEA3E0FFE92FF9EA3EFA9008945D7487F0A374ECF0A37495
:20E4A000B3F09008ACAAE0FEA3E0FFED2FFFEC3E90089460F0A3EFF012008B1390086E5B17
:20E4C000E02FF090086E5AE03EF090088840E004F070079008883FE004F001E45090086DB7
:20E4E00039E0FBA3E0FAA3E0F990086E5AE0FEA3E0FFE92FF9EA3EFA9008945D7487F0A305
:20E5000074EBF0A37495F012008B1390086E5BE02FF090086E5AE03EF0E490088841F0A3BA
:20E52000F0900806B5E0FBA3E0FAA3E0F912008204FFE5F0C313FEEF13FF90088841E0FC46
:20E54000A3E0FDC39FEC9E400301E67F9008ACAAE0FAA3E0FBED2BFFEC3AFEEF7803CEC32A
:20E5600013CE13D8F9FF90088843EEF0A3EFF0ED2BFFEF5407FFA3E4F0A3EFF09008884457
:20E58000E02459F582E43488F583759308E0FD7C0090088846E0FF74017E00A807088005B2
:20E5A000C333CE33CED8F9FFEE5CFEEF5D4E6011900888607487F0A374ECF0A374C1F080CD
:20E5C0005090088844E02452F582E43488F583759308E0FD7C0090088846E0FF74017E0001
:20E5E000A807088005C333CE33CED8F9FFEE5CFEEF5D4E90088860600D7487F0A374ECF09D
:20E60000A374C3F0800B7487F0A374E9F0A374E1F090086D39E0FBA3E0FAA3E0F990086ECA
:20E620005AE0FEA3E0FFE92FF9EA3EFAC002C0019008945D7487F0A374ECF0A374C5F090A7
:20E64000088860E0F9A3E0FAA3E090089460C9F0A3EAF0A3E9F0D001D00212008B139008C8
:20E660006E5BE02FF090086E5AE03EF090088842E004F0700790088841E004F001E52190EB
:20E6800008ACAAE07002A3E07025900806B5E0FBA3E0FAA3E0F912008204FFE5F0C313FE4B
:20E6A000EF13FF9008ACAAEEF0A3EFF001E376E49008ACAAF0A3F0900806BCE0FBA3E0FAAA
:20E6C000A3E0F9E475F001120082527F00229008945D7487F0A374ECF0A374CDF090086DAD
:20E6E00039E0FBA3E0FAA3E0F912008B1390086E5AEEF0A3EFF0900806BCE0FBA3E0FAA348
:20E70000E0F9E475F0011200827E900806ABE0FBA3E0FAA3E0F9E475F00E1200827E7F00BF
:20E7200022E490088845F0A3F0E49008888BF090088846E0FF7B097A8879471205DCF99065
:20E74000088846E0FF1206AA7DEF60087B877AED79A980067B877AED79B190089462EBF061
:20E76000A3EAF0A3E9F090086D39E0FBA3E0FAA3E0F990086E5AE0FEA3E0FFE92FF9EA3E95
:20E78000FA9008945D7487F0A374EDF0A3746BF090088846E02401FE90088845E034009033
:20E7A000089460F0A3CEF012008B1390086E5BE02FF090086E5AE03EF090088846E025E043
:20E7C000FF90088845E033FE74562FF582748B3EF583759308E0FEA3E0C39401FFEE940055
:20E7E0009008883FF0A3EFF090088846E025E0FF90088845E033FE74952FF582748B3EF5A7
:20E8000083759308E0FEA3E0FF9008883FE0FCA3E0FDC39FEE6480F8EC648098400301E88A
:20E82000CCEDAE047803CEA2E713CE13D8F82447F58274883EF583759308E0FD7C00900842
:20E840008840E05407FF74017E00A807088005C333CE33CED8F9FFEE5CFEEF5D4E605A90C6
:20E8600008888B7401F090086D39E0FBA3E0FAA3E0F990086E5AE0FEA3E0FFE92FF9EA3E0D
:20E88000FA9008945D7487F0A374EBF0A37430F090088840E02401FE9008883FE03400907B
:20E8A000089460F0A3CEF012008B1390086E5BE02FF090086E5AE03EF090088840E004F059
:20E8C00070079008883FE004F001E7E89008888BE0703C90086D39E0FBA3E0FAA3E0F990E5
:20E8E000086E5AE0FEA3E0FFE92FF9EA3EFA9008945D7487F0A374EDF0A374BAF012008BEF
:20E900001390086E5BE02FF090086E5AE03EF090088846E004F0700790088845E004F0C369
:20E9200090088846E0940790088845E064809480500301E729900806ABE0FBA3E0FAA3E031
:20E94000F9E475F00F1200827E90086E5AE0FEA3E0FFD39400EE9400500301F2A490086DBC
:20E9600039E0FBA3E0FAA3E02FF9EA3EFA9008945D7487F0A374EDF0A374BEF012008B135C
:20E9800090086E5BE02FF090086E5AE03EF07F0022900806ABE0FBA3E0FAA3E0F9E475F0A2
:20E9A0000F1200827E78A47C887D097B817A9379577E007F0C12008055E49008888CF0A3A4
:20E9C000F0FE7F07FD7B097A887947120089B17E007F077D007B097A88799C120089B1903C
:20E9E00008AA1A7409F0A37488F0A37495F0A37402F07B097A8879A3E4FF12063E3E789584
:20EA00007C887D097B097A88799C7E007F0712008927EF601F9008888CE0F0A3E04402F068
:20EA200078477C887D097B097A8879957E007F07120080559008AA1A7409F0A37488F0A313
:20EA4000748EF0A37401F07B097A8879A3E4FF12063E3E788E7C887D097B097A88799C7EFA
:20EA6000007F0712008927EF601F9008888CE0F0A3E04401F078477C887D097B097A887964
:20EA80008E7E007F07120080559008945D7487F0A374EDF0A374DCF09008888CE0FEA3E0A5
:20EAA000900888A475F00312008528EE75F003A42583F583759308E0F9A3E0FAA3E09008D0
:20EAC0009460C9F0A3EAF0A3E9F090086D39E0FBA3E0FAA3E0F912008B1390086E5AEEF090
:20EAE000A3EFF09008888CE07002A3E0701278637C887D097B877AE979E1120087F3802A37
:20EB00009008945D7487F0A374EEF0A374AAF0900888A3E004FFF090089460E4F0A3EFF063
:20EB20007B097A88796312008B1390086D39E0FBA3E0FAA3E0F990086E5AE0FEA3E0FFE908
:20EB40002FF9EA3EFA9008945D7487F0A374EEF0A374AFF0A37409F0A37488F0A37463F043
:20EB600012008B1390086E5BE02FF090086E5AE03EF09008888CE07002A3E0703F90086DE2
:20EB800039E0FBA3E0FAA3E0F990086E5AE0FEA3E0FFE92FF9EA3EFA9008945D7487F0A35E
:20EBA00074E9F0A374E1F012008B1390086E5BE02FF090086E5AE03EF001EC91E490088820
:20EBC00045F0A3F0C390088AC9E09401FF90088AC8E09400FE90088845E0FCA3E0FDC39FCC
:20EBE000EE6480F8EC648098400301EC91EDAE047803CEA2E713CE13D8F82447F58274880F
:20EC00003EF583759308E0FD7C0090088846E05407FF74017E00A807088005C333CE33CE41
:20EC2000D8F9FFEE5CFEEF5D4E605390086D39E0FBA3E0FAA3E0F990086E5AE0FEA3E0FF9D
:20EC4000E92FF9EA3EFA9008945D7487F0A374EBF0A37430F090088846E02401FE9008885B
:20EC600045E0340090089460F0A3CEF012008B1390086E5BE02FF090086E5AE03EF0900848
:20EC80008846E004F0700790088845E004F001EBC4900806ABE0FBA3E0FAA3E0F9E475F00C
:20ECA000011200825201F2A49008945D7487F0A374EFF0A3740AF090086D39E0FBA3E0FAC5
:20ECC000A3E0F912008B1390086E5AEEF0A3EFF07B097A88798B1206AD829008888BE0707C
:20ECE0004F90086D39E0FBA3E0FAA3E0F990086E5AE0FEA3E0FFE92FF9EA3EFA9008945D37
:20ED00007487F0A374EFF0A37443F012008B1390086E5BE02FF090086E5AE03EF0900806AC
:20ED2000ABE0FBA3E0FAA3E0F9E475F01701F2557B097A88798B1206AD8B1206AC9CC007AB
:20ED4000C0061206ACA6C007C0061206ACB0C007C0061206ACBA90089469EEF0A3EFF090F2
:20ED6000089467D0E0F0A3D0E0F090089465D0E0F0A3D0E0F090089463D0E0F0A3D0E0F0C7
:20ED800090086D39E0FBA3E0FAA3E0F990086E5AE0FEA3E0FFE92FF9EA3EFAC003C002C029
:20EDA000019008945D7487F0A374EFF0A374BBF09008888BE0B401087B877AE9790E80066C
:20EDC0007B877AE9791590089460EBF0A3EAF0A3E9F0D001D002D00312008B1390086E5B59
:20EDE000E02FF090086E5AE03EF090086D39E0FBA3E0FAA3E0F990086E5AE0FEA3E0FFE9EB
:20EE00002FF9EA3EFA9008945D7487F0A374F0F0A374DFF012008B1390086E5BE02FF090B7
:20EE2000086E5AE03EF012061A86900806ABE0FBA3E0FAA3E0F9E475F0161200827E900816
:20EE400006BCE0FBA3E0FAA3E0F9E475F0011200827EC390088AC9E09401FF90088AC8E0D4
:20EE60009400F9900806B5E0FBA3E0FAA3E0C98FF001F25578907C887D097B817A937963D0
:20EE80007E007F1212008055900806B5E0FBA3E0FAA3E0F912008204FFAEF0900806BCE0E6
:20EEA000FBA3E0FAA3E0F912008204C39FE5F09E400301F08790086D39E0FBA3E0FAA3E01D
:20EEC000F990086E5AE0FEA3E0FFE92FF9EA3EFA9008945D7487F0A374EBF0A37495F01232
:20EEE000008B1390086E5BE02FF090086E5AE03EF0E49008883FF0A3F0900806B5E0FBA30F
:20EF0000E0FAA3E0F912008204FFAEF0900806BCE0FBA3E0FAA3E0F912008204FDACF0D334
:20EF20009FEC9E400301F00EC3ED9401FF7B097A88798C1206A37A900806BCE0FBA3E0FAB0
:20EF4000A3E0F912008204C39401FF7B097A88798E1206A6D5900806BCE0FBA3E0FAA3E0F1
:20EF6000F912008204C39401FF7B097A88798F1206A94F90086D39E0FBA3E0FAA3E0F99069
:20EF8000086E5AE0FEA3E0FFE92FF9EA3EFAC003C002C0019008945D7487F0A374F1F0A3B9
:20EFA0007440F0900806BCE0FBA3E0FAA3E0F912008204FF90089460E5F0F0A3EFF090087D
:20EFC000888CE0FFA3E090089462CFF0A3EFF09008888EE0FF90089464E4F0A3EFF09008E1
:20EFE000888FE075F003A42490F582E43488F583759308E0F9A3E0FAA3E090089466C9F097
:20F00000A3EAF0A3E9F0D001D002D003802A90086D39E0FBA3E0FAA3E0F990086E5AE0FE87
:20F02000A3E0FFE92FF9EA3EFA9008945D7487F0A374F1F0A37467F012008B1390086E5B30
:20F04000E02FF090086E5AE03EF0900806BCE0FBA3E0FAA3E0F9E475F0011200825290084D
:20F060008840E004F070079008883FE004F0C390088840E094049008883FE0648094805028
:20F080000301EEF97F0022900806ABE0FBA3E0FAA3E0F9E475F00112008252D390086E5B63
:20F0A000E0940090086E5AE09400400301F2A490089F1EE0FEA3E0FFEE600301F162EF14D1
:20F0C000605404600301F1629008945D7487F0A374F1F0A3747EF090086D39E0FBA3E0FA3A
:20F0E000A3E0F912008B1390086E5AEEF0A3EFF0900806BCE0FBA3E0FAA3E0F9E4F5F0121B
:20F1000000827E90089F1FE004F0700790089F1EE004F07F00221202F85A900806BCE0FBE9
:20F12000A3E0FAA3E0F9E475F00112008252900806BCE0FBA3E0FAA3E0F912008204640478
:20F1400045F0701B90089F1EF0A3F0900806ABE0FBA3E0FAA3E0F9E475F0191200827E7F07
:20F1600000221206AE7BEF707290086D39E0FBA3E0FAA3E0F990086E5AE0FEA3E0FFE92F71
:20F18000F9EA3EFA9008945D7487F0A374F2F0A3746FF012008B1390086E5BE02FF09008C9
:20F1A0006E5AE03EF0900806BCE0FBA3E0FAA3E0F9E4F5F01200827E900806ABE0FBA3E0C9
:20F1C000FAA3E0F9E475F02001F29BE4FFFE12032F47EF4E600301F264FF221206AE7BEF0E
:20F1E00064016012900806ABE0FBA3E0FAA3E0F9E475F023805F90086D39E0FBA3E0FAA397
:20F20000E0F990086E5AE0FEA3E0FFE92FF9EA3EFA9008945D7487F0A374F2F0A374A1F00D
:20F2200012008B1390086E5BE02FF090086E5AE03EF0900806BCE0FBA3E0FAA3E0F9E4F549
:20F24000F01200827E900806ABE0FBA3E0FAA3E0F9E475F0228044E4FFFE1204AF19EF4E64
:20F260007002FF229008945D7487F0A374F2F0A374D4F090086D39E0FBA3E0FAA3E0F9128F
:20F28000008B1390086E5AEEF0A3EFF0900806ABE0FBA3E0FAA3E0F9E4F5F01200827E8098
:20F2A000037F01227F002290086091EBF0A3EAF0A3E9F07E007FF07D007B097A60799412C4
:20F2C0000089B17E007FF07D007B097A617984120089B19008945D7481F0A374C0F0A37496
:20F2E00042F07B097A62797C12008B1374FF900862B0F0A3F0E4900862A4F0A3F090086238
:20F30000A4E0FEA3E0FFC39404EE64809480502A7C007D3C1200813874842FF974613EFA01
:20F320007B09E0FD12068E2A900862A5E004F070CC900862A4E004F080C390086091E0F9D6
:20F34000A3E0FAA3E09008629EC9F0A3EAF0A3E9F0E4900862A4F0A3F0900862A4E0FAA343
:20F36000E0FBC39404EA64809480400301FCCBE4900862B2F0A3F0FFFEFDFC900862BC1299
:20F3800000850B7C007D3CAF03AE021200813874942FF974603EFA7B09C002C00174842F11
:20F3A000F974613EFA9008945D7409F0A3EAF0A3E9F0D001D00212008B13E4900862A6F091
:20F3C000A3F09008945D7481F0A374C0F0A37442F07B097A62797412008B139008A511745D
:20F3E00081F0A374BBF0A37481F090086091E0FBA3E0FAA3E0F91205F2909008629EEBF0E9
:20F40000A3EAF0A3E9F090089CAB7481F0A374BBF0A37481F0A37481F0A374BAF0A3740D78
:20F42000F0A37409F0A37462F0A37474F0120542FC78747C627D097B097A62797C12008755
:20F4400049EF7022900862A7E025E0FF900862A6E033FE74A82FF58274623EF5837593084E
:20F46000E4F0A3F0802F7B097A6279741205D1DAAC06AD07900862A7E025E0FF900862A6DC
:20F48000E033FE74A82FF58274623EF583759308ECF0A3EDF09008629FE475F00312008129
:20F4A000D89008629EE0F9A3E0FAA3E090086091C9F0A3EAF0A3E9F0900862A7E004F070E3
:20F4C00007900862A6E004F0C3900862A7E09404900862A6E064809480500301F3C29008BC
:20F4E00062A8E07002A3E06051900862A4E0FEA3E0FF7C007D3C1200813874A92FF9746065
:20F500003EFA9008A4097409F0A3EAF0A3E9F07B097A6279A812050357EF4E70459008A8E4
:20F520006F7481F0A374C0F0A37450F0A37481F0A374C0F0A3746601FDB6E4FFFEFDFC906F
:20F540000862A4E0FAA3E0900860A975F03C12008528EA75F03CA42583F5837593081200CE
:20F56000850B9008945D7481F0A374C0F0A37477F0900862A4E0FFA3E090089460CFF0A35A
:20F58000EFF07B097A62798012008B139008A5117409F0A37462F0A37480F09008629EE060
:20F5A000FBA3E0FAA3E0F91205F2909008629EEBF0A3EAF0A3E9F0C002C00190089CAB747C
:20F5C00009F0A37462F0A37480F0A37481F0A374BAF0A3740DF0900862A4E0FEA3E0FF7C6B
:20F5E000007D3C1200813874AD2FF974603EFA90089CB17409F0A3EAF0A3E9F0D001D00244
:20F60000120542FC900862A4E0FEA3E0FF7C007D3C1200813874AD2FF974603EFA90089416
:20F620005D7409F0A3EAF0A3E9F07B097A62798012008B137B097A6279801205472C7B0997
:20F640007A6279801200D857D3EF9414EE64809480403D9008945D7481F0A374C0F0A3747B
:20F660007FF0A3E4F0A37414F07B097A6279C012008B139008A86F7409F0A37462F0A374A4
:20F68000C0F0A37481F0A374C0F0A374A601FDB69008945D7481F0A374C0F0A374AFF0907F
:20F6A0000862A4E0FFA3E090089460CFF0A3EFF07B097A62798012008B139008A511740939
:20F6C000F0A37462F0A37480F09008629EE0FBA3E0FAA3E0F91205F2909008629EEBF0A32F
:20F6E000EAF0A3E9F090089CAB7409F0A37462F0A37480F0A37481F0A374BAF0A3740DF01B
:20F70000A37409F0A37462F0A374B4F0120542FC78B47C627D097B817AC079B61200874989
:20F72000EF900862A4701FE0FEA3E0900860C275F03C12008528EE75F03CA42583F583756A
:20F740009308E4F0801EE0FEA3E0900860C275F03C12008528EE75F03CA42583F5837593C6
:20F76000087401F0900862A4E07002A3E0600301F8689008629EE0F9A3E0FAA3E0A3C9F018
:20F78000A3EAF0A3E9F09008A5117481F0A374C0F0A374B8F090086091E0FBA3E0FAA3E053
:20F7A000F91205F290900862A1EBF0A3EAF0A3E9F0900862A1E0FBA3E0FAA3E04A4B7003CA
:20F7C00001F8689008A5117481F0A374C0F0A374BFF090086091E0FBA3E0FAA3E0F9120594
:20F7E000F290C003C002C001900862A1A3E0FAA3E0F9D3D082D083D0E0E99582EA95834043
:20F80000249008A5117481F0A374C0F0A374BFF090086091E0FBA3E0FAA3E0F91205F2900E
:20F82000E94A4B70439008925C7481F0A374C0F0A374C5F0A37409F0A37462F0A374B0F069
:20F84000900862A1E0FBA3E0FAA3E0F91200C9E47B817AC079B81200D85790086092EE8FCB
:20F86000F0120081D801F7869008629EE0F9A3E0FAA3E090086091C9F0A3EAF0A3E9F07B88
:20F88000817AC079CE900862A4E0FFA3E09008945DCFF0A3EFF0900862B0E0FFA3E09008F8
:20F8A000945FCFF0A3EFF012008B19900862B0E0F47003A3E0F46019E47F01FEFDFC90088A
:20F8C00062B1E0F9F81200840C900862BC1200850B9008629EE0F9A3E0FAA3E0A3C9F0A3DA
:20F8E000EAF0A3E9F09008945D7481F0A374C0F0A374DEF0900862A4E0FFA3E0900894600C
:20F90000CFF0A3EFF07B097A62798012008B139008A5117409F0A37462F0A37480F090085A
:20F920006091E0FBA3E0FAA3E0F91205F2909008629EEBF0A3EAF0A3E9F09008629EE0FB8A
:20F94000A3E0FAA3E04A4B700301FA669008A5117481F0A374C0F0A374BFF090086091E015
:20F96000FBA3E0FAA3E0F91205F290C003C002C0019008629EA3E0FAA3E0F9D3D082D083AB
:20F98000D0E0E99582EA958340279008A5117481F0A374C0F0A374BFF090086091E0FBA387
:20F9A000E0FAA3E0F91205F290E94A4B600301FA669008945D7481F0A374C0F0A374E4F0F6
:20F9C000A37409F0A37462F0A37480F07B097A62797412008B139008925C7409F0A37462BE
:20F9E000F0A37474F0A37409F0A37462F0A374B2F09008629EE0FBA3E0FAA3E0F91200C923
:20FA0000E4900862BCE0F8A3E0F9A3E0FAA3E0FBC000C001E47F01FEFDFC900862B3E0F99B
:20FA2000F81200840CD001D000EB4FFFEA4EFEE94DFDE84CFC900862BC1200850B7B097A63
:20FA40006279801200D8579008629EE0FBA3E0FAA3E02FF9EA3EFA90086091EBF0A3EAF06C
:20FA6000A3E9F001F90F900862A1E0F9A3E0FAA3E090086091C9F0A3EAF0A3E9F090086258
:20FA8000A1E0F9A3A3E09008629EC9F0A3EAF0A3E9F0900862BCE0FCA3E0FDA3E0FEA3E066
:20FAA000FF900862A4E0FAA3E0900860C375F03C12008528EA75F03CA42583F583759308D2
:20FAC0001200850B900862BCA3A3A3E05404FFE4FEFDFC7B04FAF9F8C3120083E89008622F
:20FAE000A47073E0FAA3E0FB900861BB75F03C12008528EA75F03CA42583F583759308E0D4
:20FB0000FCA3E0FDA3E0FEA3E04402FF900860CB75F03CEB12008528EA75F03CA42583F546
:20FB2000837593081200850B900862A4E0FAA3E0FB900861B775F03C12008528EA75F03CFF
:20FB4000A42583F583759308E0FCA3E0FDA3E0FEA3E044018071E0FAA3E0FB900861BB75BA
:20FB6000F03C12008528EA75F03CA42583F583759308E0FCA3E0FDA3E0FEA3E054FDFF90FB
:20FB80000860CB75F03CEB12008528EA75F03CA42583F5837593081200850B900862A4E068
:20FBA000FAA3E0FB900861B775F03C12008528EA75F03CA42583F583759308E0FCA3E0FD02
:20FBC000A3E0FEA3E054FEFF900860C775F03CEB12008528EA75F03CA42583F58375930867
:20FBE0001200850B9008945D7481F0A374C0F0A374EAF0900862A4E0FFA3E090089460CFE2
:20FC0000F0A3EFF07B097A62798012008B139008A5117409F0A37462F0A37480F0900862C4
:20FC20009EE0FBA3E0FAA3E0F91205F2909008629EEBF0A3EAF0A3E9F090089CAB7409F001
:20FC4000A37462F0A37480F0A37481F0A374BAF0A3740DF0A37409F0A37462F0A374B8F01F
:20FC6000120542FC78B87C627D097B817AC079B612008749EF900862A47020E0FEA3E09046
:20FC80000860CF75F03C12008528EE75F03CA42583F5837593087401F0801DE0FEA3E09077
:20FCA0000860CF75F03C12008528EE75F03CA42583F583759308E4F0900862A5E004F07093
:20FCC00007900862A4E004F001F359E4900862A4F0A3F0900862A4E0FEA3E0FFC39404EE12
:20FCE00064809480400301FDEB900860A975F03CEF12008528EE75F03CA42583F583759395
:20FD000008E0FCA3E0FDA3E0FEA3E0FFE4FBFAF9F8C3120083E8700301FDD8900862A5E0AA
:20FD20002401FE900862A4E03400900862A6F0A3CEF0900862A6E0FEA3E0FFC39404EE6450
:20FD4000809480400301FDD8900860A975F03CEF12008528EE75F03CA42583F583759308A3
:20FD6000E0FCA3E0FDA3E0FEA3E0FF900862A4E0FAA3E0900860A975F03C12008528EA75C9
:20FD8000F03CA42583F583759308E0F8A3E0F9A3E0FAA3E0FBC3120083E870299008A86F8C
:20FDA0007481F0A374C0F0A374F3F0A37481F0A374C0F0A374A6F07B817AC0794312061F78
:20FDC000A3E4FEFF22900862A7E004F07007900862A6E004F001FD32900862A5E004F0700A
:20FDE00007900862A4E004F001FCD3E4900862A4F0A3F0900862A4E0FEA3E0FFC39404EE6E
:20FE000064809480502A7C007D3C1200813874942FF974603EFA7B09E0FD120699BB9008CF
:20FE200062A5E004F070CC900862A4E004F080C312068C4A7E007F01229008A1B3EBF0A37E
:20FE4000EAF0A3E9F09008A5117481F0A374BAF0A374ACF01205F2909008A1BEEBF0A3EAAD
:20FE6000F0A3E9F09008925C7481F0A374BAF0A374B1F0A37409F0A374A1F0A374BAF012A7
:20FE800000C9E4C39008A1BBE09401FF9008A1BAE09400FE120693CBE4FBFAF9F8C3120010
:20FEA00083E87003FEFF229008A1B3E0F9A3E0FAA3E09008A1BEC9F0A3EAF0A3E9F090083F
:20FEC000A5117481F0A374BAF0A37458F09008A1BEE0FBA3E0FAA3E0F91205F2909008A1CA
:20FEE000BEEBF0A3EAF0A3E9F09008A1BEE0FBA3E0FAA3E04A4B60549008925C7481F0A347
:20FF000074BAF0A374B8F0A37409F0A374A1F0A374BCF09008A1BEE0FBA3E0FAA3E0F912AC
:20FF200000C9E4E4FFFEFDFC9008AC681200850B9008A1BCE0FEA3E0FF120686C99008A1F7
:20FF4000BFE475F004120081D801FEBEE49008A1BAF0A3F0A3F0A3F09008A1BCE0FEA3E097
:20FF6000FFC3940AEE64809480400301FFF6120693CB9008A1B61200850BE4FFFEFDFC9091
:20FF800008A1B6E0F8A3E0F9A3E0FAA3E0FBC3120083E8604EE4FFFEFDFC9008AC6812002D
:20FFA000850B9008A1BCE0FEA3E0FF120686C99008A1B6E0FCA3E0FDA3E0FEA3E0FF90080F
:20FFC000AC681200850B9008A1BAE0FEA3E0FF120686C99008A1BBE004F070079008A1BA7F
:20FFE000E004F09008A1BDE004F070079008A1BCE004F001FF5812068C4A7E007F0122229B
:020000040001F9
:20000000E49008B080F0229000FFFD12008645EBF0A3EAF0A3E9F09000FFB8120086459031
:200020000000541200866CE0FEA3E0FF900000541200866CEEF0A3EFF09000004E1200864A
:200040006CE0FBA3E0FAA3E0F912008204FDACF0C3940DEC6480948050032118AA90000021
:200060004B1200866CE0FBA3E0FAA3E0F9C003C002C001C3ED9401FDEC9400FC9000004881
:200080001200866CE0F9A3E0FAA3E09008A42FC9F0A3EAF0A3E9F0900000481200866CE0AA
:2000A000FBA3E0FAA3E02434F9E43AFA12008204C39401FEE5F094009008A432F0A3CEF0C6
:2000C000D001D002D0031205AB63EF4E60032118AA7C007D029000004E1200866CE0FBA3A7
:2000E000E0FAA3E0F91200820425E0FFE5F033FE9000004B1200866CE0FBA3E0FAA3E02F1F
:20010000F9EA3EFAC3E99DF9EA9CFA12008204FFAEF0855083855182759308EEF0A3EFF0AD
:20012000855083855182759308E0FEA3E0FFC39401EE64809480400BD3EF9401EE64809459
:200140008040032118AA85508385518275930874FFF5F0120081D8900000481200866CE0BA
:20016000FBA3E0FAA3E02437F9E43AFA12008204FFAEF0E5F060032118AAEF24FD70032124
:2001800007C2147003210D9114700321151C240360032118AA855083855182759308E0FE6C
:2001A000A3E0FF900889EC75F01412008528EE75F014A42583F583759308E0FD9000004789
:2001C0001200866CEDF0900889EC75F014EF12008528EE75F014A42583F583759308ED548E
:2001E000FEF0900000511200866CE0FBA3E0FAA3E0F91200841F120085FC021600000000F8
:20020000024100000001026C00000002029800000003000002E1855083855182759308E00A
:20022000FEA3E0FF900889D975F01412008528EE75F014A42583F583759308E4F0A3210237
:20024000C2855083855182759308E0FEA3E0FF900889D975F01412008528EE75F014A4255A
:2002600083F583759308E4F0A3048056855083855182759308E0FEA3E0FF900889D975F0A3
:200280001412008528EE75F014A42583F583759308E4F0A37402802A855083855182759301
:2002A00008E0FEA3E0FF900889D975F01412008528EE75F014A42583F583759308E4F0A3F2
:2002C0007403F0900889EC75F014EF12008528EE75F014A42583F583759308E04401F080B3
:2002E0003A900000471200866CE020E0032118A4855083855182759308E0FEA3E0900889E7
:20030000EC75F01412008528EE75F014A42583F583759308E04401F02118A485508385515E
:2003200082759308E0FEA3E0900889EA75F01412008528EE75F014A42583F583759308E06C
:20034000FEA3E064014E60032118B0FE7F07FD7B099000000A1200866CA982AA8312008987
:20036000B17E007F077D007B09900000111200866CA982AA83120089B17B099000000A124E
:2003800000866CA982AA83C001855083855182759308E0FEA3E0FF7C007D141200813874E6
:2003A000E32FF974893EA801FC7D09D0017E007F0712008927EF60488550838551827593E6
:2003C00008E0FEA3E0FF7C007D141200813874E32FF974893EFA7B09C003C002C0017B09DB
:2003E000900000111200866CA982AA83A801AC02AD03D001D002D0037E007F071200805598
:200400007B099000000A1200866CA982AA83C001855083855182759308E0FEA3E0FF7C0005
:200420007D141200813874DC2FF974893EA801FC7D09D0017E007F0712008927EF604885CF
:200440005083855182759308E0FEA3E0FF7C007D141200813874DC2FF974893EFA7B09C038
:2004600003C002C0017B09900000111200866CA982AA83A801AC02AD03D001D002D0037E7A
:20048000007F0712008055855083855182759308E0FEA3E0900889EC75F01412008528EE9B
:2004A00075F014A42583F583759308E054FEF0900000511200866CE0FBA3E0FAA3E0F91202
:2004C00000841F120085FC04E30000000004EA0000000105BD0000000206900000000300B3
:2004E00000078B12062E4F210760855083855182759308E0FEA3E0900889DB75F0141200A5
:200500008528EE75F014A42583F583759308E0FF131313541FFE900000111200866CE5825E
:200520002EF582E43583F583759308E0FEEF5407FF7401A807088002C333D8FC5E60032171
:2005400018A47B099000000A1200866CA982AA83C001855083855182759308E0FEA3E0FF84
:200560007C007D141200813874E32FF974893EA801FC7D09D0017E007F07120080557B097E
:20058000900000111200866CA982AA83C001855083855182759308E0FEA3E0FF7C007D1470
:2005A0001200813874DC2FF974893EA801FC7D09D0017E007F0712008055210760855083F6
:2005C000855182759308E0FEA3E0900889DB75F01412008528EE75F014A42583F5837593EB
:2005E00008E0FF131313541FFE900000111200866CE5822EF582E43583F583759308E0FEB7
:20060000EF5407FF7401A807088002C333D8FC5E60032118A47B09900000111200866CA9A9
:2006200082AA83C001855083855182759308E0FEA3E0FF7C007D141200813874E32FF9745F
:20064000893EA801FC7D09D0017E007F07120080557B099000000A1200866CA982AA83C0B2
:2006600001855083855182759308E0FEA3E0FF7C007D141200813874DC2FF974893EA80125
:20068000FC7D09D0017E007F0712008055210760855083855182759308E0FEA3E090088952
:2006A000DB75F01412008528EE75F014A42583F583759308E0FF131313541FFE90000011C2
:2006C0001200866CE5822EF582E43583F583759308E0FEEF5407FF7401A807088002C3331B
:2006E000D8FC5E60032118A47B09900000111200866CA982AA83C00185508385518275938E
:2007000008E0FEA3E0FF7C007D141200813874DC2FF974893EA801FC7D09D0017E007F07E6
:20072000120080557B09900000111200866CA982AA83C001855083855182759308E0FEA34F
:20074000E0FF7C007D141200813874E32FF974893EA801FC7D09D0017E007F071200805541
:20076000855083855182759308E0FEA3E0900889EC75F01412008528EE75F014A42583F56B
:2007800083759308E04401F0211475900000471200866CE030E02885508385518275930854
:2007A000E0FEA3E0900889EC75F01412008528EE75F014A42583F583759308E04401F02122
:2007C00018A4855083855182759308E0FEA3E0FF900889EC75F01412008528EE75F014A4ED
:2007E0002583F583759308E0FD900000471200866CEDF0900889EC75F014EF12008528EE12
:2008000075F014A42583F583759308ED54FDF0855083855182759308E0FEA3E0900889D942
:2008200075F01412008528EE75F014A42583F583759308E0FEA3E04E70032108F690000074
:20084000511200866CE0FBA3E0FAA3E0F91200841FE47B01FAF9F8D3120083E850619008D6
:200860008AF4E02401FF90088AF3E03400FE90088AC1E02FFF90088AC0E03EFE90088AB707
:20088000E02FFF90088AB6E03EFE90088AFDE02FFF90088AFCE03ECFC39401CF9400FE3332
:2008A00095E0FDFC900000511200866CE0FBA3E0FAA3E0F912008484D3120083E8403790A0
:2008C0000000471200866CE030E128855083855182759308E0FEA3E0900889EC75F01412FB
:2008E000008528EE75F014A42583F583759308E04402F02118A4855083855182759308E07D
:20090000FEA3E0FF900889D975F01412008528EE75F014A42583F583759308E0FCA3E0FD8E
:20092000EC6003210D27ED146033147003210A60147003210B6324036003210D2712062E32
:200940005D855083855182759308E0FEA3E0900889EC75F01412008528EE210D1690000012
:20096000511200866CE0FBA3E0FAA3E0F91200841FC3EF9401FFEE9400FEED9400FDEC94D5
:2009800000FCEF5407FFE404A807088002C333D8FCFFC0071200841FC3EF9401FFEE9400E4
:2009A000FEED9400FDEC9400FC7803120083F9855083855182759308E0FCA3E0FD900889F9
:2009C000DC75F01412008528EC75F014A42583F583E5822FF582E5833EF583759308E0FEC1
:2009E000D0E05E602B900000471200866CE030E11C900889EC75F014ED12008528EC75F0F3
:200A000014A42583F583759308E04402F02118A4900000511200866CE0FBA3E0FAA3E0F942
:200A20001200841FC3EF9401FF855083855182759308E0FCA3E0FD900889DB75F014120018
:200A40008528EC75F014A42583F583759308EFF0900889EC75F014ED12008528EC210D166F
:200A6000900000511200866CE0FBA3E0FAA3E0F91200841FC3EF9401FFEE9400FEED9400C1
:200A8000FDEC9400FCEF5407FFE404A807088002C333D8FCFFC0071200841FC3EF9401FFE8
:200AA000EE9400FEED9400FDEC9400FC7803120083F9855083855182759308E0FCA3E0FD97
:200AC000900889E375F01412008528EC75F014A42583F583E5822FF582E5833EF58375937E
:200AE00008E0FED0E05E602B900000471200866CE030E11C900889EC75F014ED120085285D
:200B0000EC75F014A42583F583759308E04402F02118A4900000511200866CE0FBA3E0FA6C
:200B2000A3E0F91200841FC3EF9401FF855083855182759308E0FCA3E0FD900889DB75F0C1
:200B40001412008528EC75F014A42583F583759308EFF0900889EC75F014ED12008528EC8C
:200B6000210D16900000511200866CE0FBA3E0FAA3E0F91200841FC3EF9401FFEE9400FEFD
:200B8000ED9400FDEC9400FCEF5407FFE404A807088002C333D8FCFFC0071200841FC3EFFA
:200BA0009401FFEE9400FEED9400FDEC9400FC7803120083F9855083855182759308E0FC82
:200BC000A3E0FD900889DC75F01412008528EC75F014A42583F583E5822FF582E5833EF58F
:200BE00083759308E0FED0E05E602B900000471200866CE030E11C900889EC75F014ED127E
:200C0000008528EC75F014A42583F583759308E04402F02118A4900000511200866CE0FB3B
:200C2000A3E0FAA3E0F91200841FC3EF9401FFEE9400FEED9400FDEC9400FCEF5407FFE419
:200C400004A807088002C333D8FCFFC0071200841FC3EF9401FFEE9400FEED9400FDEC944E
:200C600000FC7803120083F9855083855182759308E0FCA3E0FD900889E375F0141200853F
:200C800028EC75F014A42583F583E5822FF582E5833EF583759308E0FED0E05E602B9000C1
:200CA00000471200866CE030E11C900889EC75F014ED12008528EC75F014A42583F583750C
:200CC0009308E04402F02118A4900000511200866CE0FBA3E0FAA3E0F91200841FC3EF94D2
:200CE00001FF855083855182759308E0FCA3E0FD900889DB75F01412008528EC75F014A49B
:200D00002583F583759308EFF0900889EC75F014ED12008528EC75F014A42583F583759361
:200D200008E04402F08037900000471200866CE030E128855083855182759308E0FEA3E0C9
:200D4000900889EC75F01412008528EE75F014A42583F583759308E04402F02118A485504B
:200D600083855182759308E0FEA3E0900889EA75F01412008528EE75F014A42583F5837544
:200D80009308E0FEA3E064014E60032118B0211475855083855182759308E0FEA3E0FF90FE
:200DA0000889EC75F01412008528EE75F014A42583F583759308E0FD900000471200866C8B
:200DC000EDF0900889EC75F014EF12008528EE75F014A42583F583759308ED54FBF08550C6
:200DE00083855182759308E0FEA3E0FF900889D975F01412008528EE75F014A42583F5834B
:200E0000759308E0FCA3E04C6054900889EC75F014EF12008528EE75F014A42583F583758F
:200E20009308E0FF20E137900000471200866CE030E228855083855182759308E0FCA3E0EC
:200E4000900889EC75F01412008528EC75F014A42583F583759308EF4404F02118A47E0092
:200E60007F077D007B09900000181200866CA982AA83120089B1900000541200866CE0FED5
:200E8000A3E0FF900000511200866CE0FBA3E0FAA3E0F9C003C002C0017B09900000181293
:200EA00000866CA982AA83A801AC02AD03D001D002D003120080557B0990000018120086C0
:200EC0006CA982AA837D077C0012055D5EEFF47002EEF47037900000471200866CE030E2D1
:200EE00028855083855182759308E0FEA3E0900889EC75F01412008528EE75F014A42583B1
:200F0000F583759308E04404F02118A47B09900000181200866CA982AA83C003C002C00186
:200F20007B09900000111200866CA982AA839008AA91EBF0A3EAF0A3E9F0D001D002D00313
:200F40001205AC647E007F077D007B099000000A1200866CA982AA83120089B18550838546
:200F60005182759308E0FEA3E0900889D975F01412008528EE75F014A42583F583759308C0
:200F8000E0FEA3E04E60707B099000000A1200866CA982AA83C003C002C0017B09900000FE
:200FA000111200866CA982AA83A801AC02AD03D001D002D0037E007F0712008927EF7037EB
:200FC000900000471200866CE030E228855083855182759308E0FEA3E0900889EC75F01475
:200FE00012008528EE75F014A42583F583759308E04404F02118A485508385518275930842
:20100000E0FEA3E0900889D975F01412008528EE75F014A42583F583759308E0FEA3E0FFA2
:2010200064024E6009EF64034E600321112C855083855182A3A3759308E4F0A3F090000031
:20104000041200866CE4F0A3F0C390088AC9E09401FF90088AC8E09400FE855083855182F3
:20106000A3A3759308E0FCA3E0FDC39FEE6480F8EC6480985069EDAE047803CEA2E713CE1F
:2010800013D8F8FF900000111200866CE5822FF582E5833EF583759308E0FF855083855181
:2010A00082A3A3759308A3E05407FE7401A806088002C333D8FC5F6010900000041200860A
:2010C0006CE475F001120081D8855083855182A3A3759308E475F001120081D8211049902A
:2010E0000000041200866CE0FEA3E0D39404EE648094804037900000471200866CE030E2F2
:2011000028855083855182759308E0FEA3E0900889EC75F01412008528EE75F014A425838E
:20112000F583759308E04404F02118A47E007F07C006C0077F00C0078550838551827593A3
:2011400008E0FEA3E0FF7C007D141200813874DC2FF974893EFA7B09D005D007D00612008A
:2011600089B17E007F07C006C0077F00C007855083855182759308E0FEA3E0FF7C007D1431
:201180001200813874E32FF974893EFA7B09D005D007D006120089B18550838551827593C6
:2011A00008E0FEA3E0FF900889D975F01412008528EE75F014A42583F583759308E0FCA3DB
:2011C000E0FDEC600321140EED14601A14700321127D1470032113142403600321140E1240
:2011E000062E5D2113E4855083855182759308E0FEA3E0900889DB75F01412008528EE758E
:20120000F014A42583F583759308E0FF131313541FFE900000111200866CE5822EF582E4D8
:201220003583F583759308E0FEEF5407FF7401A807088002C333D8FC5E60032118A47B09AD
:20124000900000111200866CA982AA83C001855083855182759308E0FEA3E0FF7C007D14A3
:201260001200813874DC2FF974893EA801FC7D09D0017E007F07120080552113E485508399
:20128000855182759308E0FEA3E0900889DB75F01412008528EE75F014A42583F58375931E
:2012A00008E0FF131313541FFE900000111200866CE5822EF582E43583F583759308E0FEEA
:2012C000EF5407FF7401A807088002C333D8FC5E60032118A47B09900000111200866CA9DD
:2012E00082AA83C001855083855182759308E0FEA3E0FF7C007D141200813874E32FF97493
:20130000893EA801FC7D09D0017E007F07120080552113E4855083855182759308E0FEA3C6
:20132000E0900889DB75F01412008528EE75F014A42583F583759308E0FF131313541FFED5
:20134000900000111200866CE5822EF582E43583F583759308E0FEEF5407FF7401A8070865
:201360008002C333D8FC5E60032118A47B09900000111200866CA982AA83C0018550838564
:201380005182759308E0FEA3E0FF7C007D141200813874DC2FF974893EA801FC7D09D00183
:2013A0007E007F07120080557B09900000111200866CA982AA83C001855083855182759348
:2013C00008E0FEA3E0FF7C007D141200813874E32FF974893EA801FC7D09D0017E007F0713
:2013E00012008055855083855182759308E0FEA3E0900889EC75F01412008528EE75F01439
:20140000A42583F583759308E04404F08037900000471200866CE030E22885508385518284
:20142000759308E0FEA3E0900889EC75F01412008528EE75F014A42583F583759308E04497
:2014400004F02118A4855083855182759308E0FEA3E0900889EA75F01412008528EE75F004
:2014600014A42583F583759308E0FEA3E064014E60032118B0855083855182759308E0FE86
:20148000A3E0FF900889DB75F01412008528EE75F014A42583F583759308E0FDC0057C003D
:2014A0007D141200813874E32FF974893EFA7B09855083855182759308A3E0FF90088D9B96
:2014C0007402F0D00512044EFB855083855182759308E0FEA3E0FF900889DB75F0141200CB
:2014E0008528EE75F014A42583F583759308E0FDC0057C007D141200813874DC2FF9748915
:201500003EFA7B09855083855182759308A3E0FF90088D9B7401F0D00521189A900000511F
:201520001200866CE0FBA3E0FAA3E0F91200841F900000061200866C1200850B900000064C
:201540001200866CE0FCA3E0FDA3E0FEA3E0FF120085FC157500000001166C000000021670
:201560006C00000004166F0000000516FB000000060000166C855083855182759308E0FE3A
:20158000A3E09000001F120652A89000001F1200866CE0FEA3E04E701B90000030120086C2
:2015A0006CE0FEA3E04E7006FE7F032118B312062E4F8012900000321200866CE0540764A2
:2015C0000760032118A4900000301200866CE4F0A304F07B099000001F1200866CA982AA89
:2015E00083C001855083855182759308E0FEA3E0FF7C007D141200813874D92FF974893EFF
:20160000A801FC7D09D0017E007F1412008055855083855182759308A3E0FF9000002112D1
:2016200000866CE0FD7B09900000291200866CA982AA8390088D9B7402F012044EFB8550E8
:2016400083855182759308A3E0FF900000211200866CE0FD7B09900000221200866CA98226
:20166000AA8390088D9B7401F021189A2118A4855083855182759308E0FEA3E09000003384
:20168000120652A8EF4E60032118A47E007F147D007B09900000331200866CA982AA831278
:2016A0000089B1900000351200866C7480F0900000441200866CE4F0A37403F07B09900079
:2016C00000331200866CA982AA83C001855083855182759308E0FEA3E0FF7C007D1412007B
:2016E000813874D92FF974893EA801FC7D09D0017E007F14120080552118B0855083855176
:2017000082759308E0FEA3E0900889EA75F01412008528EE75F014A42583F583759308E078
:20172000FEA3E04E7002802D855083855182759308E0FEA3E0900889EA75F0141200852857
:20174000EE75F014A42583F583759308E0FEA3E064034E7076FE7F14FD7B099000001F127F
:2017600000866CA982AA83120089B1900000211200866C7480F0900000301200866CE4F0A2
:20178000A3F0900000321200866CE4F07B099000001F1200866CA982AA83C00185508385EF
:2017A0005182759308E0FEA3E0FF7C007D141200813874D92FF974893EA801FC7D09D00162
:2017C0007E007F14120080552118B07E007F147D007B099000001F1200866CA982AA8312F9
:2017E0000089B1900000211200866C7480F0900000301200866CE4F0A3F090000032120017
:20180000866CE4F07B099000001F1200866CA982AA83C001855083855182759308E0FEA371
:20182000E0FF7C007D141200813874D92FF974893EA801FC7D09D0017E007F14120080554D
:20184000855083855182759308A3E0FF900000211200866CE0FD7B09900000291200866C73
:20186000A982AA8390088D9B7402F012044EFB855083855182759308A3E0FF900000211286
:2018800000866CE0FD7B09900000221200866CA982AA8390088D9B7401F012044EFB12064B
:2018A0008C4A800C7E007F0380097E007F028003E4FEFF9000005602008645EF640260036F
:2018C000211AFC90086E5AF0A3F090086E57E0FBA3E0FAA3E02415F9E43AFA120080D3B453
:2018E000075390086E57A3E0FAA3E02416F9E43AFA740112008108D394055003212EC39075
:20190000086E57A3E0FAA3E02415F9E43AFAE41200812490088823E0FCA3E0FDA3E0FEA352
:20192000E02401FFE43EFEE43DFDE43CFC900888230200850B90086E57E0FBA3E0FAA3E03C
:201940002415F9E43AFA120080D3B4052090086E57A3E0FAA3E02416F9E43AFA74011200D0
:201960008108D394055003212EC3211AF590086E57E0FBA3E0FAA3E02415F9E43AFA120049
:2019800080D3FF7003212EC320E403211AA190086E57A3E0FAA3E02416F9E43AFA74FF1260
:2019A0000081086003212EC31205C16A90086E57E0FBA3E0FAA3E02417F9E43AFA740112DC
:2019C0000080E96405705990086E57E0FBA3E0FAA3E02415F9E43AFAE4120081249008882F
:2019E00023E0FCA3E0FDA3E0FEA3E02401FFE43EFEE43DFDE43CFC900888231200850B9071
:201A0000086D4A7480F090086D3CE0FBA3E0FAA3E0240DF9E43AFA7414120081242129B785
:201A200090086E57E0FBA3E0FAA3E02415F9E43AFA120080D3540F14700321247224FE609C
:201A4000301470032128F024FE70032128F024FE70032128F024066003212EC390086D3C1A
:201A6000E0FBA3E0FAA3E0240DF9E43AFAE421248590086D4A7404F090088833E0FCA3E032
:201A8000FDA3E0FEA3E02401FFE43EFEE43DFDE43CFC900888331200850B12068BDA212A0A
:201AA000DD90086E57E0FBA3E0FAA3E02415F9E43AFA120080D3540F64036003212EC39093
:201AC000086E57A3E0FAA3E02416F9E43AFA74FF120081086003212EC390086E57A3E0FA91
:201AE000A3E02417F9E43AFA7401120080E964056003212EC31205C16A2119C790088AF5EF
:201B0000E0FBA3E0FAA3E0F990086E5AE0FEA3E0FFE92FF9EA3EFAE41200812490086E5706
:201B20007409F0A3746DF0A37455F090088AF5E0FBA3E0FAA3E0F990086D36EBF0A3EAF0EA
:201B4000A3E9F0240EF9E43AFA90086D42EBF0A3EAF0A3E9F012055684EF64016003211CC6
:201B60008F90088AAAE07003211C681206A6909008ACF8EFF075F008A4248EF582E5F03466
:201B80001CF583759308E09008ACF8F090088AF5E0FBA3E0FAA3E0F990086E54EBF0A3EAE8
:201BA000F0A3E9F02411F9E43AFA1200820445F06003212EC390086E54E0FBA3E0FAA3E0FC
:201BC0002413F9E43AFA120080D36003212EC390086E54E0FBA3E0FAA3E02414F9E43AFA65
:201BE000120080D3705E90086E54A3E0FAA3E0240CF9E43AFA12008204C39403FFE5F094BD
:201C000000FEC3EF9423EE94005003212EC390086E54E0FBA3E0FAA3E02415F9E43AFA12E5
:201C20000080D3FF64806010EF6481600BEF64016006EF6003212EC39008ACF8E0FF12056F
:201C4000372E804B90086E54E0FBA3E0FAA3E02414F9E43AFA120080D3B480339008ACF8CE
:201C6000E0FF12068EDB80271206AE74BF012090088AF5E0FBA3E0FAA3E0F990086E54EB13
:201C8000F0A3EAF0A3E9F07D347C0012061BD090086D36E0FBA3E0FAA3E0240CF9E43AFAD4
:201CA00012008204FFAEF0BE0807BF06040204FC1A9008757DE0FCA3E0FDA3E0FEA3E0242F
:201CC00001FFE43EFEE43DFDE43CFC9008757D1200850B90086D36E0FBA3E0FAA3E0240C38
:201CE000F9E43AFA120082047004E5F0640860219008758DE0FCA3E0FDA3E0FEA3E02401E6
:201D0000FFE43EFEE43DFDE43CFC9008758D211E4E90086D42E0FBA3E0FAA3E02402F9E41E
:201D20003AFA12008204FFAEF090086E5AEEF0A3EFF0D394DCEE9405402190087581E0FCE5
:201D4000A3E0FDA3E0FEA3E02401FFE43EFEE43DFDE43CFC90087581211E4E90086D42E03F
:201D6000FBA3E0FAA3E0F9120080D36445602190087581E0FCA3E0FDA3E0FEA3E02401FFCE
:201D8000E43EFEE43DFDE43CFC90087581211E4EE92406F9E43AFA12008204E5F0543F604A
:201DA00021900875B9E0FCA3E0FDA3E0FEA3E02401FFE43EFEE43DFDE43CFC900875B92177
:201DC0001E4E1206AA0D90086D42E0FBA3E0FAA3E02410F9E43AFA12008484C3120083E807
:201DE000604290086D42E0FBA3E0FAA3E02410F9E43AFA1200841F74FFFBFAF9F8C31200F7
:201E000083E8602090087585E0FCA3E0FDA3E0FEA3E02401FFE43EFEE43DFDE43CFC9008CF
:201E20007585802A12054004EFF47002EEF4602590087581E0FCA3E0FDA3E0FEA3E02401D4
:201E4000FFE43EFEE43DFDE43CFC900875811200850B21262D90086D42E0FBA3E0FAA3E063
:201E6000240CF9E43AFA1200841F90086D36E0FBA3E0FAA3E02406F9E43AFA12046E6590A2
:201E8000087595E0FCA3E0FDA3E0FEA3E02401FFE43EFEE43DFDE43CFC9008759512008519
:201EA0000B90086D42E0FBA3E0FAA3E02409F9E43AFA120080D3B40149120080D3FF900858
:201EC0006E57E0FBA3E0FAA3E02414F9E43AFAEF1200812490086D42E0FBA3E0FAA3E0242D
:201EE0000CF9E43AFA1200841F90086E57E0FBA3E0FAA3E02404F9E43AFA1200843C0206C5
:201F0000417290086D42E0FBA3E0FAA3E02409F9E43AFA120080D36411600321202E90086A
:201F20009620E0FCA3E0FDA3E0FEA3E02401FFE43EFEE43DFDE43CFC900896201200850B1D
:201F400090086D42E0FBA3E0FAA3E02414F9E43AFA90086D3FEBF0A3EAF0A3E9F090088ADC
:201F6000F5E0FBA3E0FAA3E0F912064FC290086D42E0FBA3E0FAA3E02409F9E43AFA1200FD
:201F800080D3FF90086E57E0FBA3E0FAA3E02414F9E43AFAEF1200812490086D3FE0FBA306
:201FA000E0FAA3E02402F9E43AFA12008204FF90086E57E0FBA3E0FAA3E0F9E5F08FF0125F
:201FC00000827E90086D3FE0FBA3E0FAA3E0F912008204FF90086E57E0FBA3E0FAA3E024F6
:201FE00002F9E43AFAE5F08FF01200827E90086D42E0FBA3E0FAA3E0240CF9E43AFA1200F3
:20200000841F90086E57E0FBA3E0FAA3E02404F9E43AFA1200843C90086E57E0FBA3E0FA25
:20202000A3E0F912008204FFAEF00205EA3390086D42E0FBA3E0FAA3E02409F9E43AFA1259
:202040000080D364066043E4FFFEFDFC90087595E0F8A3E0F9A3E0FAA3E0FBD3120083E805
:20206000402590087595E0FCA3E0FDA3E0FEA3E024FFFFEE34FFFEED34FFFDEC34FFFC90F0
:202080000875951200850B21262D90086D42E0FBA3E0FAA3E02414F9E43AFA90086D3CEB81
:2020A000F0A3EAF0A3E9F09008882BE0FCA3E0FDA3E0FEA3E02401FFE43EFEE43DFDE43C0A
:2020C000FC9008882B1200850B1206AD1E90086D3CE0FBA3E0FAA3E02402F9E43AFA1200CF
:2020E00082046F7003EE65F0600321262D9008ACF6E4F0A304F09008ACF6E0FEA3E0FFC35C
:202100009405EE940040032121D47C007D331200813874552FF9746D3EFA7B0990086E5769
:20212000EBF0A3EAF0A3E9F02415F9E43AFA120080D370032121C190086D3CE0FBA3E0FA0D
:20214000A3E02402F9E43AFA12008204FFAEF090086E57E0FBA3E0FAA3E0F9120082046F58
:202160007003EE65F0705AE92402F9E43AFA12008204FFAEF090086D3CE0FBA3E0FAA3E06E
:20218000F912008204B50739E5F0B5063490086E57E0FBA3E0FAA3E02404F9E43AFA120072
:2021A000841F90086D42E0FBA3E0FAA3E0240CF9E43AFA12008484C3120083E87003212506
:2021C000889008ACF7E004F070079008ACF6E004F02120F690086D3CE0FBA3E0FAA3E0246C
:2021E0000DF9E43AFA120080D36402600321262D9008ACF6E4F0A304F09008ACF6E0FEA3BF
:20220000E0FFC39405EE9400502D90086D6A75F033EF12008528EE75F033A42583F5837510
:202220009308E0605E9008ACF7E004F070CB9008ACF6E004F080C29008ACF6E4F0A304F026
:202240009008ACF6E0FEA3E0FFC39405EE9400502F90086D6A75F033EF12008528EE75F07F
:2022600033A42583F583759308E0640760159008ACF7E004F070C99008ACF6E004F080C001
:2022800021262D9008ACF6E0FEA3E0FF7C007D331200813874552FF9746D3EFA90086E57D2
:2022A0007409F0A3EAF0A3E9F090086D42E0FBA3E0FAA3E02409F9E43AFA120080D3FF9064
:2022C000086E57E0FBA3E0FAA3E02414F9E43AFAEF1200812490086E57E0FBA3E0FAA3E02F
:2022E0002416F9E43AFA74021200812490086E57E0FBA3E0FAA3E02417F9E43AFAE41200EC
:20230000812490086D3CE0FBA3E0FAA3E02402F9E43AFA12008204FF90086E57E0FBA3E073
:20232000FAA3E0F9E5F08FF01200827E90086D3CE0FBA3E0FAA3E0F912008204FF90086E0F
:2023400057E0FBA3E0FAA3E02402F9E43AFAE5F08FF01200827E90086D42E0FBA3E0FAA36C
:20236000E0240CF9E43AFA1200841F90086E57E0FBA3E0FAA3E02404F9E43AFA1200843C44
:2023800090086E57E0FBA3E0FAA3E02415F9E43AFA7411120081249008881BE0FCA3E0FDE8
:2023A000A3E0FEA3E02401FFE43EFEE43DFDE43CFC9008881B1200850B90086D51E0FCA3E9
:2023C000E0FDA3E0FEA3E0FF90086E57E0FBA3E0FAA3E0240CF9E43AFA1200843CEF2401BE
:2023E000FFE43EFEE43DFDE43CFC90086E57E0FBA3E0FAA3E02410F9E43AFA1200843C90A5
:20240000086D3CE0FBA3E0FAA3E02404F9E43AFA1200841FEF2401FFE43EFEE43DFDE43CD1
:20242000FC90086E57E0FBA3E0FAA3E02408F9E43AFA1200843C90086E57E0FBA3E0FAA301
:20244000E0242AF9E43AFAC003C002C00190086E57A3E0FAA3E02428F9E43AFA9008AC4BAE
:20246000EBF0A3EAF0A3E9F0D001D002D0031206730790086D3CE0FBA3E0FAA3E0240DF93A
:20248000E43AFA74101200812490086D3CE0FBA3E0FAA3E0240DF9E43AFA120080D34402E0
:2024A0001200812490086D3CE0FBA3E0FAA3E02414F9E43AFA9008ACF9EBF0A3EAF0A3E9DF
:2024C000F07402120081249008ACF9E0FBA3E0FAA3E02401F9E43AFA7404120081249008CA
:2024E000ACF9E0FBA3E0FAA3E02402F9E43AFA7405120081249008ACF9E0FBA3E0FAA3E0DD
:202500002403F9E43AFA7478120081249008ACF9E0FBA3E0FAA3E02404F9E43AFA74011208
:202520000081249008ACF9E0FBA3E0FAA3E02405F9E43AFA7401120081249008ACF9E0FB60
:20254000A3E0FAA3E02406F9E43AFA7404120081249008ACF9E0FBA3E0FAA3E02407F9E4F1
:202560003AFA74021200812490086E5AE4F0A37430F090086D3CE0FBA3E0FAA3E0240CF94A
:20258000E43AFA7470212D8CE490086D4AF090086D3CE0FBA3E0FAA3E0240DF9E43AFA12D2
:2025A0000080D330E26F90086E57E0FBA3E0FAA3E02415F9E43AFA120080D3B401229008F1
:2025C000881FE0FCA3E0FDA3E0FEA3E02401FFE43EFEE43DFDE43CFC9008881F1200850B95
:2025E000E41200812490088823E0FCA3E0FDA3E0FEA3E02401FFE43EFEE43DFDE43CFC908F
:202600000888231200850B90086D4A7420F012068BDA212C4E90086D3CE0FBA3E0FAA3E05E
:20262000240DF9E43AFA120080D320E403212C4E90086D3CE0FBA3E0FAA3E0240CF9E43AEE
:20264000FA120080D3C4540F25E025E0FF7E009008ACF6EEF0A3EFF02414FFEE33FEC3902A
:20266000086E5BE09FFF90086E5AE09EFEF0A3EFF0D39400EE9400403490086E57E0FBA385
:20268000E0FAA3E02408F9E43AFA1200841F90086D3CE0FBA3E0FAA3E02404F9E43AFA1284
:2026A000008484C3120083E86003212D5890086E57E0FBA3E0FAA3E02410F9E43AFA12003A
:2026C000841F90086D3CE0FBA3E0FAA3E02408F9E43AFA12008484C3120083E87066900836
:2026E0006E57E0FBA3E0FAA3E02410F9E43AFA1200841F90086E57A3E0FAA3E0240CF9E4D6
:202700003AFA1200843C90086E57E0FBA3E0FAA3E02415F9E43AFA120080D3FF30E4259004
:20272000086D4A7401F0EF54EF1200812490086E57E0FBA3E0FAA3E02416F9E43AFA740293
:202740001200812490086E57E0FBA3E0FAA3E02415F9E43AFA120080D3540F14B408004068
:2027600003212D549001277375F004A4C58325F0C5837302012793020127AF02012832026F
:20278000012B6902012C5102012D1F02012D5802012B2390086D4AE030E0117403120081A2
:2027A0002490086D4A7440F012068BDA212C4E90086D4AE030E07890086D3CE0FBA3E0FA9A
:2027C000A3E0240DF9E43AFA120080D36412705F90086E57E0FBA3E0FAA3E02415F9E43A02
:2027E000FA74031200812490086D3CE0FBA3E0FAA3E02404F9E43AFA1200841F90086E574A
:20280000E0FBA3E0FAA3E02408F9E43AFA1200843C1200841FEF2401FFE43EFEE43DFDE4E4
:202820003CFC1200843C744212068BCD212960212C4E90088827E0FCA3E0FDA3E0FEA3E07C
:202840002401FFE43EFEE43DFDE43CFC900888271200850B90086D3CE0FBA3E0FAA3E024D1
:202860000DF9E43AFA120080D320E0032128F390086E5BE02401FF90086E5AE03400FEE4DB
:20288000FCFD90086E57E0FBA3E0FAA3E02408F9E43AFA1200843C741012068BCD90086EFE
:2028A00057E0FBA3E0FAA3E02410F9E43AFA1200841FEF2401FFE43EFEE43DFDE43CFC126D
:2028C00000843C90086E57E0FBA3E0FAA3E02415F9E43AFA74181200812490086E57E0FB3B
:2028E000A3E0FAA3E02417F9E43AFAE412008124212A37D390086E5BE0940090086E5AE087
:202900009400404590086D4AE04402F090086E57E0FBA3E0FAA3E02408F9E43AFAC003C041
:2029200002C0011200848490086E5AE0FEA3E0FFE4FCFDEB2FFFEA3EFEED39FDEC38FCD0CB
:2029400001D002D0031200843C90086D4AE054037003212B2012068BDAEF4E7003212D58C7
:2029600090086D4AE030E57490086E57E0FBA3E0FAA3E02415F9E43AFAE4120081249008EA
:202980006D3CE0FBA3E0FAA3E0240DF9E43AFA74141200812490088823E0FCA3E0FDA3E010
:2029A000FEA3E02401FFE43EFEE43DFDE43CFC900888231200850B9008883BE0FCA3E0FD7C
:2029C000A3E0FEA3E02401FFE43EFEE43DFDE43CFC9008883B1200850B212D6F90086D4A6C
:2029E000E030E46990086E57E0FBA3E0FAA3E02410F9E43AFA1200841FEF2401FFE43EFE15
:202A0000E43DFDE43CFC1200843C90086E57E0FBA3E0FAA3E02415F9E43AFA74141200810D
:202A20002490086E57E0FBA3E0FAA3E02417F9E43AFAE41200812490086D3CE0FBA3E0FABA
:202A4000A3E0240DF9E43AFA7411212D6BD390086E5BE0940090086E5AE0940040779008A8
:202A60006E57E0FBA3E0FAA3E02415F9E43AFA120080D320E45F120080D344101200812434
:202A800090086E57E0FBA3E0FAA3E02417F9E43AFAE41200812490086E57E0FBA3E0FAA3BF
:202AA000E02410F9E43AFAC003C002C0011200848490086E5AE0FEA3E0FFE4FCFDEB2FFFDB
:202AC000EA3EFEED39FDEC38FCD001D002D0031200843C8008E490086E5AF0A3F0D390088B
:202AE0006E5BE0940090086E5AE09400500890086D4AE030E12A90086E5BE02428F09008EE
:202B00006E5AE03400F090086D3CE0FBA3E0FAA3E0240DF9E43AFA741812008124212D7981
:202B2000212C4E90086D4AE020E003212D5490086E57E0FBA3E0FAA3E02415F9E43AFAE4C0
:202B40001200812490088823E0FCA3E0FDA3E0FEA3E02401FFE43EFEE43DFDE43CFC900805
:202B600088231200850B212D54D390086E5BE0940090086E5AE09400403D90086E57E0FB35
:202B8000A3E0FAA3E02408F9E43AFAC003C002C0011200848490086E5AE0FEA3E0FFE4FCF8
:202BA000FDEB2FFFEA3EFEED39FDEC38FCD001D002D0031200843C90086D3CE0FBA3E0FAB5
:202BC000A3E0240DF9E43AFA120080D330E04990086D4AE090086E5730E027E0FBA3E0FA57
:202BE000A3E02415F9E43AFA74071200812490086E57E0FBA3E0FAA3E02416F9E43AFAE46F
:202C0000800FE0FBA3E0FAA3E02415F9E43AFA741612008124212CE490086D4AE030E01A35
:202C200090086E57E0FBA3E0FAA3E02415F9E43AFA740512008124212D54D390086E5BE02C
:202C4000940090086E5AE094004003212D58212D54D390086E5BE0940090086E5AE0940005
:202C6000403D90086E57E0FBA3E0FAA3E02408F9E43AFAC003C002C0011200848490086EFC
:202C80005AE0FEA3E0FFE4FCFDEB2FFFEA3EFEED39FDEC38FCD001D002D0031200843C9043
:202CA000086D3CE0FBA3E0FAA3E0240DF9E43AFA120080D330E05590086E57E0FBA3E0FAC7
:202CC000A3E02415F9E43AFA74071200812490086E57E0FBA3E0FAA3E02416F9E43AFAE48E
:202CE0001200812490086E57E0FBA3E0FAA3E02408F9E43AFA1200841FEF2401FFE43EFEC0
:202D0000E43DFDE43CFC1200843C804CD390086E5BE0940090086E5AE09400503B8035908F
:202D2000086D4AE030E02D90086E57E0FBA3E0FAA3E02415F9E43AFA74071200812490086B
:202D40006E57E0FBA3E0FAA3E02416F9E43AFAE4120081240206B07690086D3CE0FBA3E020
:202D6000FAA3E0240DF9E43AFA74101200812490086E5AE4F0A37428F090086D3CE0FBA337
:202D8000E0FAA3E0240CF9E43AFA74501200812490086E57E0FBA3E0FAA3E02408F9E43A9F
:202DA000FA1200841F90086D3CE0FBA3E0FAA3E02408F9E43AFA1200843C90086E57E0FB01
:202DC000A3E0FAA3E0240CF9E43AFA1200841F90086D3CE0FBA3E0FAA3E02404F9E43AFAA8
:202DE0001200843C90086E57E0FBA3E0FAA3E0F912008204FF90086D3CE0FBA3E0FAA3E01D
:202E0000F9E5F08FF01200827E90086E57E0FBA3E0FAA3E02402F9E43AFA12008204FF90BD
:202E2000086D3CE0FBA3E0FAA3E02402F9E43AFAE5F08FF01200827E90086D3CE0FBA3E0CA
:202E4000FAA3E0240EF9E43AFA740575F0781200827E9008882FE0FCA3E0FDA3E0FEA3E09B
:202E60002401FFE43EFEE43DFDE43CFC9008882F1200850B9008882FE0FCA3E0FDA3E0FEB7
:202E8000A3E0FFA3E0F8A3E0F9A3E0FAA3E0FBC3EF9BFFEE9AFEED99FDEC98FC9008882F9A
:202EA0001200850B7F027E001203000790086E57E0FBA3E0FAA3E02416F9E43AFA7402124A
:202EC000008124229000FFFD12008645EBF0A3EAF0A3E9F09000FF9D120086451206ADA67A
:202EE000EF64014E7006FE7F02214261900000691200866CE0FBA3E0FAA3E0F9120082040E
:202F0000FDACF0C3940DEC648094805003214258900000661200866CE0FBA3E0FAA3E0F9F4
:202F2000C003C002C001C3ED9401FDEC9400FC900000631200866CE0F9A3E0FAA3E0900825
:202F4000A42FC9F0A3EAF0A3E9F0900000631200866CE0FBA3E0FAA3E02434F9E43AFA129F
:202F6000008204C39401FEE5F094009008A432F0A3CEF0D001D002D0031205AB63EF4E6015
:202F8000032142587C007D02900000691200866CE0FBA3E0FAA3E0F91200820425E0FFE526
:202FA000F033FE900000661200866CE0FBA3E0FAA3E02FF9EA3EFAC3E99DF9EA9CFA1200FD
:202FC0008204FFAEF0855083855182759308EEF0A3EFF0855083855182759308E0FEA3E08D
:202FE000FFC39401EE94004009D3EF94FEEE940F40032142587E007F077D007B0990000037
:20300000271200866CA982AA83120089B1900000631200866CE0FBA3E0FAA3E02437F9E4D7
:203020003AFA12008204FFAEF0E5F07013EF24FD6011147003213696147003213C96240339
:20304000214258900000041200866CE0FEA3E0FF90084C6875F01312008528EE75F013A430
:203060002583F583759308E0FD900000621200866CEDF090084C6875F013EF12008528EE10
:2030800075F013A42583F583759308ED54FDF09000006F1200866CE0FEA3E0D39407EE6492
:2030A0008094804039900000621200866CE020E103214252900000041200866CE0FEA3E07B
:2030C00090084C6875F01312008528EE75F013A42583F583759308E04402F02142527E00EA
:2030E0007F077D007B09900000201200866CA982AA83120089B19000006F1200866CE0FE10
:20310000A3E0FF9000006C1200866CE0FBA3E0FAA3E0F9C003C002C0017B099000002012CD
:2031200000866CA982AA83A801AC02AD03D001D002D003120080557B099000002012008615
:203140006CA982AA837D077C0012055D5EEFF47002EEF47036900000621200866CE030E115
:2031600027900000041200866CE0FEA3E090084C6875F01312008528EE75F013A42583F505
:2031800083759308E04402F0214252855083855182759308E0FEA3E0FF7B09900000041287
:2031A00000866CA982AA83C003C002C0017B099000004F1200866CA982AA839008AA9BEBF8
:2031C000F0A3EAF0A3E9F0D001D002D00312064280EF4E7036900000621200866CE030E1EC
:2031E00027900000041200866CE0FEA3E090084C6875F01312008528EE75F013A42583F585
:2032000083759308E04402F02142527B09900000201200866CA982AA83C003C002C0017BFF
:2032200009900000351200866CA982AA839008AA91EBF0A3EAF0A3E9F0D001D002D0031235
:2032400005AC64855083855182A3A3759308E4F0A3F0C390088AC9E09401FF90088AC8E000
:203260009400FE855083855182A3A3759308E0FCA3E0FDC39FEE6480F8EC64809840032162
:20328000336BEDAE047803CEA2E713CE13D8F8FF900000351200866CE5822FF582E5833EE0
:2032A000F583759308E0FF855083855182A3A3759308A3E05407FE7401A806088002C33322
:2032C000D8FCFD5F6003213355855083855182A3A3759308E0FEA3E07803CEA2E713CE1385
:2032E000D8F8FF900000581200866CE5822FF582E5833EF583759308E0FC5D60588550838F
:20330000855182A3A3759308E0FEA3E07803CEA2E713CE13D8F8FF900000581200866CE538
:20332000822FF582E5833EF583C083C082759308855083855182A3A3759308A3E05407FFCF
:203340007401A807088002C333D8FCF45C759308D082D083F0855083855182A3A3759308FA
:20336000E475F001120081D8213252855083855182A3A3759308E4F0A3F0C390088AC9E0F8
:203380009401FF90088AC8E09400FE855083855182A3A3759308E0FCA3E0FDC39FEE6480A7
:2033A000F8EC648098400321346DEDAE047803CEA2E713CE13D8F8FF900000581200866C88
:2033C000E5822FF582E5833EF583759308E0FF855083855182A3A3759308A3E05407FE747D
:2033E00001A806088002C333D8FCFD5F6069855083855182A3A3759308E0FEA3E07803CEF5
:20340000A2E713CE13D8F8FF900000351200866CE5822FF582E5833EF583759308E05D70AF
:2034200036900000621200866CE030E127900000041200866CE0FEA3E090084C6875F0138B
:2034400012008528EE75F013A42583F583759308E04402F0214252855083855182A3A3753D
:203460009308E475F001120081D821337A9000004F1200866CE0FEA3E0FF9000000E12003B
:20348000866CEEF0A3EFF07B09900000351200866CA982AA83C003C002C0017B09900000DB
:2034A000101200866CA982AA83A801AC02AD03D001D002D0037E007F07120080557B099024
:2034C0000000581200866CA982AA83C003C002C0017B09900000171200866CA982AA83A8C3
:2034E00001AC02AD03D001D002D0037E007F0712008055855083855182A3A3759308E4F032
:20350000A3F0C390088AC9E09401FD90088AC8E09400FC855083855182A3A3759308E0FEBA
:20352000A3E0FFC39DEC6480F8EE64809840032136047B099000001E1200866CA982AA834B
:2035400012068C879000000E1200866CE0FEA3E0FF9000001E1200866CE0540FFCA3E06F5B
:203560007002EE6C60032135EE855083855182A3A3759308E0FEA3E07803CEA2E713CE13AB
:20358000D8F8FF900000101200866CE5822FF582E5833EF583759308E0FF855083855182EE
:2035A000A3A3759308A3E05407FE7401A806088002C333D8FC5F7036900000621200866C67
:2035C000E030E127900000041200866CE0FEA3E090084C6875F01312008528EE75F013A44D
:2035E0002583F583759308E04402F0214252855083855182A3A3759308E475F001120081ED
:20360000D82135027B099000000E1200866CA982AA83C003C002C001900000041200866C1E
:20362000E0FEA3E0FF7C007D131200813874562FF9744C3EA801FC7D09D001D002D0037E44
:20364000007F1012008055900000041200866CE0FEA3E0FF90084C6875F01312008528EE8B
:2036600075F013A42583F583759308E04402F090084C6675F013EF12008528EE75F013A46E
:203680002583F583759308E0FEA3E064014E600321425E213C6C900000041200866CE0FE83
:2036A000A3E0FF90084C6875F01312008528EE75F013A42583F583759308E0FD90000062FC
:2036C0001200866CEDF090084C6875F013EF12008528EE75F013A42583F583759308ED541C
:2036E000FBF09000006F1200866CE0FEA3E0D39407EE648094804036900000621200866CBB
:20370000E030E227900000041200866CE0FEA3E090084C6875F01312008528EE75F013A40A
:203720002583F583759308E04404F02142527E007F077D007B09900000201200866CA982A8
:20374000AA83120089B19000006F1200866CE0FEA3E0FF9000006C1200866CE0FBA3E0FA35
:20376000A3E0F9C003C002C0017B09900000201200866CA982AA83A801AC02AD03D001D04F
:2037800002D003120080557B09900000201200866CA982AA837D077C0012055D5EEFF470B8
:2037A00002EEF47036900000621200866CE030E227900000041200866CE0FEA3E090084C93
:2037C0006875F01312008528EE75F013A42583F583759308E04404F0214252855083855115
:2037E00082759308E0FEA3E0FF7B09900000041200866CA982AA83C003C002C0017B099009
:2038000000004F1200866CA982AA839008AA9BEBF0A3EAF0A3E9F0D001D002D0031206427C
:2038200080EF4E7036900000621200866CE030E227900000041200866CE0FEA3E090084C39
:203840006875F01312008528EE75F013A42583F583759308E04404F02142527B09900000AE
:20386000201200866CA982AA83C003C002C0017B099000002E1200866CA982AA839008AAA6
:2038800091EBF0A3EAF0A3E9F0D001D002D0031205AC64855083855182A3A3759308E4F04C
:2038A000A3F0C390088AC9E09401FF90088AC8E09400FE855083855182A3A3759308E0FC15
:2038C000A3E0FDC39FEE6480F8EC6480985075EDAE047803CEA2E713CE13D8F8FF9000004B
:2038E0002E1200866CE5822FF582E5833EF583759308E0FD855083855182A3A3759308A3D5
:20390000E05407FC7401A804088002C333D8FCFC5D601B900000511200866CE5822FF58235
:20392000E5833EF583759308E04C759308F0855083855182A3A3759308E475F0011200814A
:20394000D82138A2855083855182A3A3759308E4F0A3F0C390088AC9E09401FF90088AC81B
:20396000E09400FE855083855182A3A3759308E0FCA3E0FDC39FEE6480F8EC64809840039C
:20398000213A46EDAE047803CEA2E713CE13D8F8FF9000002E1200866CE5822FF582E5831B
:2039A0003EF583759308E0FF855083855182A3A3759308A3E05407FE7401A806088002C310
:2039C00033D8FCFD5F6069855083855182A3A3759308E0FEA3E07803CEA2E713CE13D8F8BE
:2039E000FF900000511200866CE5822FF582E5833EF583759308E05D7036900000621200C1
:203A0000866CE030E227900000041200866CE0FEA3E090084C6875F01312008528EE75F0CC
:203A200013A42583F583759308E04404F0214252855083855182A3A3759308E475F0011270
:203A40000081D82139539000004F1200866CE0FEA3E0FF9000000E1200866CEEF0A3EFF01B
:203A60007B09900000511200866CA982AA83C003C002C0017B09900000101200866CA982EC
:203A8000AA83A801AC02AD03D001D002D0037E007F07120080557B099000002E1200866C4B
:203AA000A982AA83C003C002C0017B09900000171200866CA982AA83A801AC02AD03D00109
:203AC000D002D0037E007F0712008055855083855182A3A3759308E4F0A3F0C390088AC93B
:203AE000E09401FD90088AC8E09400FC855083855182A3A3759308E0FEA3E0FFC39DEC64E4
:203B000080F8EE6480984003213BDD7B099000001E1200866CA982AA8312068C87900000FE
:203B20000E1200866CE0FEA3E0FF9000001E1200866CE0540FFCA3E06F7002EE6C600321E0
:203B40003BC7855083855182A3A3759308E0FEA3E07803CEA2E713CE13D8F8FF90000010C7
:203B60001200866CE5822FF582E5833EF583759308E0FF855083855182A3A3759308A3E09E
:203B80005407FE7401A806088002C333D8FC5F7036900000621200866CE030E227900000B1
:203BA000041200866CE0FEA3E090084C6875F01312008528EE75F013A42583F583759308DF
:203BC000E04404F0214252855083855182A3A3759308E475F001120081D8213ADB7B099013
:203BE00000000E1200866CA982AA83C003C002C001900000041200866CE0FEA3E0FF7C00A1
:203C00007D131200813874562FF9744C3EA801FC7D09D001D002D0037E007F1012008055C4
:203C2000900000041200866CE0FEA3E0FF90084C6875F01312008528EE75F013A42583F562
:203C400083759308E04404F090084C6675F013EF12008528EE75F013A42583F5837593080F
:203C6000E0FEA3E064014E600321425E900000041200866CE0FEA3E0FF7C007D1312008175
:203C80003874562FF9744C3EFA7B09900000041200866C213E879000006C1200866CE0FB25
:203CA000A3E0FAA3E0F91200841F120085FC3CD0000000013E93000000023E96000000040B
:203CC0003E99000000053FD80000000600004252855083855182759308E0FEA3E0FF7B09B3
:203CE000900000041200866CA982AA83C003C002C0017B099000003C1200866CA982AA83E2
:203D00009008AA9BEBF0A3EAF0A3E9F0D001D002D00312064280EF4E7003214039900000C8
:203D20004E1200866CE0540764066003214252855083855182A3A3759308E4F0A3F0855032
:203D400083855182A3A3759308E0FEA3E0FFC39440EE64809480504F7B099000000E120082
:203D6000866CA982AA8312066287EF4E60399000000E1200866CE0FEA3E0FF8550838551F2
:203D800082759308E0FCA3E0B50707ECB5060321415C855083855182A3A3759308E475F0B8
:203DA00001120081D88097855083855182A3A3759308E0FAA3E0FBC39440EA648094804069
:203DC000032142527C007D13AF03AE021200813874562FF9744C3EFA7B09C003C002C0013E
:203DE000900000041200866CE0FEA3E0FF7C007D131200813874562FF9744C3EA801FC7DE2
:203E000009D001D002D0037E007F13120080559000004C1200866CE4F0A304F07B099000CD
:203E2000003C1200866CA982AA83C001855083855182A3A3759308E0FEA3E0FF7C007D13B7
:203E40001200813874562FF9744C3EA801FC7D09D0017E007F131200805585508385518204
:203E6000A3A3759308E0FEA3E0FF7C007D131200813874562FF9744C3EFA7B09855083856A
:203E80005182A3A3759308E0FEA3E0FF1206AC7221424C214252214252855083855182A3F7
:203EA000A3759308E4F0A3F0855083855182A3A3759308E0FEA3E0FFC39440EE6480948005
:203EC000502B7B099000004F1200866CA982AA83120656F1EF4E6015855083855182A3A3A1
:203EE000759308E475F001120081D880BB855083855182A3A3759308E0FEA3E0FF4E700E90
:203F0000900000041200866CE4F0A3F08043C3EF9401FFEE9400FE900000041200866CE0A1
:203F2000FCA3E0D39FEE6480F8EC648098401F855083855182A3A3759308E0FEA3E0FF9009
:203F40000000041200866CEEF0A3EFF080032142527E007F137D007B099000004F12008639
:203F60006CA982AA83120089B1855083855182759308E0FEA3E0FF9000004F1200866CEE40
:203F8000F0A3EFF09000005F1200866CE4F0A37403F07B099000004F1200866CA982AA831F
:203FA000C003C002C001900000041200866CE0FEA3E0FF7C007D131200813874562FF97486
:203FC0004C3EA801FC7D09D001D002D0037E007F131200805521425E855083855182759346
:203FE00008E0FEA3E0FF7B09900000041200866CA982AA83C003C002C0017B099000003C4F
:204000001200866CA982AA839008AA9BEBF0A3EAF0A3E9F0D001D002D00312064280EF4E06
:204020007005FEFF214261855083855182759308E0FEA3E064014E7006FE7F03214261902C
:204040000000041200866CE0FEA3E0FF90084C6675F01312008528EE75F013A42583F5834D
:20406000759308E0FCA3E064034C702AF583758213C083C082FDC005FC7D131200813874F0
:20408000562FF9744C3EFA7B09D005D007D006120089B121425E7E007F087D007B09900001
:2040A00000061200866CA982AA83120089B1855083855182A3A3759308E4F0A3F08550838D
:2040C000855182A3A3759308E0FEA3E0FFC39440EE64809480506C7B099000000E120086DF
:2040E0006CA982AA8312066287EF4E60409000000E1200866CE0FEA3E0FF8550838551826C
:20410000759308E0FCA3E0B50723ECB5061F855083855182A3A3759308E0FEA3E0FF900095
:2041200000041200866CEEF0A3EFF08016855083855182A3A3759308E475F001120081D8C6
:204140002140BD855083855182A3A3759308E0FEA3E0C39440EE64809480400321425E85D4
:204160005083855182A3A3759308E4F0A3F0C390088AC9E09401FD90088AC8E09400FC8558
:204180005083855182A3A3759308E0FEA3E0FFC39DEC6480F8EE648098504C7B09900000FC
:2041A0001E1200866CA982AA8312068C879000000E1200866CE0FEA3E0FF9000001E120098
:2041C000866CE0540FFCA3E0B50707EEB50403214252855083855182A3A3759308E475F0BA
:2041E00001120081D88087900000041200866CE0FEA3E07803CEA2E713CE13D8F8FF90002E
:2042000000061200866CE5822FF582E5833EF583C083C082759308E0FF90000004120086C9
:204220006CA3E05407FE7401A806088002C333D8FC4F759308D082D083F07B0990000006B1
:204240001200866CA982AA8312056BF912068C4A800C7E007F0380097E007F028003E4FE20
:20426000FF90000071020086459000FFFD12008645EBF0A3EAF0A3E9F09000FFB612008657
:2042800045900000561200866CE0FEA3E0FF900000561200866CEEF0A3EFF0900000501253
:2042A00000866CE0FBA3E0FAA3E0F912008204FDACF0C3940DEC6480948050032153B990AF
:2042C00000004D1200866CE0FBA3E0FAA3E0F9C003C002C001C3ED9401FDEC9400FC900025
:2042E000004A1200866CE0F9A3E0FAA3E09008A42FC9F0A3EAF0A3E9F09000004A12008608
:204300006CE0FBA3E0FAA3E02434F9E43AFA12008204C39401FEE5F094009008A432F0A395
:20432000CEF0D001D002D0031205AB63EF4E60032153B97C007D02900000501200866CE098
:20434000FBA3E0FAA3E0F91200820425E0FFE5F033FE9000004D1200866CE0FBA3E0FAA3EB
:20436000E02FF9EA3EFAC3E99DF9EA9CFA12008204FFAEF0855083855182759308EEF0A3DB
:20438000EFF0855083855182759308E0FEA3E0FFC39401EE64809480400BD3EF9404EE64E9
:2043A00080948040032153B985508385518275930874FFF5F0120081D89000004A12008604
:2043C0006CE0FBA3E0FAA3E02437F9E43AFA12008204FFAEF0E5F060032153B9EF24FEB4CB
:2043E0000D0040032153B9900143F675F004A4C58325F0C583730201442A0201458E020107
:20440000475A0201494D02014AB002014BFD02014E6402014E6402014E6402014E64020143
:204420004E6402014E6702015067855083855182759308E0FEA3E0FF9008770675F03F126D
:20444000008528EE75F03FA42583F583759308E0FD900000431200866CEDF090087706752E
:20446000F03FEF12008528EE75F03FA42583F583759308ED54FEF0900000531200866CE003
:20448000FBA3E0FAA3E0F91200D857D3EF9414EE64809480403A900000431200866CE02046
:2044A000E0032153B1855083855182759308E0FEA3E09008770675F03F12008528EE75F008
:2044C0003FA42583F583759308E04401F02153B1900000531200866CE0FBA3E0FAA3E0F9D4
:2044E000C001855083855182759308E0FEA3E0FF7C007D3F1200813874C82FF974763EA8A4
:2045000001FC7D09D0017E007F1512008055855083855182759308E0FEA3E0FF9008770619
:2045200075F03F12008528EE75F03FA42583F583759308E04401F09008770475F03FEF12E5
:20454000008528EE75F03FA42583F583759308E0FEA3E064014E60032153BF855083855170
:2045600082759308E0FEA3E0FF7C007D3F1200813874C82FF974763EFA7B0985508385510E
:2045800082759308A3E0FD1206A3B4215060855083855182759308E0FEA3E0FF9008770694
:2045A00075F03F12008528EE75F03FA42583F583759308E0FD900000431200866CEDF09011
:2045C00008770675F03FEF12008528EE75F03FA42583F583759308ED54FDF090000053127B
:2045E00000866CE0FBA3E0FAA3E0F91204A2DBEFF47002EEF47037900000431200866CE0CD
:2046000030E128855083855182759308E0FEA3E09008770675F03F12008528EE75F03FA492
:204620002583F583759308E04402F02153B1900000531200866CE0FBA3E0FAA3E0F9120042
:20464000841F1205B78EEF4E604D900000411200866CE0FEA3E0FF8550838551827593087C
:20466000E0FCA3E0FD6F7002EC6E602B900000431200866CE030E11C9008770675F03FED8E
:2046800012008528EC75F03FA42583F583759308E04402F02153B1900000531200866CE0F5
:2046A000FBA3E0FAA3E0F91200841F855083855182759308E0FAA3E0FB900876DD75F03FAA
:2046C00012008528EA75F03FA42583F5837593081200850B9008770675F03FEB12008528B4
:2046E000EA75F03FA42583F583759308E04402F09008770475F03FEB12008528EA75F03F53
:20470000A42583F583759308E0FEA3E064014E60032153BF855083855182759308E0FEA3DA
:20472000E0900876DD75F03F12008528EE75F03FA42583F583759308E0FCA3E0FDA3E0FE08
:20474000A3E0FF855083855182759308A3E09008ADEEF01206A2AA2150608550838551828C
:20476000759308E0FEA3E0FF9008770675F03F12008528EE75F03FA42583F583759308E00B
:20478000FD900000431200866CEDF09008770675F03FEF12008528EE75F03FA42583F583AB
:2047A000759308ED54FBF0900000531200866CE0FBA3E0FAA3E0F91200D857C3EE64809498
:2047C00080401F900000531200866CE0FBA3E0FAA3E0F91200D857D3EF9414EE64809480AE
:2047E0004037900000431200866CE030E228855083855182759308E0FEA3E09008770675A6
:20480000F03F12008528EE75F03FA42583F583759308E04404F02153B185508385518275E2
:204820009308E0FEA3E09008770375F03F12008528EE75F03FA42583F583759308E0604F12
:20484000900000531200866CE0FBA3E0FAA3E0F91200D857EF4E7037900000431200866CA1
:20486000E030E228855083855182759308E0FEA3E09008770675F03F12008528EE75F03FF3
:20488000A42583F583759308E04404F02153B1900000531200866CE0FBA3E0FAA3E0F9C08C
:2048A00001855083855182759308E0FEA3E0FF7C007D3F1200813874E12FF974763EA80186
:2048C000FC7D09D0017E007F1512008055855083855182759308E0FEA3E0FF9008770675E2
:2048E000F03F12008528EE75F03FA42583F583759308E04404F09008770475F03FEF120094
:204900008528EE75F03FA42583F583759308E0FEA3E064014E60032153BF8550838551822A
:20492000759308E0FEA3E0FF7C007D3F1200813874E12FF974763EFA7B0985508385518231
:20494000759308A3E0FD1206A397215060855083855182759308E0FEA3E0FF9008770675FA
:20496000F03F12008528EE75F03FA42583F583759308E0FD900000431200866CEDF09008BA
:20498000770675F03FEF12008528EE75F03FA42583F583759308ED54F7F0900000531200C5
:2049A000866CE0FBA3E0FAA3E0F91200841F120085FC49C20000000149CE000000020000C4
:2049C00049DB900000441200866CE4F08044900000441200866C7401F0803790000043126A
:2049E00000866CE030E328855083855182759308E0FEA3E09008770675F03F12008528EE23
:204A000075F03FA42583F583759308E04408F02153B1900000441200866CE0FF8550838549
:204A20005182759308E0FCA3E0FD900876F675F03F12008528EC75F03FA42583F583759374
:204A400008EFF09008770675F03FED12008528EC75F03FA42583F583759308E04408F090FA
:204A600008770475F03FED12008528EC75F03FA42583F583759308E0FEA3E064014E600388
:204A80002153BF900876F675F03FED12008528EC75F03FA42583F583759308E0FF855083F4
:204AA000855182759308A3E0FD1206A618215060855083855182759308E0FEA3E090087638
:204AC000F775F03F12008528EE75F03FA42583F583759308E0FCA3E0FDA3E0FEA3E0FF9027
:204AE0000000451200866C1200850B900000531200866CE0FBA3E0FAA3E0F91200841F1249
:204B00000085FC4B13000000014B2D0000000200004B54900000451200866CC083C082E05E
:204B2000FCA3E0FDA3E0FEA3E044018018900000451200866CC083C082E0FCA3E0FDA3E0DB
:204B4000FEA3E054FEFFEC759308D082D0831200850B80032153B1900000451200866CE0DF
:204B6000FCA3E0FDA3E0FEA3E0FF855083855182759308E0FAA3E0FB900876F775F03F12E3
:204B8000008528EA75F03FA42583F5837593081200850B9008770475F03FEB12008528EA19
:204BA00075F03FA42583F583759308E0FEA3E064014E60032153BF85508385518275930813
:204BC000E0FEA3E0900876F775F03F12008528EE75F03FA42583F583759308E0FCA3E0FD4A
:204BE000A3E0FEA3E0FF855083855182759308A3E09008ADDFF01206A1F621506085508383
:204C0000855182759308E0FEA3E0900876FF75F03F12008528EE75F03FA42583F5837593FD
:204C200008E0FCA3E0FDA3E0FEA3E0FF900000451200866C1200850B900000531200866CAB
:204C4000E0FBA3E0FAA3E0F91200841F120085FC4C60000000014C7A0000000200004CA1D6
:204C6000900000451200866CC083C082E0FCA3E0FDA3E0FEA3E044028018900000451200B1
:204C8000866CC083C082E0FCA3E0FDA3E0FEA3E054FDFFEC759308D082D0831200850B802A
:204CA000032153B1900000451200866CE0FCA3E0FDA3E0FEA3E0FF855083855182759308D4
:204CC000E0FAA3E0FB900876FF75F03F12008528EA75F03FA42583F5837593081200850B08
:204CE000900876FB75F03FEB12008528EA75F03FA42583F583759308E0FCA3E0FDA3E0FE1E
:204D0000A3E0FF900000451200866C1200850B900000531200866CE0FBA3E0FAA3E0F912C9
:204D200000841F120085FC4D37000000014D510000000200004D78900000451200866CC0BA
:204D400083C082E0FCA3E0FDA3E0FEA3E044018018900000451200866CC083C082E0FCA374
:204D6000E0FDA3E0FEA3E054FEFFEC759308D082D0831200850B80032153B190000045122F
:204D800000866CE0FCA3E0FDA3E0FEA3E0FF855083855182759308E0FAA3E0FB900876FBA1
:204DA00075F03F12008528EA75F03FA42583F5837593081200850B9008770475F03FEB12D8
:204DC000008528EA75F03FA42583F583759308E0FEA3E064014E60032153BF8550838551EC
:204DE00082759308E0FEA3E0900876FF75F03F12008528EE75F03FA42583F583759308E00A
:204E0000FCA3E0FDA3E0FEA3E0FF855083855182759308A3E09008ADE4F01206A2328550F6
:204E200083855182759308E0FEA3E0900876FB75F03F12008528EE75F03FA42583F58375EF
:204E40009308E0FCA3E0FDA3E0FEA3E0FF855083855182759308A3E09008ADE9F01206A23D
:204E60006E2150602153B9855083855182759308E0FEA3E0FF9008770675F03F120085282E
:204E8000EE75F03FA42583F583759308E0FD900000431200866CEDF09008770675F03FEF73
:204EA00012008528EE75F03FA42583F583759308ED54EFF0900000531200866CE0FBA3E068
:204EC000FAA3E0F91200841F120085FC4EDC000000014EE90000000200004EF59000004994
:204EE0001200866C7401F08043900000491200866CE4F08037900000431200866CE030E453
:204F000028855083855182759308E0FEA3E09008770675F03F12008528EE75F03FA42583F2
:204F2000F583759308E04410F02153B1900000491200866CE07003214FC58550838551828B
:204F4000759308E0FEA3E0FF7C007D3F1200813874DD2FF974763EFA7B091204A2DBEFF449
:204F60007002EEF46028855083855182759308E0FEA3E0FF7C007D3F1200813874E12FF9B5
:204F800074763EFA7B091200D857EF4E7037900000431200866CE030E428855083855182A3
:204FA000759308E0FEA3E09008770675F03F12008528EE75F03FA42583F583759308E0447E
:204FC00010F02153B1900000491200866CE0FF855083855182759308E0FCA3E0FD900877C5
:204FE0000375F03F12008528EC75F03FA42583F583759308EFF09008770675F03FED120050
:205000008528EC75F03FA42583F583759308E04410F09008770475F03FED12008528EC7597
:20502000F03FA42583F583759308E0FEA3E064014E60032153BF9008770375F03FED12000E
:205040008528EC75F03FA42583F583759308E0FF855083855182759308A3E0FD1206A63032
:2050600012068C4A2153BF900000531200866CE0FBA3E0FAA3E0F91200841F120085FC50BC
:20508000A10000000151620000000251650000000451680000000552550000000600005341
:2050A000B11206394E9000003D1200866CE060032151419000003E1200866CE0FEA3E04E58
:2050C0007006FE7F032153C2E4FFFEFDFC900000171200866CE0F8A3E0F9A3E0FAA3E0FBD0
:2050E000C3120083E8606C7B09900000171200866CA982AA831204A2DBBEFF06BFFF0321E5
:2051000053B1900000171200866CE0FCA3E0FDA3E0FEA3E0FF1205B78EEF4E6036900000C2
:20512000411200866CE0FEA3E0FF855083855182759308E0FCA3E06F7002EC6E6015215387
:20514000B1900000401200866CE05406640660032153B19000003E1200866CE4F0A3042130
:2051600053392153B12153B11206394EEF4E60032153B17E007F3F7D007B0985508385518A
:2051800082A3A3759308A982AA83120089B19000003E1200866CE4F0A37403F07B0985508A
:2051A00083855182A3A3759308A982AA83855083855182759308A3E0FD12068E2A900000C6
:2051C000401200866CE4F0FFFEFDFC900000171200866CE0F8A3E0F9A3E0FAA3E0FBC312F2
:2051E0000083E8600C900000401200866CE04402F07B099000001B1200866CA982AA831251
:2052000000D857EF4E600C900000401200866CE04404F07B09855083855182A3A375930840
:20522000A982AA83C001855083855182759308E0FEA3E0FF7C007D3F1200813874C82FF9CE
:2052400074763EA801FC7D09D0017E007F3F120080552153B7855083855182759308E0FE3E
:20526000A3E0FF9008770475F03F12008528EE75F03FA42583F583759308E0FCA3E04C70B5
:2052800002802E855083855182759308E0FEA3E0FF9008770475F03F12008528EE75F03F36
:2052A000A42583F583759308E0FCA3E064034C702AF58375823FC083C082FDC005FC7D3FC1
:2052C0001200813874C82FF974763EFA7B09D005D007D006120089B12153BF8550838551CA
:2052E00082759308E0FEA3E09008770475F03F12008528EE75F03FA42583F583759308E0FF
:20530000FEA3E064014E60032153AFFE7F3FFD7B09855083855182A3A3759308A982AA8338
:20532000120089B19000003E1200866CE4F0A3F0900000401200866CE4F07B0985508385DF
:205340005182A3A3759308A982AA83C001855083855182759308E0FEA3E0FF7C007D3F12A1
:2053600000813874C82FF974763EA801FC7D09D0017E007F3F1200805585508385518275A4
:205380009308E0FEA3E0FF7C007D3F1200813874C82FF974763EFA7B0985508385518275E0
:2053A0009308A3E0FD120699BB12068C4A800880007E007F03800B80067E007F028003E4F9
:2053C000FEFF900000580200864590086D3CE0FBA3E0FAA3E02414F9E43AFA90086D39EB8D
:2053E000F0A3EAF0A3E9F090086E57E0FBA3E0FAA3E0242CF9E43AFA900806BFEBF0A3EA66
:20540000F0A3E9F090086E57A3E0FAA3E0242BF9E43AFA90080403EBF0A3EAF0A3E9F09060
:20542000086E57A3E0FAA3E02418F9E43AFA900806ABEBF0A3EAF0A3E9F090086E57A3E055
:20544000FAA3E0241AF9E43AFA90080400EBF0A3EAF0A3E9F090086E57A3E0FAA3E0241C73
:20546000F9E43AFA900806BCEBF0A3EAF0A3E9F090086E57A3E0FAA3E0241EF9E43AFA90AD
:205480000806AEEBF0A3EAF0A3E9F090086E57A3E0FAA3E02420F9E43AFA900806B1EBF0A0
:2054A000A3EAF0A3E9F090086E57A3E0FAA3E02422F9E43AFA9008040AEBF0A3EAF0A3E9B5
:2054C000F090086E57A3E0FAA3E02424F9E43AFA900806B5EBF0A3EAF0A3E9F090086E57A2
:2054E000A3E0FAA3E02426F9E43AFA9008040DEBF0A3EAF0A3E9F090086D4AE0FD30E6672B
:20550000900806BFE0FBA3E0FAA3E0F9E412008124900806BFE0FBA3E0FAA3E02402F9E484
:205520003AFAE4F5F01200827E900806ABE0FBA3E0FAA3E0F9E475F0011200827E90080645
:20554000BCE0FBA3E0FAA3E0F9E475F0011200827E900806B1E0FBA3E0FAA3E0F9E4F5F073
:205560001200827E216474ED30E70321647490086D4AE020E1032161C9900806BFE0FBA3C7
:20558000E0FAA3E0F9120080D360032161C99008AB097481F0A374D0F0A374DFF0A3E4F03D
:2055A000A37404F090086D39E0FBA3E0FAA3E0F912064A46EF6003215647900893BBF090B0
:2055C000086D39E0FBA3E0FAA3E02405F9E43AFA900893BBE0FF7C0029F9EC3AFAA3EBF007
:2055E000A3EAF0A3E9F0120080D3FE64206004EEB43F1174BF2FF582E43493F58375930869
:20560000E4F0801F900893BBE0FF04F074BF2FF582E43493F583759308EEF0900893BBE0AE
:20562000B4209C7B097A9379BF1200D857EF4E60032156E678BF7C937D097B817AD079E484
:20564000120087F32156E69008A5117481F0A374D0F0A374EEF090086D39E0FBA3E0FAA329
:20566000E0F91205F290900893BCEBF0A3EAF0A3E9F0900893BCE0FBA3E0FAA3E04A4B7036
:205680001C900806B4E064037003215AB090086D39E0FBA3E0FAA3E0F902037A4990089CA9
:2056A000AB7481F0A374D0F0A374EEF0A37481F0A374D0F0A374F8F0A37409F0A37493F086
:2056C000A374BFF0900893BCE0FBA3E0FAA3E0F9120542FC900806BFE0FBA3E0FAA3E0F9C3
:2056E0007401120081249008AB097481F0A374D0F0A374FAF0A3E4F0A3740AF07B097A935C
:2057000079BF12064A46EF704A90086E57E0FBA3E0FAA3E02404F9E43AFA1200841F900842
:2057200006B8E0F8A3E0F9A3E0FAA3E0FBC3120083E8700321583AE4FFFEFDFC900806B8C6
:20574000E0F8A3A3A3E0C3120083E8600321593421583A9008AB097481F0A374D1F0A37484
:2057600005F0A3E4F0A3740AF07B097A9379BF12064A46EF701078BF7C937D097B817AD1B9
:205780007910120087F39008AB097481F0A374D1F0A3741DF0A3E4F0A37404F07B097A93B4
:2057A00079BF12064A46EF70032158F39008AB097481F0A374D1F0A37422F0A3E4F0A3747B
:2057C0000BF07B097A9379BF12064A46EF704E900806BFE0FBA3E0FAA3E0F9740212008176
:2057E000247B007A007900C003C002C001900806BFE0FBA3E0FAA3E02404F9E43AFA12004E
:205800008551900806BFE0FBA3E0FAA3E02402F9E43AFAE4F5F01200827E2163869008A81E
:20582000787409F0A37493F0A374B6F07B097A9379BF1205C06FEF4E702378BF7C937D0981
:205840007B817AD1792E120087F3900806B47401F0E4FFFEFDFC900806B8215A5E90080670
:20586000BFE0FBA3E0FAA3E0F9740212008124900893B6E0FBA3E0FAA3E0F9C003C002C06E
:2058800001900806BFE0FBA3E0FAA3E02404F9E43AFA12008551900893B9E0FEA3E0FF90DA
:2058A0000806BFE0FBA3E0FAA3E02402F9E43AFAEE8FF01200827E1206A9EDC004C005C093
:2058C00006C0071206AD9DE4FCFD7B587A02F9F81200829AD003D002D001D000EB2FFFEA05
:2058E0003EFEE93DFDE83CFC900804061200850B21638690086E57E0FBA3E0FAA3E024047B
:20590000F9E43AFA1200841F900806B8E0F8A3E0F9A3E0FAA3E0FBC3120083E8603EE4FF5B
:20592000FEFDFC900806B8E0F8A3A3A3E0C3120083E860289008A86F7481F0A374D1F0A3A2
:20594000743EF0A37481F0A374D1F0A3742EF07B817AD1793812061FA3216474900806BFE8
:20596000E0FBA3E0FAA3E0F9120080D364016003215A659008AB097481F0A374D1F0A37426
:2059800056F0A3E4F0A3740AF07B097A9379BF12064A46EF6003215A6590086D39E0FBA3DA
:2059A000E0FAA3E0F912062856EF4E70289008A86F7481F0A374D1F0A37461F0A37481F0CA
:2059C000A374D1F0A3742EF07B817AD1793812061FA321647412063398EF4E70289008A8F7
:2059E0006F7481F0A374D1F0A37470F0A37481F0A374D1F0A3742EF07B817AD1793812065F
:205A00001FA321647490086E57E0FBA3E0FAA3E02404F9E43AFA1200841F900806B812003D
:205A2000850B900806B47402F01206A9EDC004C005C006C0071206AD9DE4FCFD7B587A02CC
:205A4000F9F81200829AD003D002D001D000EB2FFFEA3EFEE93DFDE83CFC900804061200AB
:205A6000850B215FEF9008AB097481F0A374D1F0A3742EF0A3E4F0A37409F07B097A937958
:205A8000BF12064A46EF7009900806B404F0215FEF900806B4E0B4010F78BF7C937D097B45
:205AA000817AD1792E215F89900806B4E0B4033C9008A86F7481F0A374D1F0A3748AF0A3A5
:205AC0007481F0A374D1F0A3742EF07B817AD1793812061FA3900806B47401F0E4FFFEFD6D
:205AE000FC900806B81200850B216474900806BFE0FBA3E0FAA3E0F9120080D3640160035B
:205B0000215FEF9008AB097481F0A374D1F0A37498F0A3E4F0A37408F07B097A9379BF120D
:205B2000064A46EF701390086D39E0FBA3E0FAA3E0F91204B720215FEF9008AB097481F0BE
:205B4000A374D1F0A374A1F0A3E4F0A3740BF07B097A9379BF12064A46EF702690086D3908
:205B6000E0FBA3E0FAA3E0F91204ECBDEF4E7003215F7978BF7C937D097B817AD179AD218F
:205B80005F899008AB097481F0A374D1F0A374ADF0A3E4F0A37408F07B097A9379BF1206F9
:205BA0004A46EF701A90086D39E0FBA3E0FAA3E0F9120444EFEF4E6003215FEF215F7990E9
:205BC00008AB097481F0A374D1F0A374B6F0A3E4F0A37409F07B097A9379BF12064A46EFA8
:205BE000701A90086D39E0FBA3E0FAA3E0F9120432BEEF4E6003215FEF215F799008AB09AF
:205C00007481F0A374D1F0A374C0F0A3E4F0A3740AF07B097A9379BF12064A46EF701A90FE
:205C2000086D39E0FBA3E0FAA3E0F912043FCAEF4E6003215FEF215F799008AB097481F08A
:205C4000A374D1F0A374CBF0A3E4F0A37407F07B097A9379BF12064A46EF701A90086D39ED
:205C6000E0FBA3E0FAA3E0F912021D6FEF4E6003215FEF215F799008AB097481F0A374D18F
:205C8000F0A374D3F0A3E4F0A37407F07B097A9379BF12064A46EF701A90086D39E0FBA30F
:205CA000E0FAA3E0F91202A3A4EF4E6003215FEF215F799008AB097481F0A374D1F0A3740B
:205CC000DBF0A3E4F0A37408F07B097A9379BF12064A46EF701A90086D39E0FBA3E0FAA350
:205CE000E0F91204A4EAEF4E6003215FEF215F799008AB097481F0A374D1F0A374E4F0A388
:205D0000E4F0A37407F07B097A9379BF12064A46EF701A90086D39E0FBA3E0FAA3E0F91293
:205D200004FF6FEF4E6003215FEF215F799008AB097481F0A374D1F0A374ECF0A3E4F0A3D3
:205D40007409F07B097A9379BF12064A46EF701A90086D39E0FBA3E0FAA3E0F912057D68DE
:205D6000EF4E6003215FEF215F799008AB097481F0A374D1F0A374F7F0A3E4F0A37407F08F
:205D80007B097A9379BF12064A46EF701A90086D39E0FBA3E0FAA3E0F91205AF7BEF4E6029
:205DA00003215FEF215F799008AB097481F0A374D1F0A374FFF0A3E4F0A37408F07B097AE5
:205DC0009379BF12064A46EF702690086D39E0FBA3E0FAA3E0F91200F2A7EF4E7003215FDE
:205DE0007978BF7C937D097B817AD179FF215F899008AB097481F0A374D2F0A37408F0A3DA
:205E0000E4F0A37407F07B097A9379BF12064A46EF701A90086D39E0FBA3E0FAA3E0F91292
:205E2000045B48EF4E6003215FEF215F799008AB097481F0A374D2F0A37410F0A3E4F0A378
:205E4000740AF07B097A9379BF12064A46EF702690086D39E0FBA3E0FAA3E0F91200FE3983
:205E6000EF4E7003215F7978BF7C937D097B817AD27908215F899008AB097481F0A374D2C1
:205E8000F0A3741BF0A3E4F0A3740CF07B097A9379BF12064A46EF702690086D39E0FBA3B4
:205EA000E0FAA3E0F91204E5C1EF4E7003215F7978BF7C937D097B817AD179AD215F899055
:205EC00008AB097481F0A374D2F0A37428F0A3E4F0A37408F07B097A9379BF12064A46EF33
:205EE000701990086D39E0FBA3E0FAA3E0F91204C0EEEF4E6003215FEF807E9008AB097476
:205F000081F0A374D2F0A37431F0A3E4F0A3740AF07B097A9379BF12064A46EF70249008EB
:205F20006D39E0FBA3E0FAA3E0F91202795BEF4E7002804578BF7C937D097B817AD2793CC2
:205F400080479008AB097481F0A374D2F0A37444F0A3E4F0A3740AF07B097A9379BF1206BC
:205F60004A46EF702A90086D39E0FBA3E0FAA3E0F91204DEAAEF4E7004FE7F012278BF7C54
:205F8000937D097B817AD2793C120087F380609008AB097481F0A374D2F0A3744FF0A3E498
:205FA000F0A37409F07B097A9379BF12064A46EF701290088AB4F0A304F090086D4A7410CF
:205FC000F02164749008AB097481F0A374D2F0A37459F0A3E4F0A3740BF07B097A9379BF1C
:205FE00012064A46EF700890088AAEF0A304F09008AB097481F0A374D1F0A374ADF0A3E4F7
:20600000F0A37408F07B097A9379BF12064A46EF70181206ADA6EF4E701078BF7C937D09A5
:206020007B817AD2793C120087F3E4900893BBF09008AB097481F0A374D2F0A37465F0A304
:20604000E4F0A3740BF07B097A9379BF12064A46EF7014120658C378BF7C937D097B817A01
:20606000D27971120087F39008AB097481F0A374D2F0A3747DF0A3E4F0A3740BF07B097AC3
:206080009379BF12064A46EF701A9008B03DF0A304F078BF7C937D097B817AD279891200E0
:2060A00087F38008E49008B03DF0A3F0E49008ACACF0A3F09008AB097481F0A374D2F0A3EE
:2060C0007431F0A3E4F0A3740AF07B097A9379BF12064A46EF70459008925C7481F0A3740C
:2060E000D2F0A37495F0A37409F0A374ACF0A374ACF07B097A9379BF1200C9E478BF7C93FE
:206100007D097B817AD2793C120087F39008ACADE024FFF09008ACACE034FFF0900893BBB3
:20612000E0FD75F017A42410F582E5F03404F583759308E0FBA3E0FAA3E04A4B700A9008A0
:206140006D4A7410F0216474ED75F017A42413F9740435F0FA7B091200D8579008AB0CEE45
:20616000F0A3EFF0900893BBE075F017A42413F9740435F0FA9008AB097409F0A3EAF0A327
:20618000E9F07B097A9379BF12064A46EF7030900806BFE0FBA3E0FAA3E0F97403120081EB
:2061A00024900893BBE0FF900806BFE0FBA3E0FAA3E02401F9E43AFAEF12008124800A90C8
:2061C0000893BBE004F021611C900806BFE0FBA3E0FAA3E0F9120080D3640360032163868D
:2061E00090086E5AF0A3F090086D4AE06404600321627A90080400E0FBA3E0FAA3E0F91243
:20620000008204FF900806ABE0FBA3E0FAA3E0F9E5F08FF01200827E900806AEE0FBA3E0CC
:20622000FAA3E0F912008204FF900806BCE0FBA3E0FAA3E0F9E5F08FF01200827E90080421
:206240000AE0FBA3E0FAA3E0F912008204FF900806B1E0FBA3E0FAA3E0F9E5F08FF0120040
:20626000827E9008040DE0FBA3E0FAA3E0F912008204FF900806B52162FE900806ABE0FB12
:20628000A3E0FAA3E0F912008204FF90080400E0FBA3E0FAA3E0F9E5F08FF01200827E9008
:2062A0000806BCE0FBA3E0FAA3E0F912008204FF900806AEE0FBA3E0FAA3E0F9E5F08FF035
:2062C0001200827E900806B1E0FBA3E0FAA3E0F912008204FF9008040AE0FBA3E0FAA3E071
:2062E000F9E5F08FF01200827E900806B5E0FBA3E0FAA3E0F912008204FF9008040DE0FBFD
:20630000A3E0FAA3E0F9E5F08FF01200827E900806BFE0FBA3E0FAA3E02401F9E43AFA129E
:206320000080D375F017A42410F582E5F03404F583759308E0FBA3E0FAA3E0F91200863806
:20634000EF600790086D4A7410F01206A9EDC004C005C006C0071206AD9DE4FCFD7B587AD4
:2063600002F9F81200829AD003D002D001D000EB2FFFEA3EFEE93DFDE83CFC900804061280
:2063800000850B21647490086D4AE030E07A900806BFE0FBA3E0FAA3E02402F9E43AFA123A
:2063A000008204C39478E5F09405402A74FA75F08812008252900806BFE0FBA3E0FAA3E037
:2063C0002404F9E43AFA09E970010A740575F078120082528032900806BFE0FBA3E0FAA3D1
:2063E000E02402F9E43AFAE4F5F01200827E900806BFE0FBA3E0FAA3E0F9120080D3B4025F
:206400000790086D4A7410F0900806BFE0FBA3E0FAA3E02402F9E43AFA12008204FFAEF00E
:20642000D39478EE940590086E5A40097405F0A37478F08005EEF0A3EFF090086E5AE0FE42
:20644000A3E0FF900806BFE0FBA3E0FAA3E02404F9E43AFA12008534C003C00290086D39BB
:20646000E0FBA3E0FAA3E0F8AC02AD03D002D003120080557E007F01229000FFFD1200861B
:2064800045EBF0A3EAF0A3E9F09000FF95120086451206ADA6EF4E7006FE7F022171DB9048
:2064A0000000711200866CE0FBA3E0FAA3E0F912008204FDACF0C3940DEC648094805003C7
:2064C0002171D29000006E1200866CE0FBA3E0FAA3E0F9C003C002C001C3ED9401FDEC947A
:2064E00000FC9000006B1200866CE0F9A3E0FAA3E09008A42FC9F0A3EAF0A3E9F09000001B
:206500006B1200866CE0FBA3E0FAA3E02434F9E43AFA12008204C39401FEE5F094009008D9
:20652000A432F0A3CEF0D001D002D0031205AB63EF4E60032171D27C007D02900000711287
:2065400000866CE0FBA3E0FAA3E0F91200820425E0FFE5F033FE9000006E1200866CE0FBF6
:20656000A3E0FAA3E02FF9EA3EFAC3E99DF9EA9CFA12008204FFAEF0855083855182A3A3E4
:20658000759308EEF0A3EFF0855083855182A3A3759308E0FEA3E0FFC39401EE64809480E7
:2065A000400BD3EF9432EE6480948040032171D2855083855182A3A375930874FFF5F0120B
:2065C0000081D89000006B1200866CE0FBA3E0FAA3E02437F9E43AFA12008204FFAEF0E502
:2065E000F060032171D2EF24FD700321683124FE7003216C06240360032171D285508385B4
:206600005182A3A3759308E0FEA3E0FF900859AF75F01312008528EE75F013A42583F583F0
:20662000759308E0FD9000006A1200866CEDF0900859AF75F013EF12008528EE75F013A4C2
:206640002583F583759308ED54FEF0900000741200866CE0FBA3E0FAA3E0F91200D857D3EB
:20666000EF9408EE64809480403C9000006A1200866CE020E0032171CC855083855182A39B
:20668000A3759308E0FEA3E0900859AF75F01312008528EE75F013A42583F583759308E0F5
:2066A0004401F02171CC855083855182759308E4F0A3F0855083855182759308E0FEA3E0FF
:2066C000FFC39432EE64809480501B1206503FEF4E6013855083855182759308E475F00180
:2066E000120081D880CD855083855182759308E0FEA3E0FF4E7010855083855182A3A37589
:206700009308F0A3F08041C3EF9401FFEE9400FE855083855182A3A3759308E0FCA3E0D39C
:206720009FEE6480F8EC648098401D855083855182759308E0FFA3E0855083855182A3A313
:20674000759308CFF0A3EFF07E007F217D007B09900000231200866CA982AA83120089B16E
:20676000900000771200866CE0FEA3E0FF900000741200866CE0FBA3E0FAA3E0F9C003C04F
:2067800002C0017B09900000231200866CA982AA83A801AC02AD03D001D002D00312008094
:2067A000557B09900000231200866CA982AA83C001855083855182A3A3759308E0FEA3E0C9
:2067C000FF7C007D1312008138749D2FF974593EA801FC7D09D0017E007F09120080558531
:2067E0005083855182A3A3759308E0FEA3E0FF900859AF75F01312008528EE75F013A425B2
:2068000083F583759308E04401F0900859AD75F013EF12008528EE75F013A42583F58375F5
:206820009308E0FEA3E064014E60032171D8216BCF855083855182A3A3759308E0FEA3E01A
:20684000FF900859AF75F01312008528EE75F013A42583F583759308E0FD9000006A12003F
:20686000866CEDF0900859AF75F013EF12008528EE75F013A42583F583759308ED54FDF01B
:20688000900000771200866CE0FEA3E0D39407EE6480948040399000006A1200866CE030B1
:2068A000E12A855083855182A3A3759308E0FEA3E0900859AF75F01312008528EE75F01329
:2068C000A42583F583759308E04402F02171CC855083855182759308E4F0A3F0855083856C
:2068E0005182759308E0FEA3E0FFC39432EE64809480501B1206503FEF4E60138550838547
:206900005182759308E475F001120081D880CD855083855182759308E0FEA3E0FF4E7010A4
:20692000855083855182A3A3759308F0A3F08041C3EF9401FFEE9400FE855083855182A3F4
:20694000A3759308E0FCA3E0D39FEE6480F8EC648098401D855083855182759308E0FFA3E2
:20696000E0855083855182A3A3759308CFF0A3EFF07E007F077D007B0990000004120086BF
:206980006CA982AA83120089B1900000771200866CE0FEA3E0FF900000741200866CE0FB99
:2069A000A3E0FAA3E0F9C003C002C0017B09900000041200866CA982AA83A801AC02AD031D
:2069C000D001D002D003120080557B09900000041200866CA982AA837D077C0012055D5E14
:2069E000EFF47002EEF470399000006A1200866CE030E12A855083855182A3A3759308E0B8
:206A0000FEA3E0900859AF75F01312008528EE75F013A42583F583759308E04402F021713C
:206A2000CC7B09900000041200866CA982AA83C003C002C0017B09900000121200866CA9FD
:206A400082AA839008AA91EBF0A3EAF0A3E9F0D001D002D0031205AC647E007F077D007B47
:206A600009900000191200866CA982AA83120089B17B09900000191200866CA982AA83C073
:206A800003C002C0017B09900000121200866CA982AA83A801AC02AD03D001D002D0037EF3
:206AA000007F0712008927EF70399000006A1200866CE030E12A855083855182A3A37593DF
:206AC00008E0FEA3E0900859AF75F01312008528EE75F013A42583F583759308E04402F026
:206AE0002171CC855083855182A3A3759308E0FEA3E0FF7B09900000121200866CA982AAD3
:206B0000831204516EEF4E70399000006A1200866CE030E12A855083855182A3A375930818
:206B2000E0FEA3E0900859AF75F01312008528EE75F013A42583F583759308E04402F021AC
:206B400071CC7B09900000121200866CA982AA83C001855083855182A3A3759308E0FEA32E
:206B6000E0FF7C007D131200813874A62FF974593EA801FC7D09D0017E007F07120080552B
:206B8000855083855182A3A3759308E0FEA3E0FF900859AF75F01312008528EE75F013A4AE
:206BA0002583F583759308E04402F0900859AD75F013EF12008528EE75F013A42583F583A1
:206BC000759308E0FEA3E064014E60032171D8855083855182A3A3759308E0FEA3E0FF7CE2
:206BE000007D1312008138AC06AD0774A62DF974593CFA7B09C003C002C001855083855199
:206C000082A3A3216DDD900000741200866CE0FBA3E0FAA3E0F91200841F120085FC6C4071
:206C2000000000016E06000000026E06000000046E09000000056F170000000600006E06E9
:206C4000855083855182A3A3759308E0FEA3E0FF9000004412065043900000561200866C65
:206C6000E020E1032171CC855083855182759308E4F0A3F0855083855182759308E0FEA36A
:206C8000E0FFC39432EE6480948050777B09900000121200866CA982AA83C003C002C00117
:206CA0007B09900000201200866CA982AA839008A6E4EBF0A3EAF0A3E9F0D001D002D003D8
:206CC0001205FF55EF4E603B855083855182759308E0FEA3E0FF855083855182A3A3759353
:206CE00008E0FCA3E0B50707ECB506032170E7855083855182759308E475F001120081D8D3
:206D0000216C74855083855182759308E0FAA3E0FBC39432EA6480948040032171CC7C00D2
:206D20007D13AF03AE0212008138749D2FF974593EFA7B09C003C001855083855182A3A35A
:206D4000759308E0FEA3E0FF12008138749D2FF974593EA801FCAD03D001D0037E007F13AB
:206D600012008055900000541200866CE4F0A304F07B09900000441200866CA982AA83C065
:206D800001855083855182759308E0FEA3E0FF7C007D1312008138749D2FF974593EA8010E
:206DA000FC7D09D0017E007F1312008055855083855182759308E0FEA3E0FF7C007D13124B
:206DC000008138AC06AD0774A62DF974593CFA7B09C003C002C001855083855182759308C7
:206DE000E0FEA3E0FF749D2DF974593CFA90089765EBF0A3EAF0A3E9F0D001D002D0031209
:206E0000035E5E2171C62171CC855083855182759308E4F0A3F0855083855182759308E036
:206E2000FEA3E0FFC39432EE64809480501B1206503FEF4E6013855083855182759308E4FD
:206E400075F001120081D880CD855083855182759308E0FEA3E0FF4E701085508385518276
:206E6000A3A3759308F0A3F08046C3EF9401FFEE9400FE855083855182A3A3759308E0FCCB
:206E8000A3E0D39FEE6480F8EC648098401F855083855182759308E0FFA3E085508385511C
:206EA00082A3A3759308CFF0A3EFF080032171CC7E007F137D007B09900000571200866CDC
:206EC000A982AA83120089B1900000671200866CE4F0A37403F07B09900000571200866CC6
:206EE000A982AA83C001855083855182A3A3759308E0FEA3E0FF7C007D1312008138749D2B
:206F00002FF974593EA801FC7D09D0017E007F13120080552171D885508385518275930821
:206F2000E4F0A3F0855083855182759308E0FEA3E0FFC39432EE6480948050217B099000D6
:206F4000004412065045EF4E6013855083855182759308E475F001120081D880C78550837C
:206F6000855182759308E0FCA3E0FD64014C7003217159ED4C7005FEFF2171DB8550838549
:206F80005182759308E0FEA3E0C39401FFEE9400FE855083855182A3A3759308E0FCA3E071
:206FA000FDD39FEE6480F8EC64809840032170E7900859AD75F013ED12008528EC75F0134F
:206FC000A42583F583759308E0FEA3E064034E7039FE7F13C006C007FFC00785508385510D
:206FE00082A3A3759308E0FEA3E0FF7C007D1312008138749D2FF974593EFA7B09D005D01B
:2070000007D006120089B12171D87E007F077D007B099000000B1200866CA982AA831200CF
:2070200089B1855083855182759308E4F0A3F0855083855182759308E0FEA3E0FFC3943246
:20704000EE6480948040032170D07B09900000121200866CA982AA83C003C002C0017B095A
:20706000900000201200866CA982AA839008A6E4EBF0A3EAF0A3E9F0D001D002D003120581
:20708000FF55EF4E6036855083855182759308E0FEA3E0FF855083855182A3A3759308E0C3
:2070A000FCA3E0B50716ECB50612855083855182A3A3759308EEF0A3EFF0801485508385EF
:2070C0005182759308E475F001120081D821702F855083855182759308E0FEA3E0C39432AE
:2070E000EE6480948040032171D8855083855182A3A3759308E0FEA3E07803CEA2E713CEE3
:2071000013D8F8FF9000000B1200866CE5822FF582E5833EF583C083C082759308E0FF85CA
:207120005083855182A3A3759308A3E05407FE7401A806088002C333D8FC4F759308D082CA
:20714000D083F07B099000000B1200866CA982AA8312054B67EF4E7005FE7F03807D7E00FB
:207160007F137D007B09900000441200866CA982AA83120089B17B09900000441200866CA4
:20718000A982AA83C001855083855182A3A3759308E0FEA3E0FF7C007D1312008138749D88
:2071A0002FF974593EA801FC7D09D0017E007F13120080557B099000000B1200866CA9825B
:2071C000AA831205761712068C4A800C7E007F0380097E007F028003E4FEFF90000079026D
:2071E0000086457B097A96799A9008A7CFEFF0A3EDF0A3EBF0A3EAF0A3E9F09008A7D7E43F
:20720000F0A304F09008A7D7E07004A3E0640170279008A7CFE0FF9008A96B7401F0A374E9
:2072200009F0A374A7F0A374D7F07B0F7D0512066992EF60CF7F01229008A7D0E0FF640197
:20724000700321768FEF6404700321768FEF6407700321768F9008A7D4E0FBA3E0FAA3E0C4
:207260002404F9E43AFA120080D35403C4F8540FC868FFE4C454F048FE9008A7D4A3E0FA09
:20728000A3E02403F9E43AFA120080D35403FDEEFCEF4DFD9008A7D4A3E0FAA3E02405F922
:2072A000E43AFA120080D354034CFFED9008A7D7CFF0A3EFF09008A7D4A3E0FAA3E0240F25
:2072C000F9E43AFA120080D37E0054037806C333CE33CED8F9FDAC069008A7D4E0FBA3E02F
:2072E000FAA3E0240EF9E43AFA120080D37E0054037802C333CE33CED8F9FFEE4CFCEF4D13
:20730000FD9008A7D4E0FBA3E0FAA3E02410F9E43AFA120080D3540325E025E04CFEEDFF41
:207320009008A7D7E04EF0A3E04FF09008A7CFE075F02FA4242DF9741D35F0FA7B89120021
:2073400080D3D39403404A9008A7D4E0FBA3E0FAA3E02406F9E43AFA120080D35403C454E9
:20736000F0FE9008A7D7E04EF0A3E0F09008A7D4A3E0FAA3E02411F9E43AFA120080D35466
:2073800003C4333354C0FE9008A7D7E04EF0A3E0F09008A7CFE0FF9008A7D7E0FAA3E0FBAC
:2073A0007D071206928DEF60037F01229008A7CFE075F02FA4242DF9741D35F0FA7B8912E8
:2073C0000080D3D3940450032175229008A7D4E0FBA3E0FAA3E02408F9E43AFA120080D354
:2073E0005403C4F8540FC868FFE4C454F048FE9008A7D4A3E0FAA3E02407F9E43AFA120055
:2074000080D35403FDEEFCEF4DFD9008A7D4A3E0FAA3E02409F9E43AFA120080D354034C49
:20742000FFED9008A7D7CFF0A3EFF09008A7D4A3E0FAA3E02413F9E43AFA120080D37E00CB
:2074400054037806C333CE33CED8F9FDAC069008A7D4E0FBA3E0FAA3E02412F9E43AFA12CB
:207460000080D37E0054037802C333CE33CED8F9FFEE4CFCEF4DFD9008A7D4E0FBA3E0FAFB
:20748000A3E02414F9E43AFA120080D3540325E025E04CFEEDFF9008A7D7E04EF0A3E04F1E
:2074A000F09008A7CFE075F02FA4242DF9741D35F0FA7B89120080D3D39407404A9008A71C
:2074C000D4E0FBA3E0FAA3E0240AF9E43AFA120080D35403C454F0FE9008A7D7E04EF0A325
:2074E000E0F09008A7D4A3E0FAA3E02415F9E43AFA120080D35403C4333354C0FE9008A728
:20750000D7E04EF0A3E0F09008A7CFE0FF9008A7D7E0FAA3E0FB7D081206928DEF60037F1B
:2075200001229008A7CFE075F02FA4242DF9741D35F0FA7B89120080D3D394075003217647
:207540008F9008A7D4E0FBA3E0FAA3E0240CF9E43AFA120080D35403C4F8540FC868FFE47F
:20756000C454F048FE9008A7D4A3E0FAA3E0240BF9E43AFA120080D35403FDEF4DFF9008DE
:20758000A7D7EEF0A3EFF09008A7D4A3E0FAA3E02417F9E43AFA120080D37E0054037806F6
:2075A000C333CE33CED8F9FDAC069008A7D4E0FBA3E0FAA3E02416F9E43AFA120080D37E6A
:2075C0000054037802C333CE33CED8F9FFEE4CFEEF4DFF9008A7D7E04EF0A3E04FF0900844
:2075E000A7CFE075F02FA4242DF9741D35F0FA7B89120080D3D3940A403D9008A7D4E0FBBE
:20760000A3E0FAA3E02418F9E43AFA120080D3540325E025E0FC9008A7D4A3E0FAA3E02424
:207620000DF9E43AFA120080D354034CFE9008A7D7E04EF0A3E0F09008A7D4E0FBA3E0FA14
:20764000A3E02419F9E43AFA120080D3B401259008A7D4A3E0FAA3E0241AF9E43AFA1200A6
:2076600080D35407C454F04480FE9008A7D7E04EF0A3E0F09008A7CFE0FF9008A7D7E0FA0E
:20768000A3E0FB7D091206928DEF60037F01229008A7D0E0FF6401605CEF64076057900803
:2076A000A7D4E0FBA3E0FAA3E02401F9E43AFA12008204FFE5F0540FFCAD079008A7D1E0CF
:2076C000FBA3E0FAA3E0F9120080D3C454F04CFFED9008A7D7CFF0A3EFF09008A7CFE0FFCD
:2076E0009008A7D7E0FAA3E0FB7D061206928DEF60037F01229008A7D4E0FBA3E0FAA3E080
:207700004A4B70149008A7D0E0C454F044809008A7D7F0A3E4F080349008A7D4E0FBA3E0F3
:20772000FAA3E0F9120080D3FD54F0C454F0FB9008A7D0E0C454F04480FEEBFFED540FFD3A
:20774000EF4DFF9008A7D7EEF0A3EFF09008A7CFE0FF9008A7D7E0FAA3E0FB7D05120692F1
:207760008DEF60037F01229008A7D0E0FF64076005EF6404703D9008A7D7E4F0A304F090B5
:2077800008A7D7E07004A3E0640170279008A7CFE0FF9008A96B7401F0A37409F0A374A7C4
:2077A000F0A374D7F07B0F7D0512066992EF60CF7F01229008A7D0E06407707B9008A7CFC9
:2077C000E0FF9008A96B7404F0A37409F0A374A7F0A374D7F0E4FB7D0512066992EF600354
:2077E0007F01229008A7D8E0540FFF9008A7D4E0FBA3E0FAA3E0F9EF120081249008A7CFF3
:20780000E0FF7B097AA779D77D0612068ACAEF60037F01229008A7D7E0540FFEA3E0FF9048
:2078200008A7D4E0FBA3E0FAA3E02401F9E43AFAEE8FF01200827E9008A7D0E0640460037B
:20784000217D289008A7CFE0FF9008A96B7404F0A37409F0A374A7F0A374D7F0E4FB7D0564
:2078600012066992EF60037F01229008A7D8E0540FFF9008A7D4E0FBA3E0FAA3E0F9EF12C0
:207880000081249008A7CFE0FF9008A96B7404F0A37409F0A374A7F0A374D7F07B087D05A1
:2078A00012066992EF60037F01229008A7D4E0FBA3E0FAA3E0F9120080D3FD9008A7D8E081
:2078C000540FC4F8540FC868FFED4F120081249008A7CFE0FF7B097AA779D77D0612068AFD
:2078E000CAEF60037F01229008A7D7E0FEA3E0FFEE540FFCAD079008A7D4E0FBA3E0FAA345
:20790000E02401F9E43AFAEC8DF01200827EEEC45401FF9008A7D1E0FBA3E0FAA3E0F9EFFD
:20792000120081249008A7CFE0FF7B097AA779D77D0712068ACAEF60037F01229008A7D8B3
:20794000E05403FF9008A7D4E0FBA3E0FAA3E02403F9E43AFAEF120081249008A7D7E0FC33
:20796000A3E0FDECC4F854F0C8EDC4540F485403FF9008A7D4E0FBA3E0FAA3E02404F9E42E
:207980003AFAEF12008124EC5403FF9008A7D4E0FBA3E0FAA3E02405F9E43AFAEF12008121
:2079A000249008A7D7E0FCA3E0FDAE047802CEC313CE13D8F95403FF9008A7D4E0FBA3E0E8
:2079C000FAA3E0240EF9E43AFAEF12008124EDAE047806CEC313CE13D8F95403FF9008A739
:2079E000D4E0FBA3E0FAA3E0240FF9E43AFAEF120081249008A7D7E013135403FF9008A73D
:207A0000D4E0FBA3E0FAA3E02410F9E43AFAEF120081249008A7CFE075F02FA4242DF974E8
:207A20001D35F0FA7B89120080D3D394035003217B5F9008A7D7E0FCECC45403FF9008A7B2
:207A4000D4E0FBA3E0FAA3E02406F9E43AFAEF12008124ECC413135403FF9008A7D4E0FB7C
:207A6000A3E0FAA3E02411F9E43AFAEF120081249008A7CFE0FF7B097AA779D77D0812069B
:207A80008ACAEF60037F01229008A7D8E05403FF9008A7D4E0FBA3E0FAA3E02407F9E43A21
:207AA000FAEF120081249008A7D7E0FCA3E0FDECC4F854F0C8EDC4540F485403FF9008A70F
:207AC000D4E0FBA3E0FAA3E02408F9E43AFAEF12008124EC5403FF9008A7D4E0FBA3E0FA67
:207AE000A3E02409F9E43AFAEF120081249008A7D7E0FCA3E0FDAE047802CEC313CE13D824
:207B0000F95403FF9008A7D4E0FBA3E0FAA3E02412F9E43AFAEF12008124EDAE047806CE50
:207B2000C313CE13D8F95403FF9008A7D4E0FBA3E0FAA3E02413F9E43AFAEF1200812490FB
:207B400008A7D7E013135403FF9008A7D4E0FBA3E0FAA3E02414F9E43AFAEF1200812490D6
:207B600008A7CFE075F02FA4242DF9741D35F0FA7B89120080D3D394075003217D289008ED
:207B8000A7D7E0FCECC45403FF9008A7D4E0FBA3E0FAA3E0240AF9E43AFAEF12008124ECC6
:207BA000C413135403FF9008A7D4E0FBA3E0FAA3E02415F9E43AFAEF120081249008A7CF99
:207BC000E0FF7B097AA779D77D0912068ACAEF60037F01229008A7D8E05403FF9008A7D48B
:207BE000E0FBA3E0FAA3E0240BF9E43AFAEF120081249008A7D7E0FCA3E0FDECC4F854F066
:207C0000C8EDC4540F485403FF9008A7D4E0FBA3E0FAA3E0240CF9E43AFAEF12008124ED28
:207C2000AE047802CEC313CE13D8F95403FF9008A7D4E0FBA3E0FAA3E02416F9E43AFAEF44
:207C4000120081249008A7D7E0FEA3E07806CEC313CE13D8F95403FF9008A7D4E0FBA3E05B
:207C6000FAA3E02417F9E43AFAEF120081249008A7CFE075F02FA4242DF9741D35F0FA7BFA
:207C800089120080D3D3940A403C9008A7D7E0FCEC5403FF9008A7D4E0FBA3E0FAA3E024C3
:207CA0000DF9E43AFAEF12008124EC13135403FF9008A7D4E0FBA3E0FAA3E02418F9E43A57
:207CC000FAEF120081249008A7D7E0FEEE9008A7D430E72CE0FBA3E0FAA3E02419F9E43A9D
:207CE000FA740112008124EEC45407FF9008A7D4E0FBA3E0FAA3E0241AF9E43AFAEF802482
:207D0000E0FBA3E0FAA3E02419F9E43AFAE4120081249008A7D4E0FBA3E0FAA3E0241AF97A
:207D2000E43AFAE4120081247F0022E0FBA3E0FAA3E0F97E007F009000FFFD12008645EBCA
:207D4000F0A3EAF0A3E9F09000FFFE12008645EEF0A3EFF09000FFEF120086459000000B7A
:207D60001200866CE4F0A3F0900000191200866CE0FBA3E0FAA3E04A4B701690000016123D
:207D800000866CE0FBA3E0FAA3E0F9120085348010900000191200866CE0FBA3E0FAA3E03A
:207DA000F9900000191200866CEBF0A3EAF0A3E9F07B097A9E79BD900000031200866CEBF5
:207DC000F0A3EAF0A3E9F0900000161200866CE0FBA3E0FAA3E02407217EEE85508385514F
:207DE00082759308E0FBA3E0FAA3E0F9EB8A8389827B097A9E79BD6409700A74BD658270D9
:207E000004749E65837003217F1A9000000B1200866CE0FEA3E04E6003217F1A85508385EF
:207E20005182759308E0FBA3E0FAA3E0F9900000031200866CEBF0A3EAF0A3E9F0855083C8
:207E4000855182759308E0FBA3E0FAA3E0240BF9E43AFA120085349000FFFD12008645EB80
:207E6000F0A3EAF0A3E9F0900000161200866CE0FBA3E0FAA3E0F9C003C002C001900000C5
:207E80001C1200866CE0FBA3E0FAA3E0F5828A838B93D001D002D0031200863E9000000960
:207EA0001200866CEEF0A3EFF0900000091200866CE0FEA3E0FFC3EE648094805013855080
:207EC00083855182759308E0FBA3E0FAA3E0F98021D3EF9400EE64809480402E85508385BB
:207EE0005182759308E0FBA3E0FAA3E02403F9E43AFA12008534855083855182759308EB16
:207F0000F0A3EAF0A3E9F0217DDB9000000B1200866CE4F0A304F0217DDB9000000B1200CF
:207F2000866CE0FEA3E04E6011900000111200866CE0FEA3E04E6002807B900000111200CB
:207F4000866CE0FEA3E04E700C8550838551827593082187B7900000161200866CE0FBA3BD
:207F6000E0FAA3E02405F9E43AFA12008204FFAEF0EE3395E0FDFC7B0990000006120086F4
:207F80006CA982AA83120655089000000D1200866C1200850B74FFFFFEFDFC9000000D124D
:207FA00000866CE0F8A3E0F9A3E0FAA3E0FBC3120083E870097B097A9E79BD2187BF9000FE
:207FC00000131200866CE0FBA3E0FAA3E0F9C003C002C001900000061200866CE0FBA3E078
:207FE000FAA3E0240BF9E43AFA12008551900000031200866CE0FBA3E0FAA3E0F9C003C0EE
:2080000002C001900000061200866CE0FBA3E0FAA3E02406F9E43AFA120085519000000372
:208020001200866CE0FBA3E0FAA3E0F9EB8A8389827B097A9E79BD6409700A74BD65827024
:2080400004749E6583702E900000061200866CE0FBA3E0FAA3E0F9C003C002C00190000040
:20806000161200866CE0FBA3E0FAA3E02407F9E43AFA21814A900000031200866CE0FBA3CE
:20808000E0FAA3E0240BF9E43AFA120085349000FFFD12008645EBF0A3EAF0A3E9F09000AB
:2080A00000091200866CE0FBA3E0FAA3E0240BF9E43AFA12008534C003C002C001900000F7
:2080C0001C1200866CE0FBA3E0FAA3E0F5828A838B93D001D002D0031200863E900000091E
:2080E0001200866CEEF0A3EFF0900000091200866CE0FEC3EE6480948090000006502412DC
:2081000000866CE0FBA3E0FAA3E0F9C003C002C001900000031200866CE0FBA3E0FAA3E0E1
:20812000F980271200866CE0FBA3E0FAA3E0F9C003C002C001900000031200866CE0FBA36C
:20814000E0FAA3E02403F9E43AFA120085517B097A9E79BDC003C002C001900000061200E2
:20816000866CE0FBA3E0FAA3E0F9120085517B097A9E79BDC003C002C00190000006120091
:20818000866CE0FBA3E0FAA3E02403F9E43AFA12008551900000061200866CE0FBA3E0FA00
:2081A000A3E02409F9E43AFAE475F0011200827E900000061200866CE0F9A3E0FAA3E085AA
:2081C0005083855182759308C9218619900000161200866CE0FBA3E0FAA3E02407F9E43A14
:2081E000FA12008534C003C002C001855083855182759308E0FBA3E0FAA3E0F9D082D0833B
:20820000D0E06B7008E965827003EA65837003218788855083855182759308E0FBA3E0FAFB
:20822000A3E02406F9E43AFA12008534E92409F9E43AFA12008204640145F06003218788C9
:20824000855083855182759308E0FBA3E0FAA3E02406F9E43AFA12008534E92406F9E43A53
:20826000FA1200853412008534C003C002C001855083855182759308E0FBA3E0FAA3E02469
:2082800006F9E43AFA12008534D082D083D0E06B7008E965827003EA65836003218517850A
:2082A0005083855182759308E0FBA3E0FAA3E02406F9E43AFA12008534E92406F9E43AFA7E
:2082C00012008534E92403F9E43AFA12008534900000031200866CEBF0A3EAF0A3E9F090EC
:2082E0000000031200866CE0FBA3E0FAA3E02409F9E43AFA12008204640145F06003218325
:20830000AB855083855182759308E0FBA3E0FAA3E02406F9E43AFA12008534E92409F9E41E
:208320003AFAE4F5F01200827E900000031200866CE0FBA3E0FAA3E02409F9E43AFAE4F5A5
:20834000F01200827E855083855182759308E0FBA3E0FAA3E02406F9E43AFA12008534E991
:208360002406F9E43AFA12008534E92409F9E43AFAE475F0011200827E855083855182754F
:208380009308E0FBA3E0FAA3E02406F9E43AFA12008534E92406F9E43AFA1200853485509D
:2083A00083855182759308EB218619855083855182759308E0FBA3E0FAA3E02406F9E43A4B
:2083C000FA12008534E92403F9E43AFA12008534C003C002C001855083855182759308E006
:2083E000FBA3E0FAA3E0F9D082D083D0E06B7008E965827003EA65837068855083855182B4
:20840000759308E0FBA3E0FAA3E02406F9E43AFA12008534855083855182759308EBF0A32D
:20842000EAF0A3E9F0900000161200866CE0FBA3E0FAA3E02407F9E43AFAC002C0018550CD
:2084400083855182759308E0F9A3E0FAA3E09008A9C5C9F0A3EAF0A3E9F0D001D0021204E7
:208460009240855083855182759308E0FBA3E0FAA3E02406F9E43AFA12008534E92409F97A
:20848000E43AFAE4F5F01200827E855083855182759308E0FBA3E0FAA3E02406F9E43AFA13
:2084A00012008534E92406F9E43AFA12008534E92409F9E43AFAE475F0011200827E9000EF
:2084C00000161200866CE0FBA3E0FAA3E02407F9E43AFAC003C002C0018550838551827500
:2084E0009308E0FBA3E0FAA3E02406F9E43AFA12008534E92406F9E43AFA12008534900879
:20850000A9CEEBF0A3EAF0A3E9F0D001D002D0031204877C2181CC85508385518275930853
:20852000E0FBA3E0FAA3E02406F9E43AFA12008534E92406F9E43AFA1200853412008534A0
:20854000900000031200866CEBF0A3EAF0A3E9F0900000031200866CE0FBA3E0FAA3E0241A
:2085600009F9E43AFA12008204640145F06003218623855083855182759308E0FBA3E0FA6A
:20858000A3E02406F9E43AFA12008534E92409F9E43AFAE4F5F01200827E900000031200AB
:2085A000866CE0FBA3E0FAA3E02409F9E43AFAE4F5F01200827E855083855182759308E035
:2085C000FBA3E0FAA3E02406F9E43AFA12008534E92406F9E43AFA12008534E92409F9E4B8
:2085E0003AFAE475F0011200827E855083855182759308E0FBA3E0FAA3E02406F9E43AFA15
:2086000012008534E92406F9E43AFA12008534855083855182759308EBF0A3EAF0A3E9F00C
:208620002181CC855083855182759308E0FBA3E0FAA3E02406F9E43AFA1200853412008594
:2086400034C003C002C001855083855182759308E0FBA3E0FAA3E0F9D082D083D0E06B70DC
:2086600008E965827003EA65837068855083855182759308E0FBA3E0FAA3E02406F9E43A29
:20868000FA12008534855083855182759308EBF0A3EAF0A3E9F0900000161200866CE0FBFC
:2086A000A3E0FAA3E02407F9E43AFAC002C001855083855182759308E0F9A3E0FAA3E090D2
:2086C00008A9CEC9F0A3EAF0A3E9F0D001D0021204877C855083855182759308E0FBA3E08F
:2086E000FAA3E02406F9E43AFA12008534E92409F9E43AFAE4F5F01200827E8550838551C7
:2087000082759308E0FBA3E0FAA3E02406F9E43AFA12008534E92406F9E43AFA12008534F7
:20872000E92409F9E43AFAE475F0011200827E900000161200866CE0FBA3E0FAA3E0240706
:20874000F9E43AFAC003C002C001855083855182759308E0FBA3E0FAA3E02406F9E43AFAEC
:2087600012008534E92406F9E43AFA120085349008A9C5EBF0A3EAF0A3E9F0D001D002D0F2
:2087800003120492402181CC900000161200866CE0FBA3E0FAA3E02407F9E43AFA12008528
:2087A00034E92409F9E43AFAE4F5F01200827E900000061200866CE0FBA3E0FAA3E0F99085
:2087C00000001C020086451206AD64EF4E7003FEFF229008462FE025E0FF9008462EE033A8
:2087E000FE74D62FF58274423EF583759308E0FFA3E0900884E0CFF0A3EFF0900840FBE0BD
:20880000FEA3E0FFC3900884E1E09F900884E0E09E4003219244E0FFA3E0900884E4CFF0C4
:20882000A3EFF07E007F647D007B097A8479EC120089B17B097A6D795590086E57EBF0A391
:20884000EAF0A3E9F02414F9E43AFA74111200812490086E57E0FBA3E0FAA3E0F97404751F
:20886000F0001200827E90086E57E0FBA3E0FAA3E02402F9E43AFAE475F0A21200827E90FA
:20888000086E57E0FBA3E0FAA3E0242AF9E43AFAE4120081241205C16A90086D3FE0FBA332
:2088A000E0FAA3E02408F9E43AFA90088550EBF0A3EAF0A3E9F0900884E0E475F001120085
:2088C00081EEFEE5F025E0FFEE33FE74F02FF58274423EF583759308E0FFA3E0900884E649
:2088E000CFF0A3EFF0E4FFFEFDFC9008855F1200850B900884E6E0FEA3E0FFC394D0EE6464
:208900008094874003218BABEF64EA7003EE64037055900884E1E025E0FF900884E0E03368
:20892000FE74F02FF58274423EF583759308E0FCA3E0FDA3E0FEA3E0FF900885631200853D
:208940000B900884E1E02402F0900884E0E03400F0C3900884E7E094E8FF900884E6E09482
:2089600003CFC394018065900884E6E064037004A3E064ED6003218A9E900884E1E025E0C9
:20898000FF900884E0E033FE74F02FF58274423EF583759308E0FCA3E0FDA3E0FEA3E0FFE6
:2089A000900885631200850B900884E1E02402F0900884E0E03400F0C3900884E7E094E880
:2089C000FF900884E6E09403CFC39403CF9400FE900842CD75F003EF12008528EE75F00382
:2089E000A42583F583759308E0F9A3E0FAA3E09008945DC9F0A3EAF0A3E9F090088563E02F
:208A0000FCA3E0FDA3E0FEA3E0FF7818120083F9E490089460F0A3EFF090088563E0FCA3D8
:208A2000E0FDA3E0FEA3E0FF7810120083F9E490089462F0A3EFF090088563E0FCA3E0FD80
:208A4000A3E0FEA3E0FF7808120083F9E490089464F0A3EFF090088563E0FCA3E0FDA3A3FD
:208A6000E0FEE490089466F0A3CEF07B097A8479EC12008B13900884E8EEF0A3EFF0785B83
:208A80007C857D097B097A4179C97E007F041200805590088555E4F0A37404218D4A9008F5
:208AA00084E6E064037004A3E064EB7075C3900884E7E094E8FF900884E6E09403CFC3941A
:208AC00003CF9400FE900842CD75F003EF12008528EE75F003A42583F583759308E0F9A3CF
:208AE000E0FAA3E09008945DC9F0A3EAF0A3E9F07B097A8479EC12008B13900884E8EEF065
:208B0000A3EFF0785B7C857D097B097A4179CF7E007F0412008055E490088555F0A3F02110
:208B20008F0F900884E6E064037004A3E064EC6003218F8AC3900884E7E094E8FF9008842D
:208B4000E6E09403CFC39404CF9400FE900842CD75F003EF12008528EE75F003A42583F5D9
:208B600083759308E0F9A3E0FAA3E09008945DC9F0A3EAF0A3E9F07B097A8479EC12008BCA
:208B800013900884E8EEF0A3EFF0785B7C857D097B097A4279EA7E007F04120080559008E1
:208BA0008555E4F0A304F0E4218F0F900884E6E0FEA3E0FFC394B8EE6480948B4003218D7A
:208BC000C0C3EF94D0FFEE9407CFC39401CF9400FE9008455875F003EF12008528EE75F011
:208BE00003A42583F583759308E0F9A3E0FAA3E09008945DC9F0A3EAF0A3E9F0900884E18D
:208C0000E025E0FF900884E0E033FE74F02FF58274423EF583759308E0FFA3E090089460EF
:208C2000CFF0A3EFF07B097A8479EC12008B13900884E8EEF0A3EFF090088555E4F0A3749B
:208C400006F0900884E6E0FEA3E08EF0120085CD8C6C07D18C8A07D28CF007D38D5507D407
:208C60008CAC07D58CCC07D600008F8A785B7C857D097B097A4079FD7E007F04120080559C
:208C800090088557E4F0A304801D785B7C857D097B097A4079937E007F0412008055900824
:208CA0008557E4F0A37402F0E4218F13785B7C857D097B097A4279DE7E007F04120080557B
:208CC00090088557E4F0A37403218EAC785B7C857D097B097A4279E27E007F0412008055FA
:208CE00090088557E4F0A37404F0E47F08218F7F900884E1E025E0FF900884E0E033FE7425
:208D0000F02FF58274423EF583759308E0FFA3E090088559CFF0A3EFF0900884E1E004F057
:208D20007007900884E0E004F01206A0E6785B7C857D097B097A4679137E007F0412008091
:208D40005590088555E4F0A37403F0E4A3F0A3F07F02218F7F900884E1E025E0FF900884B7
:208D6000E0E033FE74F02FF58274423EF583759308E0FFA3E090088559CFF0A3EFF09008CB
:208D800084E1E004F07007900884E0E004F07B097A4179D31206A0EC785B7C857D097B0946
:208DA0007A4279E67E007F041200805590088555E4F0A37402F0E4A3F0A3F07F02218F7FA7
:208DC000C3900884E7E094B8FF900884E6E0940BCFC39401CF9400FE9008460075F003EF64
:208DE00012008528EE75F003A42583F583759308E0F9A3E0FAA3E09008945DC9F0A3EAF0F2
:208E0000A3E9F0900884E1E025E0FF900884E0E033FE74F02FF58274423EF583759308E082
:208E2000FFA3E090089460CFF0A3EFF07B097A8479EC12008B13900884E8EEF0A3EFF09058
:208E4000088555E4F0A37406F0900884E6E0FEA3E08EF0120085CD8E6B0BB98E8F0BBA8EDD
:208E6000B30BBB8F170BBC00008F8A785B7C857D097B097A4279DE7E007F0412008055908A
:208E8000088557E4F0A37405F0E47F02218F7F785B7C857D097B097A4279E27E007F041272
:208EA00000805590088557E4F0A37406F0E47F04218F7F900884E1E025E0FF900884E0E035
:208EC00033FE74F02FF58274423EF583759308E0FFA3E090088559CFF0A3EFF0900884E1C5
:208EE000E004F07007900884E0E004F01206A0E6785B7C857D097B097A4679137E007F048E
:208F00001200805590088555E4F0A37403F0E4A3F0A3F07F018068900884E1E025E0FF9037
:208F20000884E0E033FE74F02FF58274423EF583759308E0FFA3E090088559CFF0A3EFF015
:208F4000900884E1E004F07007900884E0E004F07B097A4179D31206A0EC785B7C857D0970
:208F60007B097A4279E67E007F041200805590088555E4F0A37402F0E4A3F0A3F07F01FE93
:208F8000FDFC9008855F1200850BE4900884EAF0A3F09008462EE0FEA3E0FF900884E2EEF5
:208FA000F0A3EFF0900884E0E0FCA3E0FDEF25E0FFEE33FE74D62FF58274423EF583759371
:208FC00008ECF0A3EDF0900884E3E0FF12068367EF4E7003FEFF22900884E3E0FF1206AFD9
:208FE0005090086E57E0FBA3E0FAA3E02404F9E43AFA1200843CC3900884E7E094D090083C
:2090000084E6E0648094875035900884E3E0FF1206AF419008855FE0F8A3E0F9A3E0FAA3AC
:20902000E05FFFEA5EFEE95DFDE85CFCE4FBFAF9F8C3120083E8600321914C2187FB900883
:2090400084E6E0FEA3E0FF64BB7003EE640B6006BE0B38BFBC35900884E3E0FF1206AF4B50
:209060009008855FE0F8A3E0F9A3E0FAA3E05FFFEA5EFEE95DFDE85CFCE4FBFAF9F8C3125A
:209080000083E8600321914C2187FB900884E6E0FEA3E0FF64D37003EE64076006BE07359C
:2090A000BFD432900884E3E0FF1206AF469008855FE0F8A3E0F9A3E0FAA3E05FFFEA5EFE8C
:2090C000E95DFDE85CFCE4FBFAF9F8C3120083E8707A2187FBC3900884E7E094B890088468
:2090E000E6E06480948B5032900884E3E0FF1206AF469008855FE0F8A3E0F9A3E0FAA3E06A
:209100005FFFEA5EFEE95DFDE85CFCE4FBFAF9F8C3120083E870352187FB900884E3E0FFF8
:209120001206AF4B9008855FE0F8A3E0F9A3E0FAA3E05FFFEA5EFEE95DFDE85CFCE4FBFA4D
:20914000F9F8C3120083E870032187FB1206ADA6EF64014E900884E3700EE0FF1206AFADEB
:20916000AC06AD07E4FF800CE0FF1206AFADAC06AD077F0112068F4F90088550E0F9A3E022
:20918000FAA3E090084665C9F0A3EAF0A3E9F0A37409F0A37485F0A37453F0A37409F0A3B4
:2091A0007484F0A374ECF090088555E0FFA3E09008466ECFF0A3EFF090088557E0FFA3E09D
:2091C00090084670CFF0A3EFF0900884E2E0FFA3E090084672CFF0A3EFF07B097A85795BB8
:2091E0001205B289900884EAEEF0A3EFF0BEFF2FBFFF2C900884E4E0FCA3E0FD9008462F78
:20920000E025E0FF9008462EE033FE74D62FF58274423EF583759308ECF0A3EDF080259050
:20922000087D8CE0FCA3E0FDA3E0FEA3E02401FFE43EFEE43DFDE43CFC90087D8C12008507
